:100000000C9492120C948B840C9460840C94358420
:100010000C940A840C94DF830C94B4830C9489832D
:100020000C945E830C94C3120C94C3120C94C312F0
:100030000C94C3120C94C3120C94C3120C94C312EC
:100040000C94C3120C94C3120C94C3120C94C312DC
:100050000C94C3120C94C3120C94C3120C9495AE5E
:100060000C94C3120C94D08A0C94A68A0C94C312DC
:100070000C94C3120C94C3120C94C3120C94C312AC
:100080000C94C3120C94C3120C94C3120C94C3129C
:100090000C94C3120C94C3120C94C3120C940D2A2A
:1000A0000C94C3120C94C3120C94C3120C94C3127C
:1000B0000C94C3120C94C3120C94C3120C94C3126C
:1000C0000C94C3120C94C3120C94C3120C94C3125C
:1000D0000C94C3120C94C3120C94C3120C94C3124C
:1000E0000C94C31207634236B79BD8A71A396856D7
:1000F00018AEBAAB558C1D3CB7CC5763BD6DEDFD4A
:10010000753EF6177231BF000000803F0800000006
:10011000BE922449123EABAAAA2ABECDCCCC4C3EFC
:1001200000000080BEABAAAAAA3E00000000BF00EB
:100130000000803F0000000000084178D3BB4387E7
:10014000D1133D190E3CC3BD4282AD2B3E68EC82FB
:1001500076BED98FE1A93E4C80EFFFBE01C4FF7F80
:100160003F00000000000C94E7610C9403380C94ED
:100170006F360C94B71A0C94644D0C941C160C94A6
:1001800042480C9464200C94957B0C94957A0C94C2
:10019000BF410C94A4760C9407AA0C9465680C9447
:1001A0005A990C9453150C945A130C94B2150C9440
:1001B000EF380C9469140C94F5210C94B6B70C9498
:1001C000DB120C94A5190C9498560C94193A0C94C3
:1001D0000E1A0C94B8180C94A6180C9462180C946F
:1001E000AE3F0C9460170C94E07C0C94C3610C94AB
:1001F0007C410C9400130C94E23B0C946B7B0C94AC
:100200007E560C94CB370C94E0390C9457150C9413
:100210002B1F0C940E1D0C94537D0C943C600C947D
:10022000057C0C9443990C9415250C949D600C94BA
:10023000C9410C94DAA70C94B5410C949E8C0C9493
:10024000AF180C9479990C9454390C944FA40C94D5
:1002500045560C9420200C948E7C0C949A550C944A
:1002600082330C94C5120C945EBB0C94101D0C943C
:10027000861B0C9482A40C9488C70C94874C0C9415
:1002800078A40C9490220C948C180C94A14D0C948E
:10029000A1130C94ADA70C949B390C94C6610C94DB
:1002A00000380C948C9D0C947EA40C94AF220C947A
:1002B000741F0C94D5750C9449130C94647A0C94A7
:1002C00043180C946E390C9406160C944A360C9410
:1002D000506F0C946E150C9414190C949E8E0C9403
:1002E000F5120C943B150C94A2410C9418320C940A
:1002F000EC190C9486150C94D0150C948C7B0C94F2
:1003000099C50C9493990C94237A0C9423600C94C3
:100310001F170C9457360C94F75B0C9463150C94D0
:10032000BBB50C944B390C94CD380C94FF8C0C94C9
:10033000367A0C9447470C94AC390C948C560C9438
:10034000B6170C940DC50C9412BE0C9457170C9450
:100350005D170C94F0400C944A8D0C94118D0C9404
:100360005F140C94D97C0C94D27B0C9429180C94B7
:1003700074A40C94D0BF0C94EC320C94DA6E0C94F0
:100380006F560C947C390C948F410C9415390C9455
:1003900034150C94CB410C94374D0C948F7B0C94FA
:1003A0000F480C94857B0C94B6600C94402F0C94F1
:1003B000F65A0C94CC170C945F710C94EA240C94AC
:1003C000A9150C941E7C0C94D7A70C94F9160C94C8
:1003D0003C990C94FF380C94CD7A0C9451360C94C3
:1003E000DC310C947C5A0C940AAA0C94393A0C9483
:1003F000779D0C94701B0C942A320C9449170C9422
:1004000083240C948E380C94CE300C943EA90C941A
:1004100058A40C9458560C94BA240C947DA40C94B3
:10042000121D0C94AF700C9466330C9446150C940A
:1004300068610C942B390C9472150C94CC1A0C94A2
:1004400062140C94699D0C944A130C94A7350C9477
:10045000D5330C943F170C94A4380C94877A0C94E1
:1004600058410C943CC50C9470600C94CE4C0C9488
:100470004F150C949D7C0C94F8600C944BA40C9438
:1004800013680C941A7B0C9443A40C94611F0C9475
:10049000027F0C94939D0C9460360C9452240C941F
:1004A000629D0C949E4D0C94C1150C9438150C94BF
:1004B0004F410C9418240C9412AA0C9405170C9418
:1004C000F7140C94DF120C94377A0C94E2390C94E4
:1004D000B58C0C9415160C9474130C94B84E0C94A3
:1004E0008B7D0C948B5A0C942A680C94E0A70C9486
:1004F0007F320C94737D0C94CF380C9447A40C94E9
:1005000033150C947CC00C946AA40C94FD4C0C9490
:1005100019380C94859D0C949D1B0C94D7550C9404
:1005200000C40C9401170C94AB390C9466A40C9481
:10053000871F0C9461150C9473170C9409170C9475
:1005400006150C9400320C94707C0C94D13C0C94E5
:100550001A180C940DAA0C9437150C947B560C9415
:1005600086170C94C2C50C94C77C0C94CE280C94AE
:1005700070A40C946D130C9452A40C94BC4E0C9467
:10058000544D0C94C9150C94B64E0C944B330C94EA
:10059000FB150C9407C50C944B130C940D180C947C
:1005A000958C0C9431560C941BC50C941A610C94C8
:1005B00089560C945B170C9416470C94FD1A0C94F6
:1005C00083380C943DA40C94B4C50C94E6370C9479
:1005D00061410C94F5160C94ED5F0C94201F0C9463
:1005E000709D0C94E67D0C940D170C94737A0C940A
:1005F00058BB0C948D340C946A410C9404AA0C944E
:100600007F4D0C94855A0C9462A40C9496390C94EA
:10061000FC320C94642C0C945CA40C9491860C9485
:1006200033610C94FD160C94CD470C94307E0C94E1
:10063000AE4D0C9466150C94F0150C949A230C9402
:1006400076150C94B75F0C94C0610C94444C0C94D8
:1006500056990C94848C0C9487190C94C0190C94A2
:10066000357A0C94E31B0C948A390C9437A90C94BA
:10067000C0384E414E494E495459494E46CDCCCCD6
:100680003D0AD7233C17B7D13877CC2B329595E666
:10069000241FB14F0A000020410000C84200401C46
:1006A0004620BCBE4CCA1B0E5AAEC59D746364691D
:1006B0006E6F70737578585B00454F46002F004988
:1006C0006E3A20003D00494E3A003D004C454741FE
:1006D000435920494E3A00000020002300260029FB
:1006E000002C002F00320000010000030106010968
:1006F00001204E6F20656D69742064617461210072
:1007000020436F756E74657220747970652E207643
:10071000616C3D00494E3A0020436F756E746572FE
:1007200020747970652E20494E434F5252454354F0
:1007300020496E74657272757074206E756D626595
:1007400072212121004952513A002D3E0020002300
:10075000002D3E00200050656E6465643A20230041
:10076000536574436D643A00737566666978436FC8
:1007700064653A0020666F7220286D73293A004341
:1007800054524C3A205363686564756C6520636D00
:10079000642000206D73203A0041726D656420660C
:1007A0006F7220002044697361726D65640020746B
:1007B000696D653A004354524C3A205265733A00D1
:1007C0003D0050696E3A004354524C3A20436F6DDD
:1007D0006D616E6420626C6F636B6564206279206A
:1007E000647269766572206F72206368616E6E65EF
:1007F0006C2066726F7A656E004354524C3A204FFB
:100800004E3A416C72656164792041637469766522
:100810000A004354524C3A2048414C543A416C72BD
:100820006561647920496E6163746976650A004385
:1008300054524C3A20584F4E3A2044697361626CCE
:1008400065640A004354524C3A20584F4E3A416C6A
:100850007265616479204163746976650A00435466
:10086000524C3A20584F464620736B69707065644D
:100870002E205072657620636D643A004354524CCA
:100880003A205475726E6564206F66662066726FDA
:100890006D3A004354524C3A20526573746F72653E
:1008A000642066726F6D3A004354524C3A20496797
:1008B0006E6F7265642C206368616E6E656C206378
:1008C0006D643D0020457865633A004354524C3ACC
:1008D000204163746976653A004354524C3A20488B
:1008E000414C543A416C726561647920496E616390
:1008F000746976650A004354524C3A20584F4E3A78
:100900002044697361626C65640A004354524C3A36
:1009100020584F4E3A416C7265616479204163748E
:100920006976650A004354524C3A20584F46462097
:10093000736B69707065642E205072657620636DEC
:10094000643A004354524C3A205475726E656420E8
:100950006F66662066726F6D3A004354524C3A20BF
:10096000526573746F7265642066726F6D3A0043EE
:1009700054524C3A204E6F7420656E6F7567682034
:100980006D656D6F727920666F722067726F75701A
:10099000206F7065726174696F6E00496E76616C6C
:1009A00069642061726700496E76616C69642061D8
:1009B0007267004354524C3A20556E6B6E6F776EDF
:1009C0002073756666697800536B69707065642082
:1009D000686F6D696520737475666600200020532A
:1009E00075623D00204974656D3D004354524C3A98
:1009F0002052414D3D004354524C3A204F75744FA4
:100A0000664D656D6F72793A2000282D29200028E7
:100A10002B2920002076616C7565206973200020E9
:100A2000756E6B6E6F776E0A005D3D005B0020692E
:100A30006E76616C6964002000206F6B003A0020C4
:100A40006661696C6564003A005265747279696E1A
:100A50006720434D440A004354524C2F706F6C6C16
:100A60003A204F75744F664D656D6F72793A20006C
:100A7000207365632072656D61696E696E670053EE
:100A800074617475732064656666657265640A00D6
:100A9000444D58000000000000444D585247425752
:100AA0000000444D5852474200000050574D00008E
:100AB000000000004D42555344494D000054484544
:100AC000524D4F00000052454C4159000000004774
:100AD000524F555000000000564354454D50000001
:100AE000004D42555356430000004143484149459B
:100AF0005200005350494C45440000004D4F544FA4
:100B000052000000005049440000000000004D4227
:100B100055530000000000554152544252444700D2
:100B200052454C415950574D00444D585247425739
:100B3000570056454E545300000000454C45564161
:100B4000544F5200434F554E544552000048554DA6
:100B50000000000000004D4552435552590000204E
:100B6000002D3E00436F6E76657274696E672000DB
:100B70002D3E0057726F6E672041737369676E6D0B
:100B8000656E742000524742783A20004853562040
:100B900064697361626C65640020764C6576656C8F
:100BA0003A0020436F6E76563A0020436F6E7653BC
:100BB0003A0020486F743A00436F6C643A00204357
:100BC0006F6E76657274656420563A00436F6E7678
:100BD000657274656420533A002D3E0057726F6E43
:100BE000672041737369676E6D656E7420002D3EDA
:100BF0000057726F6E672041737369676E6D656E23
:100C000074200053617665643A0020537566663A35
:100C1000002041543A00206973200044656C6574DB
:100C2000696E6720636F6E662E2052414D2077619A
:100C3000733A0053746F70706564006E6F74686906
:100C40006E6720746F2073746F700053746F7070D0
:100C5000696E67206368616E6E656C73202E2E2E40
:100C6000004E6F7420756E6C6F636B656420696EE7
:100C700020313073202D20636F6E74696E7565208E
:100C80002E2E2E00556E6C6F636B696E6720636F3E
:100C90006E666967202E2E2E00436F6E6669672090
:100CA0006368616E676564206C6F63616C6C792C3E
:100CB00020706F7274616C2064697361626C65642A
:100CC000002F636F6E6669672E6A736F6E007265C0
:100CD000626F6F742000436D643A20002F636F6D64
:100CE0006D616E642F002F72616D2F002F69746526
:100CF0006D2F002F6974656D2F004C6F63617469EF
:100D00006F6E3A20687474703A2F2F6C617A79682C
:100D10006F6D652E72752F707761003F6D61633D59
:100D2000002669703D0026706F72743D00266E616A
:100D30006D653D002F002000436F6D706C6574651C
:100D40002E2052656D6F766520746F706963200088
:100D500024636F6D6D616E6400536B697070696EB2
:100D6000672E2E00436C65616E557020726574614C
:100D7000696E656420746F70696320002200220030
:100D80004F75744F664D656D6F727921005D20005F
:100D90003A5B000A005D00456D7074793A205B0093
:100DA0000A003A004D41433A0055445020537973AC
:100DB0006C6F6720696E697469616C697A65642E0D
:100DC0000A005379736C6F6720706172616D733ABA
:100DD0000043757272656E74204C414E20636F6ED5
:100DE0006669672869702C646E732C67772C73753D
:100DF000626E6574293A000A5573652074686573DC
:100E00006520636F6D6D616E64733A202768656C51
:100E10007027202D207468697320746578740A2700
:100E20006D61632064653A61643A62653A65663A69
:100E300066653A3030272073657420616E642073D4
:100E4000746F7265204D41432D61646472657373E4
:100E500020696E20454550524F4D0A276970205B2E
:100E600069705B2C646E735B2C67775B2C737562A7
:100E70006E65745D5D5D5D27202D20736574207344
:100E800074617469632049500A277361766527206D
:100E90002D20736176652063757272656E742063B0
:100EA0006F6E66696720696E204E5652414D3B2039
:100EB0004F4E7C4F4646202D20656E61626C652F3B
:100EC00064697361626C65206175746F73617665C6
:100ED0000A2767657427205B636F6E666967206108
:100EE0006464725D27202D2067657420636F6E66D1
:100EF00069672066726F6D207072652D636F6E6614
:100F00006967757265642055524C20616E64207368
:100F1000746F726520616464722C204F4E7C4F4662
:100F200046202D20656E61626C652F646973616275
:100F30006C6520646F776E6C6F6164206F6E2073D8
:100F40007461727475700A276C6F616427202D209C
:100F50006C6F616420636F6E6669672066726F6D87
:100F6000204E5652414D0A2770776427202D206469
:100F70006566696E6520616E642073746F726520AA
:100F80004D5154542070617373776F72640A276FE8
:100F9000746170776427202D20646566696E652012
:100FA000616E642073746F72652048545450204100
:100FB00050492070617373776F72640A276C6F6792
:100FC000205B73657269616C5F6C6F676C657665D9
:100FD0006C5D205B7564705F6C6F676C6576656CCB
:100FE0005D27202D20646566696E65206C6F672023
:100FF0006C6576656C2028302E2E37290A276B69A0
:101000006C6C27202D20746573742077617463687D
:10101000646F670A27636C65617227202D20636CFB
:1010200065617220454550524F4D0A2773656172C4
:10103000636827202D2073656172636820312D77E6
:10104000697265206465760A277265626F6F74271E
:10105000202D207265626F6F7420636F6E74726FE3
:101060006C6C657200536F6674207265626F6F748A
:10107000696E672E2E2E00206E6577002069732022
:10108000003157543A003157543A20536561726326
:1010900068696E67206465760052414D3D000A53D1
:1010A00079736C6F6720000A312D776972652000B3
:1010B0000A6D71747420000A696E70757473200073
:1010C0000A6974656D7320000A436F6E66696775FF
:1010D0007265643A003157543A2073657475702014
:1010E0007265736F6C7574696F6E20003157543A76
:1010F000204453323438322D313030206E6F74201A
:1011000070726573656E74003157543A20445332DF
:101110003438322D313030204932432072657374B7
:101120006F726564003157543A20427573207265BE
:10113000736574206572726F72003157543A2042A1
:10114000757320526573657420646F6E6500315746
:10115000543A204453323438322D313030207072BA
:101160006573656E742C20726573657400457272C8
:101170006F7220312D7720696E6974003157543AAF
:10118000204453323438325F3130305F4932435F6C
:10119000544F5F31575F42524944474520696E6959
:1011A00074003B003D0050696E3A003B003D4C4FDF
:1011B0005700546865726D6F3A004F6E652077690D
:1011C00072652052656164790A004170706C7969BA
:1011D0006E6720636F6E66696700436F6E6669674E
:1011E000206175746F736176653A000A5379736C88
:1011F0006F67206465627567206C6576656C3A0080
:1012000053657269616C206465627567206C6576F0
:10121000656C3A0053617665640A00536574206416
:10122000796E616D69632049500A00454550524FFF
:101230004D20636C65617265640A004D5154542001
:1012400050617373776F7264207570646174656444
:101250000A004F54412050617373776F7264207598
:101260007064617465640A00636F756C64206E6FEE
:10127000742070617273653A200055706461746502
:10128000640A004E6F2049502061647265737300D8
:1012900052656C656173696E6720736F636B65740B
:1012A00020616E64207265747279002053617665E6
:1012B00064004C6F6164696E672048545450206329
:1012C0006F6E666967206F6E2073746172747570DB
:1012D0003A000000000000000000004F4E00000037
:1012E000000000004F464600000000000052455339
:1012F000540000000000544F47474C450000004890
:10130000414C540000000000584F4E000000000007
:1013100000584F46460000000000494E43524541E8
:10132000534500444543524541534500454E4142D3
:101330004C4500000044495341424C450000554E85
:10134000465245455A4500465245455A450000001B
:101350004155544F000000000046414E5F4F4E4C37
:1013600059004849474800000000004D4544495590
:101370004D0000004C4F5700000000000048454160
:10138000540000000000434F4F4C00000000004498
:10139000525900000000000053544F50000000005C
:1013A0000052474200000000000048535600000071
:1013B0000000002B002D00455461673A200047656E
:1013C0007420455441473A2000485454502F312E40
:1013D000310025733A2025730D0A002048545450DB
:1013E0002F312E310D0A486F73743A2025730D0A80
:1013F0004163636570743A202A2F2A0D0A436F6E89
:101400006E656374696F6E3A20636C6F73650D0A65
:101410000025730020000D0A0047455400666169ED
:101420006C656420746F20636F6E6E6563740A0070
:101430004552524F523A205365727665722072655A
:101440007475726E65642000436F6E666967206E06
:101450006F74206368616E6765640A00446F6E652F
:101460002E0A00436F6E6669672070617273696E41
:1014700067206661696C65640A00676F7420436F5A
:101480006E6669670A006874747020726574636FB1
:1014900064652000667265652000436F6E6669674B
:1014A000205552493A20687474703A2F2F00204416
:1014B000656661756C7420636F6E6669672073651D
:1014C0007276657220757365643A20006C617A7972
:1014D000686F6D652E7275000A282D294D554C5484
:1014E0004956454E54000A282B2950574D5F524506
:1014F0004C4159000A282D294D444E53000A282DED
:101500002955415254425249444745000A282B2943
:101510005359534C4F47000A282D29504944000A7B
:10152000282D294D43503233303137000A282D29D8
:101530004152544E4554000A282B294F5441000A69
:10154000282D29535049204C4544000A282D294D67
:101550004F544F5220435452000A282D2941432012
:101560004841494552000A282D2943435338313117
:1015700020262048444331303830000A282B295295
:101580004553544152545F4C414E5F4F4E5F4D5155
:1015900054545F4552524F5253000A282D29484156
:1015A000524452455345542C207573696E6720731D
:1015B0006F6674000A282B29434F554E544552003C
:1015C0000A282D29444854000A282B294453323430
:1015D00038322D313030000A282B294F57495245D7
:1015E000000A282D2949504D4F44425553000A28DE
:1015F0002D294D4F44425553000A282D29444D585A
:10160000000A282B2957697A6E65743578303000C6
:101610000A282B294672656552616D207072696EC9
:1016200074696E67000A282B295741544348444F78
:1016300047006C617A79686F6D652E7275000A4398
:101640006F6E666967207365727665723A00323034
:10165000313130334C0020432B2B20766572736977
:101660006F6E3A00353233356262365F3230323374
:101670002D31312D3137000A4C617A79686F6D65F3
:101680002E7275204C6967687448756220636F6EAE
:1016900074726F6C6C65722000204F464600204FBC
:1016A0004E002042595041535300757074696D6566
:1016B000006672656568656170002054696D6572C9
:1016C0003A00204C6F636B733A002000204C6F632C
:1016D0006B733A000A52414D3D00204578706972A3
:1016E00065640A00202D746172676574207A6F6EDC
:1016F000652D0020416C61726D20457870697265BE
:10170000640A0020636D643A00204375723A002039
:101710005365743A00536176656420746F204545C3
:1017200050524F4D00536176696E6720636F6E664D
:10173000696720746F20454550524F4D2E2E004C46
:101740006F6164656420455441473A004E6F2073D1
:10175000746F72656420636F6E666967004C6F61B9
:101760006465642066726F6D20454550524F4D0090
:101770006C6F6164206661696C6564004A534F4E0A
:10178000206465746563746564004C6F6164696EA0
:101790006720436F6E6669672066726F6D204545EE
:1017A00050524F4D00556E6B6E6F776E207375669D
:1017B0006669782000556E6B6E6F776E20636D647E
:1017C0002000436F756E7465723A200020696E695F
:1017D000740052656C61792D4F757420230020735D
:1017E000746F700052656C61792D4F757420230001
:1017F0003D3E003A0070756220616374696F6E202F
:101800000069646C65006F66660068656174696E86
:10181000670066616E00647279696E6700636F6F5E
:101820006C696E670020697320004F757420005545
:101830006E6B6E6F776E20737566666978200055E3
:101840006E6B6E6F776E20636D64200061637469E8
:101850006F6E0072656C61794374723A2000207279
:10186000656164206572726F7220666F7220003E3F
:101870002000203C003157543A003157543A206E32
:101880006F7420696E6974003157543A2042555381
:10189000592074696D656F7574003157543A20444E
:1018A00053323438325F4552524F525F434F4E46A7
:1018B0004947003157543A20312D776972652073BA
:1018C000686F72746564005B305D3A2000202D20E3
:1018D0002D202D20EFBBBF003E003E31202D2000EB
:1018E0000000000000636D64000073657400007602
:1018F000616C000064656C0000485356000052475C
:1019000042000066616E00006D6F64650063747272
:101910006C006875650000736174000074656D701B
:1019200000726177000020002E00696E00735F6F07
:101930007574006D79686F6D65004354524C2F6566
:101940007865633A204F75744F664D656D6F727997
:101950003A2000202D3E2000456D69743A203C005D
:10196000202D3E20004974656D436D643A200020AF
:101970002D3E20004974656D3A20003157543A20BD
:10198000427573207265736574206572726F7200A0
:101990003157543A20427573205265736574206440
:1019A0006F6E65003157543A204453323438322038
:1019B00070726573656E742C20726573657400496E
:1019C000324320526573657400005EBCE2613FDD06
:1019D00083C29C7E20A3FD1F419DC3217FFCA240AA
:1019E0001E5F01E3BD3E6082DC237D9FC1421CFE81
:1019F000A0E1BF5D0380DE3C62BEE0025CDF81638C
:101A00003D7C22C09E1D43A1FF4618FAA427799B66
:101A1000C584DA3866E5BB5907DB856739BAE40661
:101A2000581947A5FB7826C49A653BD987045AB84C
:101A3000E6A7F91B45C6987A24F8A6441A99C72543
:101A40007B3A6486D85B05E7B98CD2306EEDB35132
:101A50000F4E10F2AC2F7193CD114FADF3702ECC11
:101A600092D38D6F31B2EC0E50AFF1134DCE907218
:101A70002C6D33D18F0C52B0EE326C8ED0530DEFF3
:101A8000B1F0AE4C1291CF2D73CA947628ABF517F6
:101A9000490856B4EA6937D58B5709EBB536688AD9
:101AA000D495CB2977F4AA4816E9B7550B88D634D4
:101AB0006A2B7597C94A14F6A8742AC896154BA9BB
:101AC000F7B6E80A54D7896B353E3E2000496E765A
:101AD000616C696420636F6D6D616E64003E3E3EB3
:101AE000004E6F204D414320636F6E6669677572CB
:101AF00065643A20736574206669726D77617265FA
:101B00002773204D41430A00454550524F4D2073E5
:101B100069676E6174757265206F6B00496E6974D8
:101B200069616C697A696E6720454550524F4D2E48
:101B300000476F7420495020616464726573733A82
:101B400000276970205B69705B2C646E735B2C6787
:101B5000775B2C7375626E65745D5D5D5D27202D0E
:101B600020736574207374617469632049500A009E
:101B70004661696C656420746F20636F6E66696787
:101B80007572652045746865726E65742075736939
:101B90006E6720444843502E20596F752063616E54
:101BA00020736574206970206D616E75616C6C794D
:101BB0002100204D41534B3A002047573A00204422
:101BC0004E533A004C6F616465642066726F6D20FD
:101BD000666C6173682049503A000A75736573201A
:101BE000444843500A005374617274696E67206CF4
:101BF000616E004142434445464748494A4B4C4D7B
:101C00004E4F505152535455565758595A6162636A
:101C10006465666768696A6B6C6D6E6F707172730C
:101C20007475767778797A3031323334353637389F
:101C3000392B2F3D00426173696320006172647526
:101C4000696E6F3A004F544120696E697469616C26
:101C5000697A65640A0044454641554C54207061D8
:101C60007373776F726420666F72204F5441204106
:101C700050492E20557365206F746170776420631E
:101C80006F6D6D616E6420746F2073657400706198
:101C90007373776F726400546F6F206D616E79207B
:101CA0004D51545420636F6E6E656374696F6E207E
:101CB0006572726F72732E20526573746172742034
:101CC0004C414E002074727920616761696E206911
:101CD0006E2035207365636F6E6473006661696C96
:101CE00065642C2072633D004177616974696E6799
:101CF00020666F722072657461696E656420746F0E
:101D00007069637300636F6E6E65637465642061F0
:101D1000732000202E2E2E0020757365723A003A33
:101D2000000A417474656D7074696E67204D51547A
:101D30005420636F6E6E656374696F6E20746F20DC
:101D400000646973636F6E6E6563746564005573D8
:101D5000696E67204D5154542070617373776F72B0
:101D6000642066726F6D20636F6E666967004465FC
:101D700076696365204E616D653A004174206C653B
:101D800061737420646576696365206E616D65209A
:101D9000616E642062726F6B6572204950206D75B0
:101DA000737420626520636F6E666967757265641F
:101DB00000757074696D652C667265656865617023
:101DC0000024737461747300353233356262365F98
:101DD000323032332D31312D3137004C6967687420
:101DE0004875622000246E616D65007265616479DA
:101DF0000024737461746500526562696E642073B7
:101E00007563636573732E20495020616464726545
:101E100073733A004572726F723A20726562696E2E
:101E200064206661696C0052656E65776564207335
:101E30007563636573732E20495020616464726515
:101E400073733A004572726F723A2072656E6577ED
:101E50006564206661696C000A4E6F206C696E6B68
:101E60000033307320454550524F4D206973206E2A
:101E70006F742072656C6F616465642E20526562B8
:101E80006F6F7400416363657074696E6720636F80
:101E90006D6D616E64732E2E2E0A004E6F204D51B3
:101EA000545420636F6E66696775726564004C6F89
:101EB0006164696E6720636F6E6669672066726F22
:101EC0006D20706F7274616C2064697361626C65FF
:101ED000642E2075736520676574204F4E20746FE3
:101EE00020656E61626C6500436F6E66696720698C
:101EF000732076616C696400436F6E74696E7565FA
:101F000020776974682070726576696F75736C7973
:101F1000206C6F6164656420636F6E6669670000A2
:101F2000002100240027002A002D0030003300018A
:101F3000010000040107010A010000220025002819
:101F4000002B002E003100340002010000050108C2
:101F5000010B01050505050705080808080202022E
:101F6000020A0A0808040404040101010101010134
:101F7000010303030303030303040707070C0C0C0B
:101F80000C0C0C0C0C0202020206060606060606E3
:101F9000060B0B0B0B0B0B0B0B0102102020080880
:101FA00010204010204080020102010804020101BB
:101FB00002040810204080804020100804020180A4
:101FC00004020180402010080402010804020101FB
:101FD0000204081020408001020408102040800004
:101FE000000A0B02090C0D0E080703040100000093
:101FF00000000000000000000000000000000000E1
:10200000000000000000000000000012111000009D
:1020100000000000000000000000000000000000C0
:1020200000000000002F64617461002F736B657401
:102030006368004163636573732D436F6E74726FE1
:102040006C2D526571756573742D5072697661746B
:10205000652D4E6574776F726B3A207472756500EA
:102060004163636573732D436F6E74726F6C2D41A2
:102070006C6C6F772D486561646572733A202A0035
:102080004163636573732D436F6E74726F6C2D4182
:102090006C6C6F772D4D6574686F64733A20504F88
:1020A00053542C4745542C4F5054494F4E530041E4
:1020B00063636573732D436F6E74726F6C2D416C27
:1020C0006C6F772D43726564656E7469616C733AE9
:1020D0002074727565004F5054494F4E530044456B
:1020E0004C455445005055540047455400504F53FB
:1020F0005400617574686F72697A6174696F6E3AC1
:102100002000417574686F72697A6174696F6E3A04
:102110002000436F6E74656E742D4C656E67746835
:102120003A20006F637465742F73747265616D007B
:10213000696D6167652F6A70656700696D616765C4
:102140002F67696600746578742F68746D6C006120
:1021500070706C69636174696F6E2F6A736F6E0063
:10216000746578742F706C61696E00436F6E74656E
:102170006E742D547970653A2000436F6E6E6563FE
:1021800074696F6E3A20636C6F73650041636365B9
:1021900073732D436F6E74726F6C2D416C6C6F771F
:1021A0002D4F726967696E3A202A00556E6B6E6F0B
:1021B000776E004E6F74204D6F64696669656400C8
:1021C0004F4B004D6F766564207065726D616E6572
:1021D0006E746C7900496E7465726E616C20536523
:1021E00072766572204572726F72005061796C6F01
:1021F000616420546F6F204C61726765004E6F748C
:1022000020666F756E64005757572D417574686569
:102210006E7469636174653A204261736963207208
:1022200065616C6D3D2241636365737320726573F4
:10223000747269637465642200556E617574686FA9
:1022400072697A6564005061796C6F6164207369AA
:102250007A652077726F6E670042616420726571E3
:102260007565737400485454502F312E312000206E
:10227000000000000000000000004F4E00000000C1
:102280000000004F46460000000000005245535435
:102290000000000000544F47474C450000004841F3
:1022A0004C540000000000584F4E00000000000099
:1022B000584F46460000000000494E4352454153E6
:1022C0004500444543524541534500454E41424C2B
:1022D0004500000044495341424C450000554E46DC
:1022E0005245455A4500465245455A450000004171
:1022F00055544F000000000046414E5F4F4E4C5970
:10230000004849474800000000004D454449554DEC
:102310000000004C4F5700000000000048454154A9
:102320000000000000434F4F4C00000000004452EA
:102330005900000000000053544F500000000000FE
:1023400052474200000000000048535600000000C1
:10235000000057726F6E67207061796C6164004392
:1023600054524C2F7478743A204F75744F664D65F3
:102370006D6F72793A2000202D3E2041543A00437F
:1023800068616E20747970653A004E6F2073746FC7
:102390007265642076616C756573202D20646566B6
:1023A00061756C743A20002D3E005075623A200031
:1023B0002D3E005075623A20002D3E005075623A65
:1023C00020000000000000636D640000736574006D
:1023D0000076616C000064656C0000485356000094
:1023E000524742000066616E00006D6F64650063D5
:1023F00074726C0068756500007361740000746528
:102400006D700072617700002D3E005075623A20B9
:10241000002D3E005075623A2000556E6B6E6F774E
:102420006E20636D64200A000000000000000000C0
:10243000004F4E000000000000004F464600000024
:10244000000000524553540000000000544F47471D
:102450004C4500000048414C540000000000584F1B
:102460004E000000000000584F46460000000000EB
:10247000494E43524541534500444543524541531B
:102480004500454E41424C450000004449534142FD
:102490004C450000554E465245455A45004652456A
:1024A000455A450000004155544F000000000046C9
:1024B000414E5F4F4E4C59004849474800000000CC
:1024C000004D454449554D0000004C4F5700000059
:1024D000000000484541540000000000434F4F4CAD
:1024E0000000000000445259000000000000535456
:1024F0004F50000000000052474200000000000062
:102500004853560000000000005361766564204582
:102510005441473A0053657420455441473A2000DE
:1025200088C7BBB511241FBECFEFD1E2DEBFCDBF40
:1025300000E00CBF15E0A0E0B2E0EEEDF8EB01E04A
:102540000BBF02C007900D92AE3FB107D9F72BE049
:10255000AEEFB5E001C01D92A335B207E1F712E17D
:10256000C1E9D2E100E006C021970109802FFE01F8
:102570000E943FD4C039D10780E00807A9F70E9424
:10258000CDB50C945DDC0C940000CF93DF931F92CB
:10259000CDB7DEB76983DC01ED91FC910280F38158
:1025A000E02D41E050E0BE016F5F7F4F19950F9025
:1025B000DF91CF910895FC01818D928D0895CF9385
:1025C000DF931F92CDB7DEB76983DC01ED91FC91FB
:1025D0000280F381E02D41E050E0BE016F5F7F4F4C
:1025E00019950F90DF91CF910895FC019485FB011F
:1025F0008485981303C081E0983008F080E0089546
:10260000CF93DF931F92CDB7DEB76983DC01ED91E5
:10261000FC910280F381E02D41E050E0BE016F5F4C
:102620007F4F19950F90DF91CF910895FC01818123
:1026300091E09093AE088093D0081092AF0810926A
:10264000D10808952091CF06260F3327331F21325A
:102650003105ECF42091A808FC0190E080E02430E2
:1026600069F082E00895A091CF062191AC01415517
:10267000594FA40FB52FB11D2C930196861798F3CF
:102680008091CF06680F6093CF0680E0089581E0C7
:10269000089508950895E091810880918008E817D1
:1026A00030F4F0E0EE50F94F808190E008958FEF24
:1026B0009FEF089590918108809180082FEF3FEF60
:1026C000981748F4E92FF0E0EE50F94F208130E000
:1026D0009F5F90938108C90108958091800890912F
:1026E0008108891B990B0895CF92DF92EF92FF9298
:1026F0000F931F93CF93DF937C01CB018A0120912D
:10270000AE08222389F0EB016B01C40ED51ECC1557
:10271000DD0569F06991D701ED91FC910190F0819F
:10272000E02DC7011995F3CF642F0E942213C80131
:10273000DF91CF911F910F91FF90EF90DF90CF909D
:102740000895CF93DF931F92CDB7DEB769832091B1
:10275000AE082223F9F02091D108203258F021E070
:1027600030E0FC013383228390E080E00F90DF9122
:10277000CF9108958091AF08E82FF0E0E055F74F32
:10278000998190838F5F8093AF088093D10881E017
:1027900090E0ECCF61E0CE0101960E942213F7CFCA
:1027A00090E0FC01ED5AF04EE491F0E0EE0FFF1FD7
:1027B000E75CF04EA591B4912C918756904EFC01A8
:1027C0008491822391E009F490E0892F0895FC011F
:1027D000DC018D918111FDCF30E020E050E040E040
:1027E0008AE09191992301F1443051055CF59E32C4
:1027F00071F42F3F310509F02CF5DB01A40FB51F53
:1028000012962C934F5F5F4F30E020E0EACF829F1B
:10281000D001839FB00D1124292F990F330B205322
:1028200031092A0F3B1FDDCF2F3F310509F054F44A
:10283000443051053CF4640F751FFB01228381E095
:1028400090E0089590E080E008950097B1F1FC01D8
:10285000DB01AC01405F5F4F80E090812FE9290FE1
:10286000263098F497559295907F9C9321813FE96B
:10287000320F3630B0F42755922B9D933296E417E1
:10288000F50759F791E0892708952FEB290F263096
:1028900010F49753E8CF90539A3028F381E090E0FA
:1028A000E2CF3FEB320F363010F42753E5CF205301
:1028B0002A3010F381E020E0DFCF80E0089590E03F
:1028C00080E00895DC01ED91FC910284F385E02D18
:1028D0001994DF92EF92FF920F931F93CF93DF93A0
:1028E000EC010C891D890115110559F01D8A1C8AFE
:1028F000C801DF91CF911F910F91FF90EF90DF9072
:102900000895EC85FD858E859F85DF01A80FB91F91
:102910002C91243209F055C011962C912B3709F0D7
:1029200050C00296E80FF91FF12CE12CDF01D19085
:10293000DD2009F446C08DE7D816E9F08FEFE81ADC
:10294000F80AF4CF198A188A2C853D85211531059E
:1029500079F08E859F85280F391FF9012081222368
:1029600021F001969F878E873EC01D861C86C0CFB2
:102970000FEF1FEFBDCFE114F10419F11C928E850A
:102980009F8502966C857D85680F791FE881F981A6
:102990000684F785E02DCE011995998B888B1B8ACB
:1029A0001A8AEC85FD858E859F85E80FF91FEE0D4F
:1029B000FF1DD2828E859F850396E80EF91EFF8645
:1029C000EE86288939892115310509F4BDCF8A8918
:1029D0009B89280F391FF9012081222309F4B2CFE6
:1029E00001969B8B8A8B022F220F110B81CFDC016A
:1029F0001C96ED91FC911D971E968D919C91E80F70
:102A0000F91F8081082E000C990B0895DC011596A2
:102A10008D919C91009739F0DC01ED91FC9106803D
:102A2000F781E02D199408950097D1F0DC011696F6
:102A3000ED91FC913097A1F080858F70843021F466
:102A400081859285009771F40680F781E02D30979B
:102A500039F080858F70843019F4818592850895CE
:102A600090E080E00895089583E090E0089508954F
:102A700084E190E00895DC01ED91FC910484F585FA
:102A8000E02D60E0199581E090E008958FE090E0FE
:102A900090931E0780931D0788EC90E00895FC0139
:102AA000848195810895FC01768765870895DC010E
:102AB000ED91FC91068CF78DE02D199591E0892719
:102AC0000895862F089581E08627089521E0FC016E
:102AD0008485883008F020E0822F0895FC018485E9
:102AE00095850895FC0184899589089527EE33E042
:102AF000FC0131832083FB014089518962897389FC
:102B0000FC0142835383648375830895DC01ED9156
:102B1000FC91048CF58DE02D1994DC011196EC915B
:102B20001197E295EF70E150EB3008F039C0F0E01A
:102B30008827E256FA4E8F4F0C943FD4C115C11529
:102B4000D015A915A915B215C915C915C915A91505
:102B5000A91514966D917D918D919C9117970E9466
:102B600071D2089514966D917D918D919C911797D6
:102B700024E630E040E050E00E94D6D3CA01B9011B
:102B8000EECF14966C9170E090E080E00E946FD2DE
:102B9000089514966D917D918D919C91179708954C
:102BA00060E070E0CB010895DC011196EC91119783
:102BB000E295EF70E150EB3008F03EC0F0E088277E
:102BC000EB51FA4E8F4F0C943FD4FB15FB151C169E
:102BD000F015F0151516061606160616F015F01562
:102BE00014962D913D914D915C911797A4E6B0E01C
:102BF0000E94F5D3089514966C9184E6689FB00105
:102C00001124072E000C880B990B089520E030E06A
:102C100048EC52E414966D917D918D919C9117979B
:102C20000E94D0D20E943CD5089514966D917D915A
:102C30008D919C911797089560E070E0CB01089505
:102C4000FC01A7812A2F2E7FD1F0818182958F7080
:102C500081508330A0F4A695A150BB0B2BE531E049
:102C60000E9456D424E630E040E050E00E94D6D3E3
:102C7000DA01C90187569F4FAF4FBF4F08958FEFBD
:102C80009FEF0895DC01ED91FC91309729F090853C
:102C90009F7081E0953009F080E00895FC01A481E7
:102CA000B581109721F118969C9118979F708EEF1F
:102CB000890F823010F091111AC019964D935D93CF
:102CC0006D937C931C97A481B58118969C9118975D
:102CD000907F926018969C930480F581E02D80850A
:102CE000982F907F903619F48F70806A80870895AE
:102CF000DC0119968D919C91009739F0DC01ED91E2
:102D0000FC910280F381E02D19940895FC01238148
:102D100030E090E080E0FC01EE0FFF1FE05DF94F36
:102D2000A081B181A217B30761F4880F991F880FA2
:102D3000991FFC01E45EF94F4083518362837383E2
:102D40000895A081B181AB2B19F420813181EDCFA1
:102D5000019685309105F9F60895FC01238130E054
:102D600090E080E0FC01EE0FFF1FE05DF94F408135
:102D700051814217530761F4880F991F880F991FDB
:102D8000FC01E45EF94F6081718182819381089535
:102D900040815181452B89F431832083880F991F0D
:102DA000880F991FFC01E45EF94F10821182128294
:102DB000138260E070E0CB010895019685309105A3
:102DC00089F6F7CF880F991F880F991FFC01EC5FD8
:102DD000F94F80819181A281B3810196A11DB11D1E
:102DE00080839183A283B383089585E090E00C945F
:102DF000E21684E090E00C94E21683E090E00C94FC
:102E0000E21682E090E00C94E21681E090E00C94EF
:102E1000E21690E080E00C94E216CF93DF93EC0191
:102E2000E881F9810484F585E02D199529893A898D
:102E30002F5F3F4F3A8B298BDF91CF910895CF932E
:102E4000DF93EC018E8581110DC081E090E049890E
:102E50005A892C853D854217530708F080E0DF91A1
:102E6000CF910895E881F9810484F585E02DCE01A4
:102E700019958F3F910549F780E090E0F0CFFC0174
:102E8000848595856817790708F4CB01928B818B2F
:102E90000895DC011E962C911E97222339F0ED91A6
:102EA000FC910190F081E02D6FEF19940895FC01E1
:102EB00087859089089581E0089590E080E00895E5
:102EC000DC011296ED91FC91309761F00190F08158
:102ED000E02D309739F0862F8295807F60856F7066
:102EE000682B60870895DC011296ED91FC91309774
:102EF00051F00190F081E02D309729F08085829586
:102F00008F7090E0089590E080E00895CF93DF9374
:102F1000CDB7DEB760970FB6F894DEBF0FBECDBF5A
:102F200019821A821B821C821D821E821F821886B1
:102F30008A818F7080618A836FEF3E819F8188854F
:102F400029817A815B814C814C873E87888B372F22
:102F5000452F5C857E85892F988960960FB6F894F9
:102F6000DEBF0FBECDBFDF91CF9108950F931F93AA
:102F7000CF93DF9300D000D01F921F92CDB7DEB762
:102F800081E028960FB6F894DEBF0FBECDBFDF916B
:102F9000CF911F910F910895CF92DF92EF92FF9200
:102FA0000F931F93CF93DF9300D000D0CDB7DEB740
:102FB0008C016B017A01FC01808D883010F40E9435
:102FC0002A9487EE93E09A838983F6018281938124
:102FD000A481B5818B839C83AD83BE83B701CE0171
:102FE00001960E9439A3F801808F8830A0F4F586FD
:102FF000E486128E118E81E026960FB6F894DEBF1D
:103000000FBECDBFDF91CF911F910F91FF90EF9039
:10301000DF90CF90089580E0EFCFCF93DF93EC0166
:10302000888D883020F40E942A9488E0888FDF9170
:10303000CF910895FC01808D883040F4218D328D30
:10304000232B21F00E94FC9290E008958FEF9FEFD8
:103050000895CF93DF93FC012485283028F08FEF6B
:103060009FEFDF91CF910895EC010190F081E02D69
:103070000084F185E02D1995892B89F38C850E94B8
:10308000FC9290E0EECFCF93DF93FC01218D328D47
:103090002115310529F48FEF9FEFDF91CF9108952E
:1030A000EC01808D4217530708F0A9010E944B9351
:1030B0001816190684F7298D3A8D281B390B3A8F7B
:1030C000298FEBCF0F931F93CF93DF931F92CDB731
:1030D000DEB7FC01218D328D232B41F48FEF9FEF62
:1030E0000F90DF91CF911F910F9108958C0141E0D6
:1030F00050E0BE016F5F7F4FFC01808D0E944B93BB
:10310000181619065CF7F801818D928D0197928F40
:10311000818F898190E0E4CFCF93DF931F92CDB769
:10312000DEB741E050E0BE016F5F7F4FFC01848558
:103130000E944B931816190634F4898190E00F9081
:10314000DF91CF9108958FEF9FEFF9CFFC01848538
:10315000883010F40C944B9390E080E00895FC01CB
:103160008485883010F40C94249390E080E00895D6
:103170000F931F93CF93DF9300D000D01F921F9225
:10318000CDB7DEB78C01D80159964D915C915A9715
:103190004115510551F0ED91FC91048CF58DE02D18
:1031A00070E060E0C8011995EECFF801808D0E94B3
:1031B0002493892BB1F148E050E0BE016F5F7F4F4F
:1031C000D80158968C910E944B9318161906F4F466
:1031D000D801509684E0FE01319601900D928A95B7
:1031E000E1F78D8190E0982F88272E81820F911D25
:1031F000F801958B848B8F81282F30E0322F222786
:103200008885820F932F911D928F818F28960FB6FC
:10321000F894DEBF0FBECDBFDF91CF911F910F910C
:10322000089590E080E0F2CFCF92DF92EF92FF928C
:103230000F931F93CF93DF93CDB7DEB7AF970FB642
:10324000F894DEBF0FBECDBF7C016A0107EE13E02C
:103250001A8309831C861B8688EE93E0A0E0B0E009
:103260008D879E87AF87B88B8DEB93E09A87898790
:10327000188F0F8B198E1A8E1B8E1C8E88E089A3D7
:103280001BA70AA71CA61DA61EA61FA68091FB08A9
:103290009091FC08A091FD08B091FE088EA39FA319
:1032A000A8A7B9A78B839C83AD83BE8318861F8292
:1032B000AE01465D5F4FCE0101960E9430AC813079
:1032C0009105B1F4D701ED91FC910488F589E02DC9
:1032D0001DA30CA38CA59DA5AEA5BFA58EA39FA3E2
:1032E000A8A7B9A7A601BE016C5D7F4FC7011995BC
:1032F000AF960FB6F894DEBF0FBECDBFDF91CF9172
:103300001F910F91FF90EF90DF90CF9008950F9352
:103310001F93CF93DF93EC018B01888D883010F4DD
:103320000E942A94B80182E00E947394888F8830AA
:1033300050F41D870C871A8E198E81E0DF91CF9192
:103340001F910F91089580E0F9CF0F931F93CF93B2
:10335000DF938C01EA01FC018485883048F40E94E7
:103360009A92892B39F481E090E0F801938382836B
:10337000D0E0C0E0CE01DF91CF911F910F91089571
:10338000EF92FF920F931F93CF93DF937C01809175
:103390006A08D4E0833309F0D8E00AE518E0C0E019
:1033A000F801219131918F01F701848195812817CE
:1033B000390729F0CF5FDC13F3CF80E006C08C2FF4
:1033C0000E9438948431B1F781E0DF91CF911F9151
:1033D0000F91FF90EF900895CF93DF93EC018C85D0
:1033E0008830D0F40E943894843189F0882379F0B1
:1033F000883169F021E08C3159F4E881F981008449
:10340000F185E02DCE01199521E0892B09F420E00A
:10341000822FDF91CF91089580E0FBCFCF92DF9292
:10342000EF92FF920F931F93CF93DF93CDB7DEB749
:10343000AF970FB6F894DEBF0FBECDBF8C016B0106
:103440007A0187EE93E09A8389831B821C821D8216
:103450001E821C861B8648EE53E060E070E04D87BC
:103460005E876F87788B2DEB33E03A872987988FBB
:103470008F8B198E1A8E1B8E1C8E28E029A39BA77A
:103480008AA71CA61DA61EA61FA6D8011C968C9155
:10349000883060F40E943894882321F0F8018485F4
:1034A0000E941C9488E0D8011C968C938091FB08A4
:1034B0009091FC08A091FD08B091FE088EA39FA3F7
:1034C000A8A7B9A78B839C83AD83BE8318861F8270
:1034D000AE01465D5F4FB601CE0101960E9430AC51
:1034E0000097C1F0D801ED91FC910684F785E02D9D
:1034F00087EE93E09DA38CA38CA59DA5AEA5BFA54B
:103500008EA39FA3A8A7B9A7A701BE016C5D7F4F9B
:10351000C8011995AF960FB6F894DEBF0FBECDBFA8
:10352000DF91CF911F910F91FF90EF90DF90CF909F
:1035300008950F931F93182F0E9458A604C09695C4
:103540008795779567951A95D2F78B019C01015065
:103550001109210931090E3F1F4F2F4F3F4F20F016
:1035600061E070E080E090E01F910F910895CF93AB
:10357000DF93EC018C85883060F40E9438948731A9
:1035800011F08C3131F48C850E947D928115984028
:1035900088F3DF91CF910895FC018485883010F481
:1035A0000C947D9290E080E00895CF93C62F0E9406
:1035B000161361EE8FEF98E00E94A1136C2F8FEF2E
:1035C00098E00E94A113CF910C9422A60E9416139A
:1035D00081E00E9432A591E0811190E0892F089549
:1035E000ECEBF0E080818A7B808360E084E10E94E4
:1035F00086A460E085E10C9486A4CF93DF93EC0170
:1036000064EE77E18FE39AE00E9435876C817D81DB
:103610008FE39AE00E943D9D6EED77E18FE39AE0A3
:103620000E9435878FE39AE00E94588560E08C8184
:103630000E94B4A4E881F9810484F585E02D60E05E
:10364000CE01199581E090E0DF91CF910895EF923E
:10365000FF921F93CF93DF93192F7B01C82FD92F90
:10366000D7FF03C0D195C195D10961E08C2F0E948D
:10367000B4A482E0E816F10499F460E08C2F0E9473
:1036800086A462EA76E18FE39AE00E9435878FE3B1
:103690009AE0DF91CF911F91FF90EF900C945885A5
:1036A000612FEF2851F46095661F6627661F8C2FE7
:1036B0000E9486A46EE976E1E6CF661F6627661F44
:1036C0008C2F0E9486A469E976E1DDCF63EB73E17C
:1036D000811102C065EB73E18EE899E00C943587A7
:1036E00065E670E18EE899E00E943587F0E0E0E061
:1036F000199584EF91E008956FE07AE0811102C09E
:103700006AE07AE08FE39AE00C943587DC01559605
:103710002C915597273781F4ED91FC91008CF18D18
:10372000E02D199569EB76E08FE39AE00E943587EA
:103730008FE39AE00C9458850895EF92FF920F93CF
:103740001F93CF93DF93EC018B018091AA06909198
:10375000AB060097A9F0FC0120852F70263081F47C
:103760000E949698FC0190859F70943049F4818561
:103770009285DF91CF911F910F91FF90EF90089567
:10378000EE88FF88C70101970D97D0F469EE73E0CA
:10379000C8010E94A0D8892B99F48FE2888F85E018
:1037A0008E9DB0018F9D700D11246052774E46E0C2
:1037B00050E0CE0149960E94ACCCCE014896D9CFBC
:1037C00090E080E0D6CF4F925F926F927F92AF925F
:1037D000BF92DF92EF92FF920F931F93CF93DF93ED
:1037E00000D000D0CDB7DEB77C01D62E8091A906DF
:1037F000882309F4BEC0D70114969C9180910002E1
:10380000891708F4B6C08091A7069091A806BAE07F
:103810006B13F0C0895A994FFC011082D70118969A
:103820000D911C910115110509F49FC0F8016185E6
:1038300072856115710591F44580568067807084AA
:103840008091F5089091F608A091F708B091F808DA
:10385000481659066A067B0609F487C0D8011B96EC
:103860004D915C911C974115510509F47EC0F701FB
:10387000248153968C91539790E0322F377002C079
:10388000959587953A95E2F780FF6FC0A22EB12CEF
:10389000C501887F9370892B39F451968D919C9145
:1038A000887F9370A82AB92AD8018D919C91DC0158
:1038B000ED91FC916115710509F486C00688F789C0
:1038C000E02D1995019709F050C06CE3F801808153
:1038D00091810E945C85A50170E060E02AE0D8013A
:1038E0008D919C910E940C85F801228180819181AB
:1038F0006AED78E1222311F068ED78E10E943587C6
:10390000D8011D966D917C911E978D919C910E947E
:10391000CF8660E2F801808191810E945C85D801A8
:103920001F966D917C9150978D919C910E94CF86AE
:10393000F8012281808191816DEC78E1222311F0E0
:1039400067EC78E10E94358767E576E0D8018D91D4
:103950009C910E94CF86F80180819181DC01ED91DC
:10396000FC91008CF18DE02D19951092A806109213
:10397000A706D70115968D919C911697009771F027
:1039800014963C9120910102231740F0DC01ED9147
:10399000FC910190F081E02D6D2D199581E090E072
:1039A00026960FB6F894DEBF0FBECDBFDF91CF9144
:1039B0001F910F91FF90EF90DF90BF90AF907F909D
:1039C0006F905F904F9008950488F589E02D27EE61
:1039D00033E03A832983D80115964D905D906D9020
:1039E0007C9018974B825C826D827E82BE016F5FF5
:1039F0007F4F67CF8F3491050CF0BBCFBDE06B17C5
:103A000009F4B7CF9C012F5F3F4F3093A806209356
:103A1000A706895A994FFC016083ABCF0C94D8CA92
:103A20000C94D8CACF93C1E068EE73E080E090E0D8
:103A30000E9425A66C2F8EE899E00E94369DCF5FEC
:103A4000C43191F784EF91E0CF910895EF92FF9206
:103A50000F931F93CF93DF930097C1F0FC01208158
:103A60002223A1F08C0187ECE82E83E2F82EC1E03E
:103A7000D0E0B701C8010E9475CC892B49F021968E
:103A8000F5E0EF0EF11CCE30D10599F7D0E0C0E0A3
:103A9000CE01DF91CF911F910F91FF90EF9008958C
:103AA000CF93DF9300D000D01F921F92CDB7DEB727
:103AB000E8E7F9E0128A118A80E090E1958784872F
:103AC00084E890E0948B838B81E0868780E090E2AD
:103AD000908B878787E7858B1C821B8289E992E020
:103AE0009A838983FE83ED838FEF9FEF98878F837F
:103AF00065E277E18EE899E00E94358760914D0696
:103B000070914E06CE0101960E945D8C88E799E087
:103B10000E94861B65E177E18EE899E00E94358777
:103B20008EE899E00E9458850E944EAF28960FB605
:103B3000F894DEBF0FBECDBFDF91CF91089565E051
:103B4000FC01808191810E940E99009749F0FC014F
:103B50008085982F907F21F082958F7090E0089556
:103B600090E080E00895FC0186819781009799F0AC
:103B7000FC0120852F70223029F4618572858385B0
:103B800094850895253039F460E00E940E990097DD
:103B900011F0FC01F2CF60E070E0CB0108950F93CB
:103BA0001F93CF93DF93FC01C281D3812097C9F18A
:103BB0008B0188858F70853021F5CE010E949A9DFA
:103BC0008017110671F16CF1602FCE010E940E99E1
:103BD000FC01892B31F180858F70823039F4618549
:103BE0007285838594850E9471D206C08330C9F4A2
:103BF0006185728583859485DF91CF911F910F91A7
:103C00000895672B71F4823029F469857A858B8554
:103C10009C85E9CF833029F469857A858B859C85DD
:103C2000EBCF60E070E0CB01E7CFCF93C62F63E02E
:103C3000FC01808191810E940E99FC01892B11F178
:103C40009085892F8D70F1F4907F926090878185A7
:103C50009285A385B4858827BB278C2B8187928783
:103C6000A387B48760E677E08FE39AE00E94358708
:103C70006C2F8FE39AE00E94369D8FE39AE0CF91FC
:103C80000C945885CF91089563E0FC018081918167
:103C90000E940E99009719F0FC01818508958FEF1D
:103CA0000895FF920F931F93CF93DF93CDB7DEB7A5
:103CB00064970FB6F894DEBF0FBECDBF8C01F62E11
:103CC0008FE290E09A838983FE01339688E0DF01DA
:103CD0001D928A95E9F7F8016681FF2011F081E0D5
:103CE0006827D80114968C910E9486A4F8018781D8
:103CF0009085A185B285883E9340A105B10508F461
:103D00008BC06AE278E18FE39AE00E943587D801A0
:103D100014966D917C918FE39AE00E943D9D65E23F
:103D200078E18FE39AE00E9435876F2D70E08FE392
:103D30009AE00E943D9D8FE39AE00E9458856CE4D2
:103D400078E1CE0101960E946ACCF80182819381CC
:103D50000E94441EFF2009F46BC06DE178E18431BC
:103D600051F066E178E1853131F06AE078E18F3039
:103D700011F462E178E1CE010B960E947ECC65EFF2
:103D800077E18FE39AE00E943587D8011296ED9192
:103D9000FC9113970190F081E02D60817181ED918C
:103DA000FC910288F389E02D9E012F5F3F4FAE0109
:103DB000455F5F4FC8011995BC018FE39AE00E94EF
:103DC0003D9D63EF77E18FE39AE00E943587D8014C
:103DD0001296ED91FC910190F081E02D608171814E
:103DE0008FE39AE00E94CF86BE016F5F7F4F8FE323
:103DF0009AE00E94CF8660EF77E18FE39AE00E941D
:103E00003587BE01655F7F4F8FE39AE00E94CF86C2
:103E10008FE39AE00E94588564960FB6F894DEBF4F
:103E20000FBECDBFDF91CF911F910F91FF900895ED
:103E300066E078E1823009F49ECF61E078E19BCFC3
:103E4000DC01ED91FC910484F585E02D62E019958B
:103E500081E090E00895CF92DF92EF92FF920F936E
:103E60001F93CF93DF93CDB7DEB760970FB6F8946B
:103E7000DEBF0FBECDBF7C016B01CA01B9012AE0D4
:103E8000AE014F5F5F4F0E9419CDD701ED91FC91BC
:103E90000288F389E02D9801AE014F5F5F4FB601B4
:103EA000C701199560960FB6F894DEBF0FBECDBF5F
:103EB000DF91CF911F910F91FF90EF90DF90CF9006
:103EC0000895892B71F0FB01828193810E94B59A3C
:103ED00062E572E18EE899E00E94358788EC90E017
:103EE000089590E080E0F2CF892B71F0FB01828190
:103EF00093810E94679A6BE372E18EE899E00E94D9
:103F0000358788EC90E0089590E080E0F2CFEF9262
:103F1000FF920F931F93CF93DF93CDB7DEB72C970C
:103F20000FB6F894DEBF0FBECDBF8C017B0187EECC
:103F300093E09A8389831B821C821D821E8298874C
:103F40008F8319861A861B861C8605301105ECF0B6
:103F5000BE01695F7F4FF701808591850E94E7135D
:103F6000892B99F0CE0107960E94589BBE01695F8C
:103F70007F4FF701868197810E94E713892B61F0BB
:103F8000CE0107960E94029C0EC0CE0101960E94AF
:103F9000589B0430110554F7CE0101960E94029CF3
:103FA00003301105A4F1BE01695F7F4FF7018481E1
:103FB00095810E94E713892B51F1CE0107960E944B
:103FC000AD9BBE01695F7F4FF701828193810E94A3
:103FD000E713892B19F1CE0107960E94039B64E138
:103FE00072E18EE899E00E94358780E00E94EC9CA7
:103FF00088EC90E02C960FB6F894DEBF0FBECDBFD4
:10400000DF91CF911F910F91FF90EF900895CE0116
:1040100001960E94AD9B023011059CF6CE010196DF
:104020000E94039B01301105D1F6CE0101960E943A
:10403000039B6BE172E18EE899E00E943587CFCF58
:104040000F931F93CF93DF938C01EB010297C4F082
:104050008A819B810E9409CC8093010299270E944A
:10406000FF9C0230110549F08C819D810E9409CC92
:104070008093000299270E94099DC8ECD0E002C0FD
:10408000C0E9D1E060E072E18EE899E00E943587F6
:10409000609101028EE899E00E94369D6BEE71E11D
:1040A0008EE899E00E943587609100028EE899E0E1
:1040B0000E94369D8EE899E00E945885CE01DF91DE
:1040C000CF911F910F910895CF93DF93EB0102974A
:1040D000A4F16BED72E18A819B810E9457CC892B00
:1040E00029F40E94579C6F770E949C9C64EE72E1B9
:1040F0008A819B810E9457CC892B29F40E94579C6E
:1041000060680E949C9C6AED71E18EE899E00E94D3
:1041100035870E94579C6095661F6627661F70E072
:104120008EE899E00E943D9D8EE899E00E945885B6
:1041300088EC90E0DF91CF9108950E94501DF8CF58
:10414000CF92DF92EF92FF920F931F93CF93DF9363
:10415000EC016A017B018E819F81892BF1F48881BA
:1041600099810E949A9D082F10E005301105ACF44A
:104170000E946B8EFC01892B19F08085807F8087DF
:1041800080858F708087FF83EE83BF01888199814E
:104190000E94159D0F5F1F4FE8CFEE81FF81309782
:1041A00081F08085982F9F7051F4807F8260808796
:1041B000EE81FF81C186D286E386F48602C092300A
:1041C000B9F3DF91CF911F910F91FF90EF90DF90A6
:1041D000CF9008958F929F92AF92BF92CF92DF922D
:1041E000EF92FF920F931F93CF93DF93EC0188819F
:1041F00099810E949A9D082F10E0043011059CF4CB
:104200000E946B8EFC01892B19F08085807F80874E
:1042100080858F708087BF01888199810E94159D5C
:104220000F5F1F4FEACF60E0888199810E940E994D
:104230007C01009751F1FC0180858F70843039F545
:10424000C184D284C114D10401F1F6018081882394
:10425000E1F080E9882E8AE0982EB12CA12C1A2D4D
:10426000C4010E9485CCAC01B401C6010E949ECC61
:10427000892B09F493C0FFEFAF1ABF0A89E0880EBB
:10428000911CE7E1AE16B10451F71FEF03C0823075
:10429000E1F711851887E880F98061E0C7010E9485
:1042A0000E999B838A8362E0C7010E940E999D83C9
:1042B0008C8364E0C7010E940E999F838E83103126
:1042C00081F0143109F45CC0DF91CF911F910F91FF
:1042D000FF90EF90DF90CF90BF90AF909F908F9026
:1042E00008958BE090E00E943CCA8C01FC01D383CE
:1042F000C28380E592E0918380831682CE010E9482
:10430000AA9D97FD2AC0F80195838483F8018481D2
:104310009581009719F0863491052CF080E290E0A9
:10432000F8019583848361E070E0CE010E94CF1D87
:1043300020E030E04AE754E40E94D0D20E9443D506
:10434000611571058105910589F0F8016783708712
:10435000818792871A870987B7CF919581959109AF
:10436000F8019583848381E08683D0CF88E893E148
:10437000A0E0B0E0F80187839087A187B287EACFF9
:1043800084E090E00E943CCAFC01D383C2832EE209
:1043900032E0318320839A87898796CFC6010E94B5
:1043A000EB8B8A2D90E0B0E0A0E0F7018187928747
:1043B000A387B4878085807F826080876BCFCF930F
:1043C000DF93EC01798368831A8619861B861C8E1D
:1043D0001B8E0E944216882329F0CE01DF91CF91D7
:1043E0000C94EA20DF91CF9108952F923F924F9243
:1043F0005F926F927F928F929F92AF92BF92CF9275
:10440000DF92EF92FF920F931F93CF93DF93CDB77D
:10441000DEB762970FB6F894DEBF0FBECDBF5C016A
:104420004B0129013A01CA01B9010E943CD51B0187
:104430003F926F938AE394E09F938F93CE0101960E
:104440007C019F938F930E9425D90F900F900F901E
:104450000F900F900F9020E030E0A901C301B2014E
:104460000E9472D5181624F077FA709477F8709439
:10447000F70101900020E9F731976F01CE18DF08AE
:104480008EE28083A2E0B0E0AC0FBD1FAC0DBD1D7D
:10449000BA8BA98BB10137FE03C071956195710983
:1044A000072E000C880B990B0E9471D29B01AC0166
:1044B000C301B2010E945DD420E030E040E251E44B
:1044C0000E94D0D20E943CD5605DE989FA89608360
:1044D000FE01EC0DFD1D1382D501ED91FC910288CA
:1044E000F389E02D9801A701B401C50119956296E1
:1044F0000FB6F894DEBF0FBECDBFDF91CF911F91F5
:104500000F91FF90EF90DF90CF90BF90AF909F9072
:104510008F907F906F905F904F903F902F90089575
:104520001F93CF93DF93FC01162FC389D489818910
:1045300092899C012F5F3F4F328B218BC80FD91F6F
:10454000CE010E948ED3181721F0612FCE010E9458
:1045500096D381E090E0DF91CF911F910895FC0107
:1045600081899289248535858217930740F42389B0
:104570003489820F931F0E948ED390E008958FEFAD
:104580009FEF0895DA01E0911207F0E0FE2FEE2789
:10459000E60FF71F90E0982F8827A901BD018E0F25
:1045A0009F1F0C94EF8FCF93DF931F92CDB7DEB791
:1045B0002091120730E0322F2227260F371F90E07C
:1045C000982F8827498341E050E0BE016F5F7F4FFD
:1045D000820F931F0E94EF8F0F90DF91CF9108956C
:1045E000CF93DF931F92CDB7DEB741E050E0BE011D
:1045F0006F5F7F4F0E94648F89810F90DF91CF9111
:1046000008952091120730E0322F2227620F731F86
:1046100090E0982F8827860F971F0C94F02263E074
:1046200070E00C9401239F92AF92BF92CF92DF92E1
:10463000EF92FF920F931F93CF93DF93EC017B01D7
:1046400080916A08811121C01B821A8288EE93E052
:10465000A0E0B0E08C839D83AE83BF8385E693E0CA
:104660009983888388E08C8788EE93E09E878D8786
:10467000CE01DF91CF911F910F91FF90EF90DF90CE
:10468000CF90BF90AF909F90089534E0932E8333E6
:1046900011F028E0922E8AE5C82E88E0D82E10E08E
:1046A00098E0B92EA12CD6012D913D916D01F70115
:1046B000848195812817390791F4812F0E943894BD
:1046C000082F873111F08C3139F5812F0E94249306
:1046D000892B59F50C3119F4812F0E941C941F5F0E
:1046E0009112E1CFA11008C0D701ED91FC91008497
:1046F000F185E02DC70119951B821A8288EE93E09F
:10470000A0E0B0E08C839D83AE83BF8385E693E019
:1047100099838883BC86A8CF843149F08111DFCF8B
:10472000F601329711821082DACFB12ED8CFAA24A7
:10473000A394D5CF8F929F92AF92BF92CF92DF92E8
:10474000EF92FF920F931F93CF93DF93CDB7DEB716
:104750002F970FB6F894DEBF0FBECDBF5C014B01A3
:104760007A0180916A088823C9F104E0833309F053
:1047700008E0B501CE0101960E9413238AE5C82EF8
:1047800088E0D82E10E0F601219131916F01F501FA
:10479000848195812817390751F4812F0E9438941C
:1047A000873129F4A701B401812F0E949A921F5FDB
:1047B0000113E9CFC7012F960FB6F894DEBF0FBEE5
:1047C000CDBFDF91CF911F910F91FF90EF90DF90C0
:1047D000CF90BF90AF909F908F900895F12CE12CD7
:1047E000E9CFDA01E0911207F0E0FE2FEE27E60FA5
:1047F000F71F90E0982F8827A901BD018E0F9F1FFA
:104800000C94648F44E050E0BC018FE090E00C9485
:10481000EF8F44E050E0BC0185E090E00C94EF8F16
:1048200044E050E0BC0181E090E00C94EF8F0895EB
:104830009F92AF92BF92CF92DF92EF92FF920F932F
:104840001F93CF93DF938C015B01942EE52EFC0127
:10485000C688D788F08C80E591E00E948AA18F2DD0
:104860000E944092C92DDE2D8C179D0708F4EC01A3
:104870009E01A501B6018F2D0E94BD91F801868988
:1048800097898C0F9D1F978B868BCE01DF91CF91DF
:104890001F910F91FF90EF90DF90CF90BF90AF905E
:1048A0009F900895CF93FC01C08D80E591E00E9418
:1048B0008AA160E270E08C2F0E94548F62E070E069
:1048C0008C2F0E94012384FD16C062E070E08C2FC3
:1048D0000E94012383FF0AC048E162E070E08C2F50
:1048E0000E94D32280E090E0CF91089580E591E08E
:1048F0000E948AA1E3CF40E162E070E08C2F0E9429
:10490000D32281E0F0CFFF920F931F93CF93DF93D9
:10491000EB01FC01178A168A2A81211109C02B811B
:10492000211106C02C81211103C02D81222301F108
:1049300041155105E9F08A01FC01F08C80E591E018
:104940000E948AA1AE014E5F5F4F24E030E06CE030
:1049500070E08F2D0E94C222B8018F2D0E944794D3
:1049600081E090E0DF91CF911F910F91FF9008952A
:1049700080E0F7CF0F931F93CF938C01FC016481EC
:10498000758181E20E947394C82F8830F8F480E525
:1049900091E00E948AA18C2F0E940F23833131F075
:1049A0008C2FCF911F910F910C941C9462E070E0BA
:1049B0008C2F0E94548FF80184819581EC2FF0E0B8
:1049C000EE0FFF1FE65AF74F91838083CF911F911F
:1049D0000F9108950F931F93CF93DF931F921F9210
:1049E000CDB7DEB7FC0124852830E0F48C0180E5EA
:1049F00091E00E948AA122E030E0AE014F5F5F4F5C
:104A000060E170E0F80184850E94F12389819A8138
:104A10009827892798270F900F90DF91CF911F91AA
:104A20000F91089590E080E0F6CF0F931F93CF93FE
:104A3000DF931F921F92CDB7DEB7FC01248528308B
:104A4000E0F48C0180E591E00E948AA122E030E050
:104A5000AE014F5F5F4F64E070E0F80184850E9413
:104A6000F12389819A819827892798270F900F90A1
:104A7000DF91CF911F910F91089590E080E0F6CFE4
:104A8000CF93DF93EC0187EE93E0998388831A82BA
:104A90001B821C821D8280E591E00E948AA1BE01DA
:104AA0006E5F7F4F44E050E08FE090E00E94648FA3
:104AB000CE01DF91CF9108950E94B090882331F00C
:104AC00080916A08843329F0873381F090E080E098
:104AD000089580E591E00E948AA185E390E00E941C
:104AE000F02285FD0DC082E090E0089580E591E020
:104AF0000E948AA18EE290E00E94F02280FFF3CF14
:104B000081E090E008951092A80881E08093A708C2
:104B10001092820861E084E10E9486A461E085E150
:104B20000E9486A4E9EBF0E080818E7F8083808103
:104B30008D7F808388E48093B80085E48093BC00F7
:104B40000895CF93DF9391E09093AE06882361F0B0
:104B5000C091B800D091BA000E94F01A0E9483253B
:104B6000D093BA00C093B800DF91CF910895CF924F
:104B7000DF92EF92FF920F931F93CF93FC01C181BD
:104B80000E940DA56B017C018091A808811164C071
:104B900081E08093A8088093A7089FEF9093A608D0
:104BA0001092A5081092A40880938308809183082E
:104BB000CC0FC82BC093830880918208813009F004
:104BC00081C0109282080E940DA56B017C0180912A
:104BD00083088093BB008091AA089091AB08A091B4
:104BE000AC08B091AD08892B8A2B8B2BA1F00E94C9
:104BF0000DA50091AA081091AB082091AC08309146
:104C0000AD086C197D098E099F090617170728073B
:104C1000390708F442C08091BC0083FDD8CF85ECF1
:104C20008093BC000E940DA56B017C018091A808B7
:104C3000813009F449C08091A508811167C0809135
:104C4000A508E4E8F8E0A2EFB6E090E0981751F18B
:104C500021912D939F5FFACF8091AA089091AB0884
:104C6000A091AC08B091AD08892B8A2B8B2B09F44D
:104C70008BCF0E940DA50091AA081091AB0820913E
:104C8000AC083091AD086C197D098E099F09061793
:104C900017072807390708F077CF8091A9080E94E5
:104CA000A12580E010928108809380088FEF98E022
:104CB0000E945A13CF911F910F91FF90EF90DF90B8
:104CC000CF90089585EEACCF8091AA089091AB0863
:104CD000A091AC08B091AD08892B8A2B8B2B09F4DD
:104CE000A5CF0E940DA50091AA081091AB082091B4
:104CF000AC083091AD086C197D098E099F09061723
:104D000017072807390708F091CFC7CF81E099CF5F
:104D10008F929F92AF92BF92EF92FF921F93CF9389
:104D2000DF93EC010E9458A64B015C0110E08BE47C
:104D3000E82EF12C0E9458A6681979098A099B0966
:104D4000683E73408105910510F5ED85FE8530972D
:104D500009F0199560EFCE010E94D51ACE010E948C
:104D6000B725182F80FD0FC08A81813009F41A827F
:104D7000812FDF91CF911F91FF90EF90BF90AF9067
:104D80009F908F900895C7010197F1F7D3CF81E0ED
:104D90008A83EECF1F93CF93DF93EC01162F0E94EF
:104DA0008826CE010E94161362ED8FEF98E00E94D4
:104DB000A113612F70E06095709584E0660F771FF6
:104DC0008A95E1F7612B8FEF98E00E94A1130E9472
:104DD00022A6CE010E94B725811711F084E08A83B4
:104DE000DF91CF911F910895CF93DF93EC0163EC96
:104DF0000E94D51ACE01DF91CF910C94B7250F9365
:104E00001F93CF93DF93EC01162F042F0E94882667
:104E1000002341F0CE010E94F426682F6460CE0189
:104E20000E94CA26CE010E94161365EA8FEF98E011
:104E30000E94A113612F8FEF98E00E94A113DF91D0
:104E4000CF911F910F910C9422A6EF92FF920F9396
:104E50001F93CF93DF938C017B0140E065E50E94B7
:104E6000FF26E70188E0E80EF11C699140E0C801E7
:104E70000E94FF26CE15DF05C1F7DF91CF911F916C
:104E80000F91FF90EF900895CF93DF93EC010E9474
:104E9000161340E060EFCE010E94FF26DF91CF9114
:104EA0000C9422A60F931F93CF93DF93EC010E94E3
:104EB000882680FD36C0CE010E94F42660E0CE0137
:104EC0000E94CA26CE010E948826CE010E94161397
:104ED00064EB8FEF98E00E94A1130E9422A6CE01FE
:104EE0000E948826082F10E082FF16C082E08A8385
:104EF0008881882341F0CE010E94F426682F6160EA
:104F0000CE010E94CA2615950795802F8170DF91EA
:104F1000CF911F910F9108958A81823049F71A82AB
:104F2000E7CF80E0F4CFCF92DF92EF92FF920F9322
:104F30001F93CF93DF938C01EB017A01FC018581F4
:104F400096810E9452278823C1F1BE01F801858114
:104F500096810E94252740E06EEBF80185819681BD
:104F60000E94FF26E7016701F9E0CF0ED11CF8018E
:104F7000E580F680C7010E948826C7010E941613AB
:104F800066E98FEF98E00E94A1130E9422A6C70154
:104F90000E94882661EEC7010E94D51AC7010E94AF
:104FA000B7258993CC16DD0611F7F8018581968126
:104FB0000E94522791E0813009F090E0892FDF9123
:104FC000CF911F910F91FF90EF90DF90CF900895B8
:104FD000CF93DF93EA010E949327882381F0DE01BB
:104FE00089E090E0815039F0ED91E927F0E0E75356
:104FF000F64E9491F7CF81E02885291380E0DF9168
:10500000CF910895CF93DF9300D000D000D0CDB7DB
:10501000DEB7AE014F5F5F4F0E94E827882331F073
:105020008D818F33A9F020F48F31A1F080E007C08B
:105030008F3521F08F37D1F78CE001C08BE02996B6
:105040000FB6F894DEBF0FBECDBFDF91CF910895AC
:105050008AE0F5CF89E0F3CF6F927F928F929F9293
:10506000AF92BF92CF92DF92EF92FF920F931F9376
:10507000CF93DF93FC01248521118CC0872E762EDF
:10508000EC010E945227882309F486C0CE010E94B9
:10509000882640E060EFCE010E94FF2610E000E08D
:1050A00066246A94AA24A394B12CE02EE694E69494
:1050B000E694F12C802F8770650101C0CC0C8A9595
:1050C000EAF78B85082E000C990B0817190734F5A1
:1050D000FE01EE0DFF1D93809C20CE010E948826CC
:1050E000CE010E94161368E78FEF98E00E94A1138B
:1050F000992011F080E8982E692D8FEF98E00E949A
:10510000A1130E9422A6CE010E948826982F907497
:1051100085FF0BC0992369F08EEF2AC099249394E0
:1051200008171907D1F2912CD8CF911102C087FF2F
:10513000602EFE01EE0DFF1D938187FF28C0C92A56
:10514000C3820F5F1F4F0034110509F0AECF6B868D
:10515000FFEF6F1202C081E08C872396E72DF82DB8
:10516000CF01089629912193E817F907D9F781E033
:10517000DF91CF911F910F91FF90EF90DF90CF9033
:10518000BF90AF909F908F907F906F900895C09444
:10519000C922D6CF80E0ECCF8FEFEACFCF92DF925B
:1051A000EF92FF920F931F93CF93DF93CDB7DEB7AC
:1051B00069970FB6F894DEBF0FBECDBFE091AC0685
:1051C000F091AD06309709F483C08091210790914A
:1051D0002207892B09F47CC08FEF83871486138202
:1051E000148215821682178210861186128666E84E
:1051F00070E18EE899E00E9435878EE899E00E9480
:1052000058858E010F5E1F4FBE016E5E7F4F8091ED
:10521000AC069091AD060E942C2818160CF058C0D0
:10522000A895DE0111969E012E5E3F4F7D01F9018A
:1052300041919F01842F90E054E0959587955A9570
:10524000E1F782599D4FFC0180818C93E42FEF7030
:10525000F0E0E259FD4F808111968C9311971296E0
:10526000A017B10721F7198AB70180912107909102
:1052700022070E9496986C0161E870E18EE899E03F
:105280000E943587B7018EE899E00E94CF86C1144D
:10529000D104B9F0C6010E9414157C01892B09F4D0
:1052A000B3CF6CE770E18EE899E00E943587B701D3
:1052B0008EE899E00E94CF868EE899E00E9458859A
:1052C000A3CF67E770E18EE899E00E943587F4CFBD
:1052D00088EC90E069960FB6F894DEBF0FBECDBFA4
:1052E000DF91CF911F910F91FF90EF90DF90CF90C2
:1052F00008950F931F93CF93DF936FEB79E18FE3C3
:105300009AE00E94598781E00E9432A50E94F01A1B
:1053100061E085E10E94B4A460E084E10E94B4A44D
:10532000C4E1D0E010E001E0612F85E10E9486A495
:1053300010276AE070E080E090E00E9425A62197A7
:1053400099F764E170E080E090E00E9425A60E9459
:1053500055A1C091AC06D091AD06209701F1CE01C8
:105360000E94E61A8823D9F0CE010E94442764EAFD
:1053700079E18FE39AE00E9459878091AC06909181
:10538000AD06FC0100830E94522760E979E181119A
:1053900002C06BE779E18FE39AE00E94598781E0D0
:1053A000DF91CF911F910F91089585ED8093BC00FF
:1053B0008091AA089091AB08A091AC08B091AD087B
:1053C0000796A11DB11D23E0B695A79597958795E2
:1053D0002A95D1F72091BC0024FD03C01092A808A3
:1053E00008954091AA085091AB086091AC08709163
:1053F000AD08452B462B472B69F30097A105B10556
:1054000041F025E32A95F1F700000197A109B109C0
:10541000E1CF8091A9080C94A1251F920F920FB69D
:105420000F9211240BB60F922F933F934F935F93DC
:105430006F937F938F939F93AF93BF93EF93FF935C
:105440008091B900887F803609F44DC008F040C0D3
:10545000883209F4A9C028F5803109F49DC0C8F448
:10546000882309F4FBC0883009F496C0FF91EF91BE
:10547000BF91AF919F918F917F916F915F914F916C
:105480003F912F910F900BBE0F900FBE0F901F906A
:105490001895883109F488C0803241F78093A608B6
:1054A00014C0803409F49DC040F48033B9F38833CC
:1054B000E9F68093A60885ECB0C0803509F485C074
:1054C000883509F496C0883489F60E94D529CECF54
:1054D000883909F48CC038F5883729F050F48836BB
:1054E00011F0803719F683E08093A8081092F10636
:1054F00057C0883809F47BC0803919F0803809F02A
:10550000B5CF8091F106803208F071C0E091F106CC
:1055100081E08E0F8093F1068091BB00F0E0EF52A6
:10552000F94F80833DC0803B39F0E0F4803A09F4C4
:1055300079C0883A09F09ACF84E08093A808109245
:10554000D0061092CF06E0917E08F0917F08199561
:105550008091CF0681110FC081E08093CF06109219
:10556000AF0609C0803C09F4A6CF883C09F4A3CF5C
:10557000883B09F07BCFE091D00681E08E0F8093CD
:10558000D006F0E0E155F94F80818093BB00909107
:10559000D0068091CF0629C0809183088093BB00FC
:1055A00085EC8093BC0062CF9091A5088091A408FF
:1055B000981758F5E091A50881E08E0F8093A50813
:1055C000F0E0EC57F74F8081E9CFE091A50881E04A
:1055D0008E0F8093A5088091BB00F0E0EC57F74F49
:1055E00080839091A5088091A4089817C8F285E857
:1055F000D8CFE091A50881E08E0F8093A508809117
:10560000BB00F0E0EC57F74F80838091A708811131
:105610005CCF81E08093820884EA8093BC00109282
:10562000A80824CF85EC8093BC001092A808809134
:10563000F106803230F4E091F106F0E0EF52F94FDC
:1056400010826091F10670E0E0917C08F0917D0895
:1056500081ED96E019951092F10608CF1092A608F8
:1056600034CF4F925F926F927F92AF92BF92CF9260
:10567000DF92EF92FF920F931F93CF93DF9300D0AF
:105680001F92CDB7DEB72B013C0129833A834B83B0
:105690005C83A6019501C801B701640D751D861DC7
:1056A000971D211531054105510511F00E94B4D314
:1056B00029813A814B815C816217730784079507C2
:1056C000D0F4241535054605570530F521E0822F25
:1056D0000F900F900F900F90DF91CF911F910F912E
:1056E000FF90EF90DF90CF90BF90AF907F906F9042
:1056F0005F904F900895461657066806790650F455
:1057000021E089819A81AB81BC8184159505A6052C
:10571000B705E8F220E0DBCF21E046165706680621
:105720007906A8F2F7CF8F929F92AF92BF92CF9255
:10573000DF92EF92FF920F931F93CF93DF937C0141
:105740004A015901C091AA06D091AB06062F660FF7
:10575000110B209709F45CC088858F70863009F0A2
:1057600055C06DEE73E0CE010E9496986C0182E008
:105770008816910449F062EF73E0E3E08E1691041D
:1057800029F0D0E0C0E006C066EF73E0CE010E94D1
:105790009698EC01C114D104D9F1F60180858F707F
:1057A0008430B1F561857285A801C7010E94CED809
:1057B000A8016BEF73E0C7010E94B0D8209779F180
:1057C00088858F70843059F569857A85A801C7016D
:1057D0000E94B0D8A8016BEF73E0C7010E94B0D857
:1057E000A114B10429F0A801B501C7010E94B0D8E5
:1057F000C701DF91CF911F910F91FF90EF90DF9044
:10580000CF90BF90AF909F908F900895D0E0C0E070
:10581000A80163E379E1C7010E94ACCCC9CFF2E0F3
:105820008F16910481F083E08816910429F060912D
:10583000130770911407CACFA8016DE279E1C7017F
:105840000E948ECCC7CFA8016AE279E1F8CFCF924F
:10585000DF92EF92FF920F931F93CF93DF93CDB719
:10586000DEB7C154D1090FB6F894DEBF0FBECDBF6D
:105870006C01AB0130E020E060E4CE0101967C01D8
:105880000E94932BF70101900020E9F731978F01D7
:105890000E191F09A801B701C6010E94C0D8892BA3
:1058A00011F010E000E0C801CF5BDF4F0FB6F894B5
:1058B000DEBF0FBECDBFDF91CF911F910F91FF9043
:1058C000EF90DF90CF900895CF92DF92EF92FF920A
:1058D0000F931F93CF93DF93CDB7DEB7C054D10999
:1058E0000FB6F894DEBF0FBECDBF80911D0790911B
:1058F0001E07059709F449C06115710509F445C0F3
:1059000069017A018B0140E450E0CE0101960E94CA
:10591000CED86FE270E0CE0101960E9495D8892B17
:1059200041F4980143E050E060E4CE0101960E940A
:10593000932B4FE350E0B601CE0101960E94B0D800
:105940000E94B498882309F180911D0790911E0749
:105950000697D9F48091D208811117C0B701CE0102
:1059600001960E9426A781E090E0C05CDF4F0FB651
:10597000F894DEBF0FBECDBFDF91CF911F910F9185
:10598000FF90EF90DF90CF90089590E080E0EDCF12
:10599000EF92FF920F931F93CF937C018C01C0E095
:1059A000C330E1F0F801428150E070E060E02AE0AD
:1059B00030E08EE899E00E94498668E279E18EE85D
:1059C00099E00E943587CF5F0F5F1F4FC43041F7CA
:1059D000CF911F910F91FF90EF900895F7014581AE
:1059E00050E070E060E02AE030E08EE899E00E944C
:1059F000498666E279E1E3CFCF93DF931F921F924E
:105A0000CDB7DEB78091470B9091480B009711F40A
:105A100083E59BE0BE016F5F7F4F681B790B072E0C
:105A2000000C880B990B0F900F90DF91CF91089588
:105A30004F925F926F927F928F929F92AF92BF929E
:105A4000DF92EF92FF920F931F93CF93DF93CDB727
:105A5000DEB760970FB6F894DEBF0FBECDBFFC0176
:105A600019861A861B861C869A859F7090669A876F
:105A7000A081B181109709F4F7C08C91882309F4B3
:105A8000F3C000811181D8019C91992309F443C08E
:105A90009D3209F4EDC090539A3028F00F5F1F4FEC
:105AA00011830083EECFC801D12CDC017D01E81AFF
:105AB000F90A2D91022E000C330B205331092A30A4
:105AC0003105A0F35F016EE270E0C8010E9495D835
:105AD000FC01009709F448C0DC014D018E1A9F0AB1
:105AE00011968C911197082E000C990BC097119666
:105AF0000A9798F38181282F082E000C330B20532E
:105B000031092A30310518F480330CF06EC020E0E2
:105B100030E0A90108C0D12CF12CE12CD3CF29E031
:105B200030E040E050E0AAE0B0E00E94F5D32B0165
:105B30003C012281822F022E000C990BC0978A30E3
:105B4000910570F420330CF458C02A330CF059C07E
:105B5000092E000CAA0BBB0B480E591E6A1E7B1E99
:105B60008114910409F052C0C8010E9427CC2A85F3
:105B70002F70206A2A872B013C016CE270E0D5016E
:105B80008D919C910E9495D8009709F068C0F5010D
:105B9000118210824D865E866F86788A88E0FE01CB
:105BA0003996DE01119601900D928A95E1F72981CF
:105BB0003A814B815C816D817E818F819885609671
:105BC0000FB6F894DEBF0FBECDBFDF91CF911F910E
:105BD0000F91FF90EF90DF90BF90AF909F908F90CC
:105BE0007F906F905F904F9008958A330CF097CF1D
:105BF000032E000C440B550B96CF80E090E0DC01A7
:105C0000ABCF89E090E0A0E0B0E0A6CFC801B3E060
:105C10008B169104DCF4E8E0EE16F104BCF40E946B
:105C200027CC9B01AC01A4E6B0E00E94F5D3DD20B7
:105C300041F07094609450944094411C511C611C3C
:105C4000711C460E571E681E791E97CF0E9405CC08
:105C50002B013C018A858F7080678A878ECF0196E1
:105C6000D5018D939C9396CF412C512C320192CF2C
:105C7000C8010196DD24D39418CFCF92DF92EF9222
:105C8000FF920F931F93CF93DF93EC01A881B9810B
:105C9000109781F18C91882369F108811981F801AD
:105CA0009081992351F09D3241F090539A3028F021
:105CB0000F5F1F4F19830883F0CFC8010E9427CCC4
:105CC0006B017C016CE270E0C8010E9495D80097DE
:105CD00069F419821882C701B601DF91CF911F9133
:105CE0000F91FF90EF90DF90CF90089501969983E8
:105CF0008883F1CFC12CD12C7601EDCF67E776E117
:105D00008EE899E00E94358764E676E18EE899E0B6
:105D10000E94358766E576E18EE899E00E94358736
:105D20006EE476E18EE899E00E9435878EE899E08E
:105D30000E9458856EE376E18EE899E00E943587EF
:105D400062E376E18EE899E00E94358765E276E1CC
:105D50008EE899E00E94358760E176E18EE899E06F
:105D60000E94358761E076E18EE899E00E943587F0
:105D700069EF75E18EE899E00E9435876EEE75E176
:105D80008EE899E00E94358761EE75E18EE899E032
:105D90000E94358767ED75E18EE899E00E943587AE
:105DA00068EC75E18EE899E00E94358760EC75E15A
:105DB0008EE899E00E94358764EB75E18EE899E002
:105DC0000E9435876AE975E18EE899E00E9435877F
:105DD0006BE775E18EE899E00E94358766E675E12C
:105DE0008EE899E00E94358769E575E18EE899E0D3
:105DF0000E9435876BE475E18EE899E00E94358753
:105E00006FE375E18EE899E00E94358767E375E1FD
:105E10008EE899E00E9435876CE275E18EE899E0A2
:105E20000E9435876FE175E18EE899E00E94358721
:105E300067E175E18EE899E00E9435876CE075E1D5
:105E40008EE899E00E9435876DEF74E18EE899E065
:105E50000E94358764EF74E18EE899E00E943587EF
:105E600066EE74E18EE899E00E94358768ED74E192
:105E70008EE899E00E9435878EE899E00C94588569
:105E80000F931F93CF93DF9300D000D0CDB7DEB731
:105E90000E947E2E61ED7DE08EE899E00E943587BC
:105EA000CE0101960E944025CE0101960E94C82C89
:105EB00007EE13E01A8309838091FB089091FC0898
:105EC000A091FD08B091FE088B839C83AD83BE83B7
:105ED000CE0101960E94C82C1A8309831B821C8262
:105EE0001D821E8280E591E00E948AA144E050E07C
:105EF000BE016D5F7F4F81E090E00E94648FCE0114
:105F000001960E94C82C1A8309831B821C821D8261
:105F10001E8280E591E00E948AA144E050E0BE012B
:105F20006D5F7F4F85E090E00E94648FCE01019607
:105F30000E94C82C67EF7DE08EE899E00E943587CB
:105F400088EC90E026960FB6F894DEBF0FBECDBF6A
:105F5000DF91CF911F910F910895009789F0FC0177
:105F600020852F70253061F40E940E99009741F032
:105F7000FC0120852F70243019F4818592850895C5
:105F800090E080E00895CF92DF92EF92FF920F931E
:105F90001F93CF93DF9300D000D0CDB7DEB78091B1
:105FA000A90681119AC080911D0790911E07029742
:105FB0000CF493C080914D0690914E06009709F421
:105FC0008CC06FEF73E00E9496988C01009709F4E3
:105FD00084C00E949A9DE82EF12CE114F10409F48A
:105FE0007CC070E060E0C8010E94AD2F6C01EA94B3
:105FF000EF2809F481C061E0C8010E940E99FC01FC
:1060000001851285CE0101960E944025CE010196A0
:106010000E948DA162EC7DE08EE899E00E943587B8
:10602000B6018EE899E00E94CF866CE674E08EE8B7
:1060300099E00E94CF86B8018EE899E00E943D9DCC
:106040006CE674E08EE899E00E94CF866BE678E01B
:106050008EE899E00E94CF868EE899E00E945885EC
:1060600062E072E08DE59AE00E948719D092530AAF
:10607000C092520A1093550A0093540A8BE698E096
:10608000892BE9F58DEF93E09093570A8093560A98
:106090008091150790911607009741F070E060E03D
:1060A0000E94AD2F909314078093130780911307DC
:1060B00090911407009731F19093590A8093580AF0
:1060C00010925B0A10925A0A81E08093A90669EA4D
:1060D0007DE08EE899E00E94358726960FB6F89409
:1060E000DEBF0FBECDBFDF91CF911F910F91FF900B
:1060F000EF90DF90CF90089502E012E083CF8BE61F
:1061000098E0C2CF82ED92E0892B19F48DEF93E0F5
:10611000D3CF82ED92E0D0CF0F931F93CF9364EA59
:106120007DE08EE899E00E94358702E719E0C0E043
:10613000F80181918F01803130F466E074E08EE8DF
:1061400099E00E94CF86C530C9F0F80131974081AF
:1061500050E070E060E020E130E08EE899E00E94DD
:10616000498662EA7DE08EE899E00E943587CF5F3C
:10617000C630F1F6CF911F910F91089540917709A4
:1061800050E070E060E020E130E08EE899E00E94AD
:1061900049868EE899E00E945885E9CFEF92FF92F8
:1061A0000F931F93CF93DF9300D000D01F92CDB7F2
:1061B000DEB77B01CE0107969F938F9301979F9344
:1061C0008F9301979F938F9301979F938F9301973D
:1061D0009F938F9301979F938F938E010F5F1F4F14
:1061E0001F930F9388E094E09F938F93DB011396A6
:1061F0008C9113978F9312968C918F930E9455D9FF
:106200000FB6F894DEBF0FBECDBF0697ECF468E67C
:1062100072E188E999E00E943587D70112966D9165
:106220007C9188E999E00E94CF8680E991E02796E9
:106230000FB6F894DEBF0FBECDBFDF91CF911F9197
:106240000F91FF90EF90089580916A0990916B09EA
:10625000892BA9F10E94F899882389F182E70E948D
:10626000E39980916A0990916B09DC01ED91FC91B1
:106270000088F189E02D64E070E0199580916A0949
:1062800090916B09DC01ED91FC910280F381E02D8E
:1062900046E050E0B801199586E0F801A2E7B9E0C0
:1062A00001900D928A95E1F780916A0990916B09AE
:1062B000DC01ED91FC910488F589E02D19950E948F
:1062C0008C306AE772E18EE899E00E94358788ECAD
:1062D00090E0ADCF2F923F924F925F926F927F925C
:1062E0008F929F92AF92BF92CF92DF92EF92FF92E6
:1062F0000F93CF93DF9300D01F92CDB7DEB77C0111
:106300007A8369835C834B83DB011C92FC0160818F
:10631000662309F44EC030FF4CC0F9E06F9FB00116
:1063200011246F587D4DCD010E94ACCCD701119640
:106330008C91807F41F04B815C8167E574E08981BD
:106340009A810E94B0D8E981FA8101900020E9F792
:10635000319729813A81E21BF30B19012E0E3F1E62
:106360004B815C814E1B5F0B415051095C834B8319
:10637000D7011196EC9111978E2F807F09F4F7C009
:10638000E295EF70E150EC3008F0F1C0F0E08827C2
:10639000E353FE4C8F4F0C943FD4DC317F32EC3210
:1063A0004B3366332A32FC32FC32FC321832003274
:1063B000823329803A80DCCFF7018481282F30E0B6
:1063C00050E040E0002359F030E0A4E6B0E00E9445
:1063D00008D42FEF30E040E050E00E94D6D35F9326
:1063E0004F933F932F938CE194E09F938F93FC8185
:1063F000FF932B812F933F922F920E94E8D8B2C037
:1064000017968C9117978F9316968C9116978F935A
:1064100015968C9115978F9314968C918F938FE18D
:1064200094E09F938F93BC81BF93EB81EF93E3CF75
:1064300017968C9117978F9316968C9116978F932A
:1064400015968C9115978F9314968C918F9383E268
:1064500094E0E7CF1496CD90DD90ED90FC901797E7
:10646000F7FE34C084E6882E912CA12CB12CC701F4
:10647000B601A50194010E94D6D39B01AC018827E7
:106480009927DC01821B930BA40BB50BBF93AF9331
:106490009F938F9366277727CB016C197D098E090F
:1064A0009F09A50194010E94D6D35F934F933F9318
:1064B0002F9387E294E09F938F933C813F934B818E
:1064C0004F933F922F920E94E8D84CC0C701B6016B
:1064D00024E630E040E050E00E94D6D39F938F93B3
:1064E0007F936F935F934F933F932F9388E294E052
:1064F0009F938F939C819F93AB81AF93E2CFC70112
:106500000E942016BC01D7011696CC9016971796BC
:10651000DC901797D0FADD24D0F814969C9114974C
:106520001596FC90EB80BC80292F30E050E040E0D5
:1065300077FD35C0011135C07F936F931F921F9275
:106540001F929F931F92FF92DF92CF9281E394E07C
:106550009F938F93FC81FF932B812F933F922F92D8
:106560000E94E8D80FB6F894DEBF0FBECDBF898178
:106570009A810F900F900F900F90DF91CF910F9114
:10658000FF90EF90DF90CF90BF90AF909F908F9053
:106590007F906F905F904F903F902F9008950023D1
:1065A00061F0292F30E0A4E6B0E00E9408D42FEF7C
:1065B00030E040E050E00E94D6D35F934F933F938A
:1065C0002F931F92FF92DF92CF9284E394E09F93E8
:1065D0008F93BF92EF9275CF15968C9115971F925E
:1065E0008F9316969C91169717968C9181708F9326
:1065F0009F9387E394E015CF14968D909D90AD9076
:10660000BC90179720E030E0A901C501B4010E94B9
:106610006AD22401350187FF04C077FA709477F8B5
:106620007094C301B2010E943CD56B01072E000C8F
:10663000880B990B0E9471D29B01AC01C301B2017E
:106640000E945DD420E030E04AE754E40E94D0D2BA
:106650000E94C7D50E943CD5062F772E20E030E05F
:10666000A901C501B4010E946AD287FF07C07F92C9
:106670000F93DF92CF928DE394E0D3CE7F920F936E
:10668000DF92CF928EE394E09F938F933C813F9370
:106690004B814F93B0CE14968C9114971F928F9389
:1066A00015968C9115971F928F9316968C911F9229
:1066B0008F9384E394E09F938F93BC81BF93EB818E
:1066C000EF933F922F920E94E8D84CCF17968C916F
:1066D00017971F928F9314968C9114971F928F93F4
:1066E00015968C9115971F928F9316968C911F92E9
:1066F0008F9381E394E09F938F93BC81BF93EB8151
:10670000EF93DFCE14966D917C914B815C81C1013A
:106710000E94CED82CCFEF92FF920F93CF93DF93AE
:10672000CDB7DEB7A0970FB6F894DEBF0FBECDBFD2
:106730007C0100E020E033E040E250E0BE016F5F0A
:106740007F4F0E946A31BE016F5F7F4F8FE39AE0F7
:106750000E94CF8661E17CE08FE39AE00E9435875A
:10676000F701618162956F708FE39AE00E94369D18
:106770006AE07CE08FE39AE00E943587F70161814F
:106780006F708FE39AE00E94369D8FE39AE00E943B
:106790005885A0960FB6F894DEBF0FBECDBFDF912F
:1067A000CF910F91FF90EF900895AF92BF92CF924B
:1067B000EF92FF920F931F93CF93DF9300D000D0FF
:1067C0001F921F92CDB7DEB75C0109831A832B831A
:1067D0003C834D835E836F83788763E578E18FE345
:1067E0009AE00E943587CE0101960E948B33E11416
:1067F000F10439F06CE478E1C7010E9475CC009790
:1068000021F1F5010281138101151105E1F0898162
:10681000811159C08A818F70813009F45CC038F1D0
:10682000823019F1082F10E06FE278E18FE39AE0EF
:106830000E943587B8018FE39AE00E943D9D8FE367
:106840009AE00E94588590E080E028960FB6F89470
:10685000DEBF0FBECDBFDF91CF911F910F91FF9093
:10686000EF90CF90BF90AF900895CC20B9F0CE01BB
:1068700001960E941D99892B09F444C0C8010E9409
:10688000B31D672B682B692BD9F480E00E94991AFD
:10689000AB01BC01C8010E94A02012C0C8010E9427
:1068A000441E8E3019F048F4813051F4CE01019627
:1068B0000E941D99892B21F0E1CF83518330B0F3E1
:1068C00081E090E0C2CF8031C0F48E30B8F68130E4
:1068D000A9F28230B9F06FE378E18FE39AE00E9489
:1068E000358769818FE39AE00E94369D8FE39AE0B5
:1068F0000E94588501E010E097CF8351833008F45F
:10690000BDCFE9CF40E050E0BA01C8010E94A0200D
:1069100060E0C5010E94511ED3CFCF92EF92FF924B
:106920000F931F93CF93DF9300D000D01F921F923D
:10693000CDB7DEB77C0109831A832B833C834D835B
:106940005E836F83788762EC77E18FE39AE00E9441
:106950003587CE0101960E948B338981811129C030
:106960000A810F70013069F128F010E00230D1F592
:10697000CC20E1F0CE0101960E941D99F701028121
:106980001381892B69F0C8010E94B31D672B682B06
:10699000692B61F480E00E94991AAB01BC0103C02D
:1069A00040E050E0BA01C8010E94A02081E090E0E0
:1069B0002AC08031B0F58E30B8F58130A9F182302F
:1069C000B9F165EB77E18FE39AE00E943587698141
:1069D0008FE39AE00E94369D8FE39AE00E945885EB
:1069E00001E010E065EA77E18FE39AE00E943587E5
:1069F000B8018FE39AE00E943D9D8FE39AE00E94E8
:106A0000588590E080E028960FB6F894DEBF0FBE60
:106A1000CDBFDF91CF911F910F91FF90EF90CF905D
:106A200008958351833068F6F70102811381ABCF5B
:106A300040E050E0BA01F70182819381B5CFCF9257
:106A4000DF92EF92FF920F931F93CF93DF93611525
:106A5000710509F458C06A017B018C01CB010E94C9
:106A60004216D82F882371F1D70114968D919C91ED
:106A70000097E9F1FC01C0852C2F2F703EEF320FFB
:106A8000323010F0211128C0C295CF70D0FE59C00D
:106A9000C7010E94441EF8018083CC2351F1C295A6
:106AA000C07F81818F70C82BC183D7011496ED916F
:106AB000FC9181859285A385B485F80184839583B3
:106AC000A683B7838D2FDF91CF911F910F91FF90F8
:106AD000EF90DF90CF900895253049F460E00E9458
:106AE0000E99009721F0DC011896CC91CDCFC0E033
:106AF000CDCFD7011496ED91FC9180858F708230B7
:106B000021F0833081F0D0E0DDCF4185528563856F
:106B10007485F80181818F70806A818344835583F5
:106B200066837783CFCF4185528563857485F8016D
:106B300081818F70806781834483558366837783E7
:106B4000C1CFCC23B1F2C295C07FF801AACF0F9379
:106B50001F93CF93DF9300D000D01F921F92CDB729
:106B6000DEB719821A821B821C821D821E821F823E
:106B700018862A812F702A83FC0102811381C801A3
:106B80000E94441E813041F020F0823011F08530A7
:106B900081F490E080E002C081E090E028960FB69A
:106BA000F894DEBF0FBECDBFDF91CF911F910F9143
:106BB000089540E052E0B801CE0101960E941F35D1
:106BC000CE0101960E941D99E9CFCF93DF9300D0AB
:106BD00000D01F921F92CDB7DEB7FC01862F8F70B9
:106BE0006181607F682B618388E0DE0111960190EE
:106BF0000D928A95E1F729813A814B815C816D8103
:106C00007E818F81988528960FB6F894DEBF0FBEDF
:106C1000CDBFDF91CF910895CF93DF9300D000D007
:106C20001F921F92CDB7DEB7FC01608398E0DE01B2
:106C3000119601900D929A95E1F729813A814B8145
:106C40005C816D817E818F81988528960FB6F8943E
:106C5000DEBF0FBECDBFDF91CF910895DC0111964D
:106C6000EC911197E295EF70E150EB3008F037C0EE
:106C7000F0E08827E15CF94C8F4F0C943FD45136FB
:106C800051366F364A364A3660365736573657369B
:106C90004A364A3614966D917D918D919C91179745
:106CA000089514966C9170E090E080E00895149639
:106CB0006D917D918D919C9117970E943CD508957F
:106CC00014966D917D918D919C91179724E630E0FB
:106CD00040E050E00E94D6D3CA01B901089560E0B7
:106CE00070E0CB0108958F929F92AF92BF92CF92A6
:106CF000DF92EF920F931F93CF93DF9300D000D0DA
:106D00001F921F92CDB7DEB709831A832B833C8372
:106D10004D835E836F837887FC012081318121154B
:106D20003105A1F490E080E028960FB6F894DEBF1C
:106D30000FBECDBFDF91CF911F910F91EF90DF90EC
:106D4000CF90BF90AF909F908F9008958C01C90114
:106D50000E949A9DC82ED12CF6E0CF16D104ACF437
:106D60000E946B8EFC01892B19F08085807F8087C3
:106D700080858F708087BF01F801808191810E949A
:106D8000159DFFEFCF1ADF0AE7CF65E0F80180819C
:106D900091810E940E998C01892B21F28981803189
:106DA00008F6CE0101960E942E3616161706180612
:106DB000190644F4F8018085982F9D70A1F08F701A
:106DC000873089F0F80180858F70808764EA77E0EA
:106DD0008FE39AE00E9435878FE39AE00E945885FE
:106DE00081E090E0A1CF0E9458A64B015C01CE014A
:106DF00001960E942E36860E971EA81EB91EF80117
:106E000081869286A386B48682E0E11087E099812C
:106E10009295907F892BF801808769E977E08FE36D
:106E20009AE00E943587CE0101960E942E36AB0172
:106E3000BC012AE030E08FE39AE00E94498663E9D2
:106E400077E08FE39AE00E943587F801418552850B
:106E5000638574852AE030E08FE39AE00E944986DA
:106E6000BBCFCF93DF93EC016115710539F48F81AE
:106E700081708F8381E0DF91CF9108958981982F70
:106E800092959F7029F180E09430A8F79B01770FCD
:106E9000440B550B2959310941095109A4E6B0E0C9
:106EA0000E94F5D32BE531E040E050E00E94D6D3BC
:106EB00037FF02C030E020E02536310514F024E62B
:106EC00030E02F5F220F8F818170282B2F83D2CF4C
:106ED0008F7080628983DACF2F923F924F925F92B8
:106EE0006F927F928F929F92AF92BF92CF92DF92DA
:106EF000EF92FF920F931F93CF93DF93CDB7DEB73F
:106F00006A970FB6F894DEBF0FBECDBF1C0109878C
:106F10001A872B873C874D875E876F87788B22E1A6
:106F2000E216F10408F035C0F701EE51FD4F308153
:106F30003D8BCE0109960E94201697FD04C0BC012E
:106F4000C1010E9431379A85892F8F70D101119626
:106F5000EC911197E07FE82B1196EC9311978985BE
:106F60008C93E295EF70EC3008F063C0F0E0882776
:106F7000E354F84C8F4F0C943FD4AC39E637E637E6
:106F80004B39CB37E039153954395439543915391F
:106F900015391D8ACECF10E092959F709D3008F074
:106FA00011C4E92FF0E08827E752F84C8F4F0C947A
:106FB0003FD41938193A393A193AE239E239193ACB
:106FC000193AE23BE23B193A193AEF3892959F7031
:106FD0009D3008F014C1E92FF0E08827ED50F84CFF
:106FE0008F4F0C943FD41938CD38C03883380338CC
:106FF0000038A438CF38FF38FF388E388E38EF3855
:107000008889F10187838F85D10116968C93169715
:107010008E8515968C9315978D8514968C93149761
:107020009295907F11968C9111978F70982B119655
:107030009C93FD89FF2309F463C0D10111968C91C3
:1070400082958F702F2F30E08217130609F458C0F5
:1070500064E67BE08FE39AE00E943587F10161816D
:1070600062956F708FE39AE00E94369D61E67BE047
:107070008FE39AE00E9435876D898FE39AE00E9442
:10708000369D6FE57BE08FE39AE00E943587D10162
:107090000C9119821A821B821C821D821E821F8201
:1070A00018868D898295807F9A819F70892B8A832B
:1070B0000983EE24EA94FE2C11961C9111971296E6
:1070C0002C91129713963C91139714964C91149708
:1070D00015965C91159716966C91169717967C915C
:1070E000CE0101960E946C37F101208331834283E7
:1070F00053836483758386839783C1010E948B3396
:1071000088E0F1016FC18F859889F10186838781BD
:1071100090FB80F987838E8585838BCF8D859E85B7
:10712000AF85B889B7FD0EC08F3F9105A105B105A8
:1071300029F024F08FEF90E0A0E0B0E0D1011496A8
:107140008C9377CF80E0FACF6D857E858F85988987
:1071500020E06D39BFEF7B078B079B076CF02FEFAB
:107160006115E4E67E078105910534F424E630E0FC
:1071700040E050E00E94D6D3D10114962C9359CF11
:107180008F859889F1018683878190FB80F98783B9
:107190008E8585838D8584834CCF8D85CFCFCD849F
:1071A000DE84EF84F88820E030E0A901C701B60151
:1071B0000E946AD260E087FD0FC020E030E04FE718
:1071C00053E4C701B6010E9472D56FEF181624F080
:1071D000C701B6010E9443D5F10164832ACFD101D2
:1071E00011968C9111978F70806C11968C931197DA
:1071F0008D859E8515969C938E9314971ACF61EF7B
:107200007BE08FE39AE00E9435876A8562956F7014
:107210008FE39AE00E94369D6EEE7BE08FE39AE06A
:107220000E943587F1016181C0C092959F709330B3
:1072300091F09C30A1F24D855E856F857889F101D2
:1072400044835583668377839295907F81818F7085
:10725000982B9183EECEC1010E941D99D101149605
:107260008C9314978F85988916968C9316971796FA
:107270008C91179790FB80F917968C9317978E85B2
:1072800015968C93159711968C9111978F7080623B
:1072900011968C93CECECE0109960E941D99D101F4
:1072A00014968C931497EFCF92959F709D3008F0B1
:1072B00066C0E92FF0E08827EF59F64C8F4F0C9409
:1072C0003FD419387C39AB392B39AB39AB396E39EE
:1072D0009B399B399B398A399639EF388D859E8544
:1072E000AF85B889F10184839583A683B7838181B3
:1072F0008F70806681839DCE6D8570E090E080E028
:107300000E946FD2D10114966D937D938D939C93BF
:1073100017978FCE6D857E858F8598890E9471D253
:10732000F101648375838683978383CE6D857E8523
:107330008F859889E5CF9295907FF10181818F703B
:10734000982B91838D859E85AF85B889848395839D
:10735000A683B7836ECE9295907FD10111968C91C2
:1073600011978F70982B11969C938D859E85AF8574
:10737000B889F10184839583A683B7835ACE6CEDD7
:107380007BE08FE39AE00E9435876A8562956F7093
:107390008FE39AE00E94369D69ED7BE08FE39AE0EF
:1073A0000E943587D10111966C9162956F708FE3C1
:1073B0009AE00E94369D8FE39AE00E94588539CE6C
:1073C00011E0EACD4D855E856F857889F1014483B2
:1073D0005583668377839295907F81818F70982BF8
:1073E000918388E0DE01119601900D928A95E1F774
:1073F00029813A814B815C816D817E818F81988565
:107400006A960FB6F894DEBF0FBECDBFDF91CF9165
:107410001F910F91FF90EF90DF90CF90BF90AF90B2
:107420009F908F907F906F905F904F903F902F90A4
:107430000895963009F4C1C048F46D85913071F01B
:107440006FEF70E0933051F060E008C0973009F4BE
:10745000C0C09A506D857E859230B0F784E68F87E4
:1074600088898E7F888B1E868A858F7080628A8746
:107470006D872E8530E0AFEFB0E00E9408D4C12CBC
:10748000D12C7601CA946115F4E67F078105910538
:1074900044F424E630E040E050E00E94D6D3690195
:1074A0007A01112309F475C0DA8AC98A2D852E8BD9
:1074B000022F10E088898695A82FA150BB0BB88FAA
:1074C000AF8B119609F0A4C09601203831050CF05D
:1074D00087C08FE790E08C199D09809FD001819F24
:1074E000B00D909FB00D11242FEF30E00E9456D4C4
:1074F00021E83EE740E050E00E94D6D3D101179644
:107500002C93ABE9B0E0A70196010E94F5D33FE7C9
:10751000432E512C612C712CA30192010E94D6D3D1
:107520002C593F4F4F4F5F4F5901AEEFB1E0A701CC
:1075300096010E94F5D3A30192010E94D6D3D801EF
:107540000E94F5D32FEF30E040E050E00E94D6D308
:1075500089012F3F310519F014F00FEF10E06CECAA
:107560007BE08FE39AE00E943587B5018FE39AE0D4
:107570000E943D9D6EEB7BE08FE39AE00E94358791
:10758000B8018FE39AE00E943D9D8FE39AE00E944C
:1075900058856CE87BE08FE39AE00E9435878FE3A3
:1075A0009AE00E94588565E87BE08FE39AE00E94AC
:1075B0003587C1010E948B333CCD6D857E858F85DB
:1075C000988924E630E040E050E00E94D6D3B9012B
:1075D00045CF6D857E858F8598890E943CD53ECFAD
:1075E000A7012058310941095109ABE9B0E00E94D7
:1075F000F5D32FE730E040E050E00E94D6D32C597D
:107600003F4F4F4F5F4F5901D10117961C92A7CFA3
:107610002F89388DAAEBBFEF0E944ED424E6822E2C
:10762000912CA12CB12CA50194010E94D6D3290143
:107630003A01B4E64B0E511C611C711C26E430E08B
:10764000AF89B88D0E9456D4A50194010E94D6D36B
:1076500049015A01EEE18E0E911CA11CB11C298931
:107660003A89203831050CF094C08FE790E0821BF6
:10767000930B809FD001819FB00D909FB00D11247E
:10768000A50194010E9400D49B01AC01AFEFB0E0D2
:107690000E94F5D324E63AE640E050E00E94D6D3BB
:1076A000D10117962C93A7019601240D351D461D77
:1076B000571DAEEFB1E00E94F5D323EE30E040E07D
:1076C00050E00E94D6D3298B3A8B4B8B5C8BE98997
:1076D000FA89FA8FE98FAFEFB0E0A70196010E9417
:1076E000F5D32FE730E040E050E00E94D6D3790197
:1076F000FE89AF2FB0E029893A894B895C890E94C5
:10770000F5D32FEF30E040E050E00E94D6D389015E
:107710002F3F310519F014F00FEF10E068EB7BE01C
:107720008FE39AE00E9435872AE030E0B301A2019E
:107730008FE39AE00E94498662EB7BE08FE39AE058
:107740000E9435872AE030E0B501A4018FE39AE07A
:107750000E9449866AEA7BE08FE39AE00E943587BF
:10776000B7018FE39AE00E943D9D62EA7BE08FE3E0
:107770009AE00E943587B8018FE39AE00E943D9D10
:1077800069E97BE08FE39AE00E943587698D7A8D05
:10779000F8CEA70196012058310941095109ABE9FA
:1077A000B0E00E94F5D32FE730E040E050E00E94C7
:1077B000D6D32C593F4F4F4F5F4F7901D1011796C8
:1077C0001C92ACCF63E77BE08FE39AE00E943587A1
:1077D0006A8562956F708FE39AE00E94369D60E73C
:1077E0007BE01CCDFC019181892F82958F7021F067
:1077F000823029F080E008959F70906291839B0110
:1078000077FF02C030E020E02E3681E0380714F028
:107810002DE631E02683878130FB80F9878381E084
:1078200008950F931F93CF93DF938C01FC01C081C8
:10783000D1816FE270E0CE010E94DDD80097D9F0CF
:10784000FC011192CF010E94261DEC0168E677E051
:107850008FE39AE00E943587BE018FE39AE00E9491
:107860003D9D8FE39AE00E945885CE01DF91CF9134
:107870001F910F910895CE010E94261DEC01892BC6
:10788000A1F3F80111821082F0CF8F929F92AF92F4
:10789000BF92CF92DF92EF92FF920F931F93CF93FD
:1078A000DF93CDB7DEB767970FB6F894DEBF0FBE94
:1078B000CDBF8C017B014C018BE0880E911C9F8A0F
:1078C0008E8AF801128611861386148E138E672B0A
:1078D00009F463C0A0901F07B0902007A114B10461
:1078E00009F45BC06FE270E0C7010E9495D86C019B
:1078F000892B09F44AC0F701DE01119690E080E07F
:10790000BD012191222341F02F3231F084319105C4
:1079100019F02D930196F5CF860F971FFC01108269
:10792000C5010E949698F80191838083B6016F5F2C
:107930007F4F4FE050E0C4010E94CED8CE01469662
:107940000E94113CF801948F838F8E899F89892B27
:1079500009F41386C8010E944216882319F0C80151
:107960000E94EA2067960FB6F894DEBF0FBECDBF27
:10797000DF91CF911F910F91FF90EF90DF90CF900B
:10798000BF90AF909F908F900895B701C5010E945E
:107990009698F80191838083DDCFF80111821082DF
:1079A000D9CF8F929F92AF92BF92CF92DF92EF92F8
:1079B000FF920F931F93CF93DF93CDB7DEB7CD55D3
:1079C000D1090FB6F894DEBF0FBECDBF8C016B019D
:1079D0006115710519F041155105D1F460EA7DE09A
:1079E0008FE39AE00E94358767E97DE08FE39AE0B4
:1079F0000E943587B8018FE39AE00E94CF8665E93F
:107A00007DE08FE39AE00E9435878FE39AE030C0F3
:107A1000460F571FDA011C920E94FC2C4B0163E9B0
:107A20007DE08FE39AE00E943587B4018FE39AE00E
:107A30000E943D9D60E97DE08FE39AE00E943587DA
:107A4000B8018FE39AE00E94CF866DE87DE08FE376
:107A50009AE00E943587BAE38B16B1E09B06F4F4F6
:107A600060E87DE088E999E00E94358788E999E03F
:107A70000E945885C35ADF4F0FB6F894DEBF0FBE81
:107A8000CDBFDF91CF911F910F91FF90EF90DF90CD
:107A9000CF90BF90AF909F908F9008956EE77DE05C
:107AA0008FE39AE00E943587B6018FE39AE00E9447
:107AB000CF866CE77DE08FE39AE00E9435878FE305
:107AC0009AE00E9458851A821982FE0133968EE34D
:107AD000DF011D928A95E9F780911D0790911E079D
:107AE000059791F563E070E0C8010E94272C7C01A6
:107AF000892BE9F5E0911109F0911209808180FF4D
:107B0000B9CF61E070E0C8010E94272C892B09F4ED
:107B1000B1CF64E270E0C8010E94DDD8892B09F082
:107B2000A9CF64E67DE08FE39AE00E943587B80133
:107B30008FE39AE00E94CF868FE39AE00E945885F7
:107B4000C8010E94F0A296CF61E070E0C8010E94D7
:107B5000272C7C01892B21F562E070E0C8010E948E
:107B6000272C7C0169E57DE0892B09F44ACFE00EE2
:107B7000F11E60E57DE0C7010E9475CC892BC1F440
:107B8000F60101900020E9F73197EC19FD093297D1
:107B900078F0C8010E94F0A2C6010E94348B6ACF1F
:107BA0004FE350E0B801CE0101960E94CED8DFCF5E
:107BB00064E270E0C8010E94DDD8892B09F05ACF39
:107BC000B701CE018F5B9F4F0E94453CCE018F5B7A
:107BD0009F4F0E944216882339F1B601CE018F5B78
:107BE0009F4F0E945F9E18161906F4F4898188231E
:107BF000D9F080911D0790911E070597A9F068E3C1
:107C00007DE08FE39AE00E943587BE016F5F7F4F72
:107C10008FE39AE00E94CF868FE39AE00E94588516
:107C2000CE0101960E94F0A2CE018F5B9F4F0E9471
:107C3000781620CFCF92DF92EF92FF926A017B01FC
:107C400063E0FC01808191810E940E99FC01892BE7
:107C5000A9F080858D7091F4C094D094E094F09454
:107C6000CC24CA9481859285A385B4858C219D21DD
:107C7000AE21BF2181879287A387B487FF90EF90C1
:107C8000DF90CF900895CF92DF92EF92FF926A013A
:107C90007B0163E0FC01808191810E940E99FC01CF
:107CA000892BA9F09085892F8D7089F4907F92603F
:107CB0009087CC24FF2441855285638574854C29A7
:107CC0005D296E297F294187528763877487FF90DA
:107CD000EF90DF90CF900895CF92DF92FF920F93B5
:107CE0001F93CF93DF93F12C6115710509F499C0AF
:107CF0006A01EB018C01CB010E944216F82E882309
:107D000009F48FC0D2FE09C0D8018C918B3009F4E0
:107D10004BC0E8F58A3009F44CC0D0FE09C0F80128
:107D2000608186EF860F843018F0CE010E94151E08
:107D3000D1FE6EC0D80114964D915D916D917C91EC
:107D4000179711968C9182958F70873038F0893013
:107D500008F43EC08A50823008F46CC0CE010E9404
:107D60004E16EC81FD81309709F452C080858F70EA
:107D70009EEF980F923010F081114AC0D8011196F1
:107D80009C91907F80858F70892B808741C08C303B
:107D9000B9F040E050E062E070E08D3009F0BDCF16
:107DA000CE010E94433EB9CF40E050E061E070E078
:107DB000F7CF40E050E061E070E0CE010E941A3E53
:107DC00040E050E062E070E0CE010E941A3EA5CF94
:107DD000EC81FD813097E1F080858F709EEF980FE8
:107DE000923010F0811114C04187528763877487E5
:107DF000EC81FD818085807F83608087EC81FD81BF
:107E00008085982F907F8F708067903609F4BDCF62
:107E100063E07CE08FE39AE00E943587C8010E940E
:107E20008B338F2DDF91CF911F910F91FF90DF90BA
:107E3000CF900895CE010E944E16EACFCF92DF92E6
:107E4000EF92FF926A017B0163E0FC0180819181E6
:107E50000E940E99009791F0FC0120852F7022302E
:107E600069F461857285838594856C217D218E21DD
:107E70009F21FF90EF90DF90CF90089560E070E039
:107E8000CB01F7CFCF92DF92EF92FF920F931F9328
:107E9000CF93DF9300D000D01F921F92CDB7DEB7F3
:107EA0006C017B0160FF03C0E894E0F8F4F8F4FC97
:107EB0000DC00E94FC2C663971058105910530F0DA
:107EC00080911D0790911E07059709F5A70144278A
:107ED0005770052E000C660B770BC6010E94433EBF
:107EE0006FE77AE08FE39AE00E9435878FEF9FEF8C
:107EF00028960FB6F894DEBF0FBECDBFDF91CF91AD
:107F00001F910F91FF90EF90DF90CF90089519820D
:107F10001A821B821C821D821E821F8218868A8101
:107F20008F708A8340E053E0B601CE0101960E9433
:107F30001F3540E057E060E070E0C6010E941E3F40
:107F4000E62AF72A09811A812B813C814D815E81C5
:107F50006F817885C6010E9441A7CACF4F925F9278
:107F60006F927F928F929F92AF92BF92CF92DF9249
:107F7000EF92FF920F931F93CF93DF93CDB7DEB7AE
:107F80002C970FB6F894DEBF0FBECDBF6D7F61306A
:107F9000710509F4BAC0DC011296ED90FC90E11471
:107FA000F10409F4B2C04C01C7010E94B31D2B01BA
:107FB0003C0161E070E0C7010E94CF1D41145104F3
:107FC0006104710409F4A1C020E030E04AE754E400
:107FD0000E94D0D20E9443D569877A878B879C877D
:107FE000672B682B692B09F490C00E9458A69B014F
:107FF000AC01A12CB12C6501E984FA840B851C85A8
:10800000C301B2010E94312B882309F47EC0F40120
:108010006280738070E060E0C3010E94CF1D20E0A9
:1080200030E048EC52E40E94D0D20E9443D56B016C
:108030007C0180E00E94991AAB01BC01C3010E943F
:10804000A02019821A821B821C821D821E821F821E
:1080500018868A818F708A83D40112966D917C91E3
:1080600040E053E0CE0101960E941F35CE010196FB
:108070000E94D4152B013C0166E474E08FE39AE082
:108080000E94CF86B301A2018FE39AE00E94339D44
:1080900065E574E08FE39AE00E94CF86B701A60100
:1080A0008FE39AE00E94339D8FE39AE00E94588507
:1080B000C40CD51CE61CF71C8A818F7080668A83ED
:1080C000CD82DE82EF82F886F4016281738140E026
:1080D00052E0CE0101960E946C3E69E574E08FE3A8
:1080E0009AE00E94CF86B701A6018FE39AE00E9432
:1080F000339D8FE39AE00E94588560E072E0D401DE
:1081000012968D919C910E94423F90E080E02C96C7
:108110000FB6F894DEBF0FBECDBFDF91CF911F9198
:108120000F91FF90EF90DF90CF90BF90AF909F9016
:108130008F907F906F905F904F900895AF92BF9215
:10814000CF92EF920F931F93CF93DF93CDB7DEB70C
:10815000C856D1090FB6F894DEBF0FBECDBF5C0183
:10816000A2960FAFA297A3961FAFA397A4962FAF87
:10817000A497A5963FAFA597A6964FAFA697A796AB
:108180005FAFA797A8966FAFA897A9967FAFA9975B
:108190009E2D28E0FE01EF59FF4FDE01A75ABF4F89
:1081A00001900D922A95E1F7A296EFADA297E150CA
:1081B000ED3008F0F0C0EC2CF0E08827ED51FF4BDB
:1081C0008F4F0C943FD458416141BF41C941B541E3
:1081D000F0404F41CB41CB416A417C41A2418F41AC
:1081E000992331F0C5010E949F1D009709F447C0F3
:1081F00067E0CE01875A9F4F0E940C366FE777E009
:108200008FE39AE00E9435876A966FAD6A978FE395
:108210009AE00E94369D64E777E08FE39AE00E943F
:108220003587CE01875A9F4F0E942E36AB01BC0185
:108230002AE030E08FE39AE00E9449868FE39AE0DB
:108240000E9458856A960FAD6A976B961FAD6B9723
:108250006C962FAD6C976D963FAD6D976E964FAD4A
:108260006E976F965FAD6F97A0966FADA097A19632
:108270007FADA197C5010E94733681E090E0C85997
:10828000DF4F0FB6F894DEBF0FBECDBFDF91CF91A9
:108290001F910F91EF90CF90BF90AF9008959111E3
:1082A00005C0C5010E949F1D009749F366E0A1CF5C
:1082B000992329F0C5010E949F1D009701F362E0F8
:1082C00098CF911105C0C5010E949F1D0097B9F27A
:1082D00061E08FCF40E050E061E070E0C5010E94B6
:1082E0001E3F672B682B692B29F4C5010E949F1D37
:1082F000009729F26BE07DCF40E050E061E070E054
:10830000C5010E941E3F672B682B692B31F0C50108
:108310000E949F1D009709F4B2CF6AE06ACF40E047
:1083200050E062E070E0C5010E941E3F672B682BA1
:10833000692B31F0C5010E949F1D009709F49FCF62
:108340006CE057CF40E050E062E070E0C5010E9471
:108350001E3F672B682B692B31F4C5010E949F1DBE
:10836000009709F48CCF6DE044CF911106C0C50190
:108370000E949F1D009709F482CF63E03ACF9923B2
:1083800031F0C5010E949F1D009709F478CF65E088
:1083900030CF64E02ECF90E080E071CF2F923F92FB
:1083A0004F925F926F927F928F929F92AF92BF9205
:1083B000CF92DF92EF92FF920F931F93CF93DF93B1
:1083C000CDB7DEB7C85CD1090FB6F894DEBF0FBEDB
:1083D000CDBF1C01CF54DF4F0883C15BD040CE54CA
:1083E000DF4F1883C25BD040CD54DF4F2883C35B7F
:1083F000D040CC54DF4F3883C45BD040CB54DF4FE8
:108400004883C55BD040CA54DF4F5883C65BD04019
:10841000C954DF4F6883C75BD040C854DF4F7883AF
:10842000C85BD040C754DF4FF982E882C95BD040B7
:10843000C354DF4FC882CD5BD040CE53DF4FA882FC
:10844000C25CD0400E94FC2C6B01C554DF4F798385
:108450006883CB5BD040683C7105A4F466EF79E09B
:1084600088E999E00E943587B60188E999E00E9481
:108470003D9D88E999E00E945885AA24AA94BA2CC7
:108480000C94974B0E9458A6CB53DF4F6883798397
:108490008A839B83C55CD040CE54DF4F8881C25B0A
:1084A000D0408F70682E712C20911D0730911E07CF
:1084B000CD53DF4F39832883C35CD040C754DF4F8F
:1084C000E881F981C95BD040309721F0808181112A
:1084D0000C943D4FD1011B968C91882341F0C10132
:1084E0000B96C754DF4F99838883C95BD0406114D2
:1084F000710411F00C94864FC754DF4FE881F98165
:10850000C95BD040309711F00C94414FF101638C5E
:10851000748C6114710411F40C94864FCE54DF4FA7
:108520008881C25BD0408F7011F00C94864F662D0D
:10853000CE018F549F4F0E94E535C756DF4F2883E9
:10854000C959D040C656DF4F3883CA59D040C556A6
:10855000DF4F4883CB59D040C456DF4F5883CC59A6
:10856000D040C356DF4F6883CD59D040C256DF4F4D
:108570007883CE59D040C156DF4F8883CF59D04041
:10858000C056DF4F9883C05AD0400C94864FD1011B
:108590002D913C91232B09F470CFB4E06B1671043C
:1085A00099F5CE53DF4FE880C25CD040CF54DF4F07
:1085B0000881C15BD040CE54DF4F1881C25BD040F0
:1085C000CD54DF4F2881C35BD040CC54DF4F38817E
:1085D000C45BD040CB54DF4F4881C55BD040CA5408
:1085E000DF4F5881C65BD040C954DF4F6881C75BFD
:1085F000D040C854DF4F7881C85BD040C1010E9491
:1086000073365C010C94974B28E0FE01EF54FF4F4A
:10861000DE01A755BF4F01900D922A95E1F7CF5487
:10862000DF4F1881C15BD040143009F4E5C248F433
:10863000112309F467C0912C812CAA24AA94BA2C86
:1086400052C388EF810F8230B0F788E0FE01EF540B
:10865000FF4FDE01119601900D928A95E1F7CE54FD
:10866000DF4F8881C25BD040807F09F447C3CE01D1
:108670008F549F4F0E94D4154B015C0181149104CB
:10868000A104B10409F43AC3193041F4B094A094A0
:1086900090948094811C911CA11CB11CB101CE014D
:1086A0008F549F4F0E94CC9D60E0CE018F549F4F0E
:1086B0000E940C366A962FAF6A976B963FAF6B9706
:1086C0006C964FAF6C976D965FAF6D976E966FAF70
:1086D0006E976F967FAF6F97A0968FAFA097A1967A
:1086E0009FAFA19722E06216710409F45EC30CF0FB
:1086F0000BC3442443946114710409F457C3912CAF
:10870000812C2CC519821A821B821C821D821E821A
:108710001F8218862A812F702A83CE54DF4F28812A
:10872000C25BD040207F09F486CFEAE06E16710468
:1087300009F41EC25CF46114710459F102E0601680
:10874000710409F4D4C0912C812C0DC21BE0611678
:10875000710409F4B9C12CE062167104A1F7B101EA
:10876000CE0101960E94CC9DCE018F549F4F0E9456
:108770002016BC01CE0101960E94313788E0FE012F
:108780003196DE01AF54BF4F01900D928A95E1F70B
:10879000E7C1892B59F063EB79E08FE39AE00E94FF
:1087A00035878FE39AE00E945885CDCFC1010E94A2
:1087B000F5598C0161E070E01816190614F070E0AC
:1087C00060E08FE39AE00E943D9D67E574E08FE3EF
:1087D0009AE00E94CF86CE018F549F4F0E942E3682
:1087E000AB01BC012AE030E08FE39AE00E944986A9
:1087F0008FE39AE00E945885CE018F549F4F101648
:10880000110614F00C94314F0E942E36912C812CBD
:10881000672B682B692B89F562E0CE018F549F4F3F
:108820000E940C36CF56DF4F2883C159D040CE5618
:10883000DF4F3883C259D040CD56DF4F4883C359EC
:10884000D040CC56DF4F5883C459D040CB56DF4F71
:108850006883C559D040CA56DF4F7883C659D04087
:10886000C956DF4F8883C759D040C856DF4F988319
:10887000C859D04088248394982C44244394DD2400
:10888000D3943AC061E0CE018F549F4F0E940C36C2
:10889000C757DF4F2883C958D040C657DF4F3883AA
:1088A000CA58D040C557DF4F4883CB58D040C45733
:1088B000DF4F5883CC58D040C357DF4F6883CD5823
:1088C000D040C257DF4F7883CE58D040C157DF4FDA
:1088D0008883CF58D040C057DF4F9883C059D040CD
:1088E00088248394982C44244394D12C05C0912C43
:1088F000812C412CDD24DA94B101CE0101960E9435
:10890000CC9D8A81982F92959F70945F9F70923032
:1089100060F4CE54DF4F9881C25BD04092959F7037
:10892000923019F48F7080628A83D10118969C91DD
:10893000973071F4CE54DF4F8881C25BD040807E87
:10894000803211F0803421F48A818F7080628A83B2
:10895000F101A185B285892F90E0109741F0ED914A
:10896000FC911197048CF58DE02DCD0119957C01BA
:10897000CF54DF4F0881C15BD040CE54DF4F188108
:10898000C25BD040CD54DF4F2881C35BD040CC5474
:10899000DF4F3881C45BD040CB54DF4F4881C55B8B
:1089A000D040CA54DF4F5881C65BD040C954DF4F16
:1089B0006881C75BD040C854DF4F7881C85BD04026
:1089C000CE0101960E946C37CF57DF4F2883C158E4
:1089D000D040CE57DF4F3883C258D040CD57DF4FFD
:1089E0004883C358D040CC57DF4F5883C458D04039
:1089F000CB57DF4F6883C558D040CA57DF4F7883C5
:108A0000C658D040C957DF4F8883C758D040C85791
:108A1000DF4F9883C858D040CE0101960E948B3317
:108A2000442051F1CE54DF4F8881C25BD040829503
:108A30008F709FE0980F9F70923020F08A5F8F7048
:108A40008230D0F48A8182958F7081508230A0F478
:108A50002D8130E0AFEFB0E00E9408D42FEF611518
:108A6000F4E67F078105910534F424E630E040E028
:108A700050E00E94D6D32D8388E0FE013196DE01BE
:108A8000AF54BF4F01900D928A95E1F702E1902A11
:108A9000512CAA24AA94BA2CD10118968C9118971B
:108AA000873009F075C5C554DF4FE881F981CB5B8C
:108AB000D040EE35F1400CF07AC36FE679E088E9FA
:108AC00099E00E943587D5CCB101CE0101960E9474
:108AD000CC9DCA54DF4F8881C65BD0409A81929565
:108AE0009F7039F0923049F0912C812C5524539489
:108AF0003BC09A819F7090629A8390E08536910581
:108B000014F084E690E08E8388E0FE013196DE0169
:108B1000AF54BF4F01900D928A95E1F762E0CE010C
:108B20008F549F4F0E94E535EA962FAFEA97EB9658
:108B30003FAFEB97EC964FAFEC97ED965FAFED97AD
:108B4000EE966FAFEE97EF967FAFEF97C158DF4F7E
:108B50008883CF57D040C058DF4F9883C058D0404B
:108B6000812CE2E19E2E512C412CDD24DA9491CF10
:108B7000B101CE0101960E94CC9DC954DF4F68819E
:108B8000C75BD040C854DF4F7881C85BD04071705C
:108B9000CE0101960E94F23B482E912C812C552447
:108BA0005394882311F388E0FE013196DE01AF541F
:108BB000BF4F01900D928A95E1F762E0CE018F548C
:108BC0009F4F0E94E535E2962FAFE297E3963FAFC5
:108BD000E397E4964FAFE497E5965FAFE597E696A7
:108BE0006FAFE697E7967FAFE797E8968FAFE89786
:108BF000E9969FAFE997B4CF19E06116710409F4C3
:108C000059C0C1010E94F5591816190654F562E0C1
:108C1000CE018F549F4F0E940C36AA962FAFAA9771
:108C2000AB963FAFAB97AC964FAFAC97AD965FAFFF
:108C3000AD97AE966FAFAE97AF967FAFAF97E0961A
:108C40008FAFE097E1969FAFE19788248394982CAB
:108C5000AA24AA94BA2C512C44244394DD24D394FE
:108C60001BCF61E0CE018F549F4F0E940C36A2961D
:108C70002FAFA297A3963FAFA397A4964FAFA49709
:108C8000A5965FAFA597A6966FAFA697A7967FAF5D
:108C9000A797A8968FAFA897A9969FAFA997882462
:108CA0008394982CAA24AA94BA2C512C442443943B
:108CB000D12CF2CE40E050E061E070E0C1010E94B2
:108CC0001E3F672B682B692B89F040E050E061E084
:108CD00070E0C1010E941A3E8824839494E0992E8A
:108CE000AA24A394B12C512C412CCEC040E050E0DA
:108CF00061E070E0C1010E94433EEECF85E0882E26
:108D0000912CA12CB12CC0CC8AE06816710409F416
:108D1000C8C19BE06916710409F0F1CCCE54DF4F55
:108D20008881C25BD04082958F70823009F032C258
:108D3000C501B40124E630E040E050E00E94D6D303
:108D4000CA54DF4F8881C65BD04090E0280F391F9E
:108D500037FF02C030E020E02536310514F024E66C
:108D600030E0CA54DF4F2883C65BD04062E0CE01BA
:108D70008F549F4F0E94E5352A962FAF2A972B9646
:108D80003FAF2B972C964FAF2C972D965FAF2D971B
:108D90002E966FAF2E972F967FAF2F9760968FAF3F
:108DA000609761969FAF6197D6C1412CD10119960A
:108DB0008D919C911A97009789F518968C9190E067
:108DC00010E5C12ED12CE12CF12C8530910549F014
:108DD000C12CD12C7601449721F0C12CD12C7601E5
:108DE000CA94CE54DF4FE881C25BD040E295EF7069
:108DF000E150EB3008F046C1F0E08827ED5FF84B1A
:108E00008F4F0C943FD41647164742484248424879
:108E10000F48CD47CD47CD4747474747DC01ED9148
:108E2000FC91048CF58DE02D1995CACFCB54DF4F02
:108E30001881C55BD040C501B40124E630E040E0B4
:108E400050E00E94D6D3DA01C901810F911DA11D06
:108E5000B11DB7FF03C080E090E0DC018F3F9105BA
:108E6000A105B10529F024F08FEF90E0A0E0B0E07B
:108E7000CB54DF4F8883C55BD040812CB2E19B2E61
:108E8000512CAA24AA94BA2CDD24DA9405CECB5412
:108E9000DF4F088119812A813B81C55BD040C254D4
:108EA000DF4F088319832A833B83CE5BD04014E6CF
:108EB00081169104A104B1040CF041C0A4E6B0E015
:108EC000C254DF4F288139814A815B81CE5BD0401B
:108ED0000E94F5D3860E971EA81EB91EC114D10498
:108EE000E104F104B9F0A70196010E94F5D3362FF1
:108EF000272FB501A40177FF03C040E050E0BA017D
:108F0000832E922E5C01481559056A057B0514F4E1
:108F10004A015B01CB54DF4F88829982AA82BB82CF
:108F2000C55BD040CE54DF4F8881C25BD0408F708C
:108F30008066CE54DF4F8883C25BD0409ECFC50190
:108F4000B40124E630E040E050E00E94D6D3C254A1
:108F5000DF4F88819981AA81BB81CE5BD040280FE9
:108F6000391F4A1F5B1FC114D104E104F10461F0F1
:108F700057FF03C020E030E0A901C216D306E40683
:108F8000F50614F4A7019601CB54DF4F28833983EB
:108F90004A835B83C55BD04070CFCB54DF4F688181
:108FA00079818A819B81C55BD0400E943CD5C254A7
:108FB000DF4F688379838A839B83CE5BD040C50172
:108FC000B40124E630E040E050E00E94D6D3C25421
:108FD000DF4F688179818A819B81CE5BD040620FAF
:108FE000731F841F951FC114D104E104F10461F0C3
:108FF00097FF03C060E070E0CB01C616D706E80615
:10900000F90614F4C701B6010E9471D2CB54DF4FA8
:10901000688379838A839B83C55BD0402ECFCB54F2
:10902000DF4F88819981AA81BB81C55BD040880EC2
:10903000991EAA1EBB1EC114D104E104F104C9F09B
:10904000A4E6B0E0A70196010E94F5D3362F272FA2
:10905000B501A40177FF03C040E050E0BA01832EC0
:10906000922E5C01481559056A057B0514F44A01E6
:109070005B01CB54DF4F88829982AA82BB82C55B99
:10908000D040FBCE88E0FE013196DE01AF54BF4FE9
:1090900001900D928A95E1F7912C812C55245394DF
:1090A000F0CECE54DF4F8881C25BD04082958F7066
:1090B000823009F055C0C501B40124E630E040E03B
:1090C00050E00E94D6D3C954DF4F8881C75BD0409F
:1090D000C854DF4F6881C85BD040962F9170280F2D
:1090E000391F2E3691E039072CF437FF05C02DE6E5
:1090F00031E002C030E020E0C954DF4F2883C75B75
:10910000D040C854DF4F8881C85BD04030FB80F925
:10911000C854DF4F8883C85BD04062E0CE018F54D3
:109120009F4F0E94E53562962FAF629763963FAFDF
:10913000639764964FAF649765965FAF6597669641
:109140006FAF669767967FAF679768968FAF6897A0
:1091500069969FAF6997812CA2E19A2E512C18C075
:1091600088E0FE013196DE01AF54BF4F01900D92B1
:109170008A95E1F767EA79E088E999E00E94358706
:1091800088E999E00E945885912C812C55245394AC
:10919000412C77CE88E0FE013196DE01AF54BF4FFF
:1091A00001900D928A95E1F76BE979E0E5CFC35420
:1091B000DF4F1881CD5BD040112309F46CC01296AB
:1091C000ED91FC9180858F70853009F075C0CD538D
:1091D000DF4FE881F981C35CD040359709F46CC05A
:1091E000C1010E94F55921E0181619060CF020E083
:1091F000D22EC754DF4F48815981C95BD040CE532E
:10920000DF4F2881C25CD040BE016F547F4FD10137
:1092100012968D919C910E942E59B1E06B167104AB
:1092200009F04AC0CE54DF4F8881C25BD040807FB6
:1092300009F442C0CE53DF4FC880C25CD040ED2C51
:10924000C755DF4F0881C95AD040C655DF4F188136
:10925000CA5AD040C555DF4F2881CB5AD040C4559B
:10926000DF4F3881CC5AD040C355DF4F4881CD5AAB
:10927000D040C255DF4F5881CE5AD040C155DF4F44
:109280006881CF5AD040C055DF4F7881C05BD04055
:10929000C1010E949E40CF54DF4F8881C15BD04006
:1092A000853009F444C170F48330C9F1C554DF4FEF
:1092B0001882CB5BD040B8C0C354DF4F1882CD5B5F
:1092C000D040E9CF863009F47CC0873079F7C101FE
:1092D0000E94441E182F863009F062C063E479E0D2
:1092E0008FE39AE00E94358766E070E08FE39AE0B2
:1092F0000E943D9D8FE39AE00E94588562E0CE0176
:109300008F549F4F0E940C3629AF3AAF4BAF5CAFE2
:109310006DAF7EAF8FAF21969FAF21973DC0C1014A
:109320000E94441E853021F093E0A92EB12CFFC18C
:109330006AE579E08FE39AE00E94358765E070E0A6
:109340008FE39AE00E943D9D8FE39AE00E9458854A
:10935000B101CE018F549F4F0E94CC9D61E0CE01A0
:109360008F549F4F0E940C3622962FAF2297239640
:109370003FAF239724964FAF249725965FAF25974D
:1093800026966FAF269727967FAF279728968FAFA1
:10939000289729969FAF2997689480F890F886CFF0
:1093A00065E279E08FE39AE00E943587612F70E0F3
:1093B0008FE39AE00E943D9D8FE39AE00E945885DA
:1093C000B3CF40E050E061E070E0C1010E941E3F79
:1093D000672B682B692B09F0A7C0EFEFDE129AC04C
:1093E000C1010E94F559181619060CF496C0B10176
:1093F000CE018F549F4F0E94CC9D61E0CE018F54CF
:109400009F4F0E940C3629AB3AAB4BAB5CAB6DABBC
:109410007EAB8FAB98AF689480F890F8F6E0C554B7
:10942000DF4FF883CB5BD04084010160CE54DF4F27
:109430008881C25BD040982F9F70923050F4CF54F7
:10944000DF4F9881C15BD040992319F084010160FE
:109450001160807F09F491C01260C354DF4F2881EE
:10946000CD5BD04021111D7FA801B101CE018F54E9
:109470009F4F0E946C3E4801AA24A394B12C511026
:1094800094C5D10119968D919C91009709F06FC3F5
:1094900040E050E062E070E0C1010E941E3F672B97
:1094A000682B692B09F495C367EC77E088E999E0AC
:1094B0000E94358788E999E00E94588592FCBCC4D7
:1094C00065EB77E08FE39AE00E943587B5018FE383
:1094D0009AE00E943D9D6EEA77E08FE39AE00E9459
:1094E00035870E9458A6AB01BC01CB53DF4F0881E2
:1094F00019812A813B81C55CD040401B510B620B16
:10950000730B8FE39AE00E94339D8FE39AE00E94F1
:1095100058850DC1DD2009F46ACF6BE079E08FE357
:109520009AE00E94358700CF66EF78E0F8CF0FEF22
:10953000D01209C0C1010E94F559181619062CF065
:1095400069ED78E0ECCFDD20D9F362E0CE018F54F5
:109550009F4F0E940C3629A73AA74BA75CA76DA77F
:109560007EA78FA798AB689480F890F815E0C55453
:10957000DF4F1883CB5BD04057CF40E052E0B101C2
:10958000CE018F549F4F0E941F35811165CF65CF4B
:109590003FEFD312E7C0C1010E94F559DD24D394F7
:1095A000181619060CF4E1C0D12C6BEC78E08FE3AF
:1095B0009AE00E9435870D2D0D2C000C110BC25422
:1095C000DF4F19830883CE5BD040B8018FE39AE068
:1095D0000E943D9D64EC78E08FE39AE00E9435871D
:1095E000642D70E08FE39AE00E943D9D8FE39AE046
:1095F0000E945885C754DF4FE880F980C95BD0408E
:10960000E114F10409F4BAC061E374E2C7010E94F5
:1096100075CC01E010E0892B09F44BC06AE374E2D9
:10962000C7010E9475CC02E010E0892B09F441C00B
:1096300065E574E2C7010E9475CC05E010E0892B56
:10964000C1F16EE574E2C7010E9475CC06E010E03E
:10965000892B79F163ED74E2C7010E9475CC03E1B7
:1096600010E0892B31F16CED74E2C7010E9475CCDA
:1096700004E110E0892BE9F066EA74E2C7010E9478
:1096800075CC0EE010E0892BA1F06FEA74E2C701FF
:109690000E9475CC0FE010E0892B59F065EE74E262
:1096A000C7010E9475CC10E000E0892B11F405E1A0
:1096B00010E0C1010E94441E282F30E0C554DF4F46
:1096C00039832883CB5BD040232B61F4C254DF4F16
:1096D00088819981CE5BD040C554DF4F99838883C0
:1096E000CB5BD0400115110509F491C0C554DF4F83
:1096F000A881B981CB5BD040A017B107C9F168EA56
:1097000078E08FE39AE00E943587C554DF4F688187
:109710007981CB5BD0408FE39AE00E943D9D8FE33F
:109720009AE00E9458856DEFA62EBB24BA94C5011D
:10973000C853DF4F0FB6F894DEBF0FBECDBFDF9129
:10974000CF911F910F91FF90EF90DF90CF90BF903E
:10975000AF909F908F907F906F905F904F903F90D1
:109760002F900895DD2009F420CF442443941DCF89
:10977000C754DF4F19821882C95BD040B1E06B1625
:109780007104A9F4C354DF4FE881CD5BD040EE23D0
:1097900099F0CE54DF4F8881C25BD040807FF1E0EA
:1097A000C354DF4FF883CD5BD040811105C0C35453
:1097B000DF4F1882CD5BD040CF54DF4F0881C15BB3
:1097C000D040C554DF4F0883CB5BD040063108F052
:1097D000B8C1E02FF0E08827EF50F44B8F4F0C9486
:1097E0003FD4444C644D544D874C444C374DFD4C54
:1097F000CE4C444C444C9E4D9E4DAE4DAE4D7F4D97
:109800007F4DA14DA14DA14D7F4D7F4D7F4DF1016C
:1098100081859285009709F4B1CFDC01ED91FC912F
:109820000488F589E02DCE53DF4FA880C25CD0407C
:10983000C42CCF54DF4F0881C15BD040CE54DF4FE2
:109840001881C25BD040CD54DF4F2881C35BD0402C
:10985000CC54DF4F3881C45BD040CB54DF4F4881BC
:10986000C55BD040CA54DF4F5881C65BD040C95455
:10987000DF4F6881C75BD040C854DF4F7881C85B39
:10988000D04019950C940143C554DF4F1882CB5B2F
:10989000D040C354DF4F2881CD5BD040222309F450
:1098A000EECD3D2D3170E32ECE53DF4FC880C25C2C
:1098B000D040C755DF4F0881C95AD040C655DF4F49
:1098C0001881CA5AD040C555DF4F2881CB5AD040A5
:1098D000C455DF4F3881CC5AD040C355DF4F488143
:1098E000CD5AD040C255DF4F5881CE5AD040C155D5
:1098F000DF4F6881CF5AD040C055DF4F7881C05BC1
:10990000D040C1010E949E40E89491F8B8CDC101B9
:109910000E94441E853009F007CD63E978E08FE3AB
:109920009AE00E94358765E070E08FE39AE00E943C
:109930003D9D8FE39AE00E945885B101CE018F547E
:109940009F4F0E94CC9DD10118968C918530B9F41F
:109950006EE0CE018F549F4F0E940C3629A33AA38C
:109960004BA35CA36DA37EA38FA398A7689480F8F4
:1099700090F8C554DF4F1882CB5BD0406FC061E0D8
:10998000CE018F549F4F0E940C36298F3A8F4B8FF8
:109990005C8F6D8F7E8F8F8F98A3E8CFC1010E945F
:1099A000441E182F863031F56CE778E08FE39AE09B
:1099B0000E94358766E070E08FE39AE00E943D9D4B
:1099C0008FE39AE00E94588562E0CE018F549F4F4A
:1099D0000E940C36298B3A8B4B8B5C8B6D8B7E8B6C
:1099E0008F8B988F40E050E068E070E0C1010E94EA
:1099F0001A3EBCCF6EE578E0D5CC40E050E061E0A7
:109A000070E0C1010E941E3F672B682B692B61F536
:109A1000D11027C0B101CE018F549F4F0E94CC9D21
:109A200061E0CE018F549F4F0E940C3629873A8700
:109A30004B875C876D877E878F87988B40E050E0EF
:109A400068E070E0C1010E94433E689480F890F89D
:109A5000B6E0C554DF4FB883CB5BD0404424439479
:109A600018CF64E478E05BCD6FE278E058CDDD207C
:109A7000C1F062E0CE018F549F4F0E940C362983C3
:109A80003A834B835C836D837E838F83988768944E
:109A900080F890F8E5E0C554DF4FE883CB5BD04019
:109AA000DDCF62E178E03BCDCE54DF4F8881C25BF1
:109AB000D0408F70823008F05CCFC1010E94441EFC
:109AC000853009F053CF30CCCE54DF4F8881C25B54
:109AD000D0408F70823008F04CCFDD2081F069EFEC
:109AE00077E08FE39AE00E94358761E0C1010E9430
:109AF000151E60E071E1C1010E94423F15CCCE54B9
:109B0000DF4F8881C25BD040982F9F70923008F061
:109B100030CFC554DF4FF881CB5BD040FF2309F431
:109B20009DCF807F31F4B101CE018F549F4F0E94B1
:109B3000CC9D689480F803E0902A1BCF689492F83B
:109B400018CFCE54DF4F8881C25BD040807F19F49C
:109B5000689490F80ECF13E0912A0BCFC554DF4FD5
:109B60001882CB5BD040812C54E0952E77CFDC015E
:109B7000ED91FC91008CF18DE02DCF54DF4F0881E9
:109B8000C15BD040CE54DF4F1881C25BD040CD5472
:109B9000DF4F2881C35BD040CC54DF4F3881C45B9A
:109BA000D040CB54DF4F4881C55BD040CA54DF4F13
:109BB0005881C65BD040C954DF4F6881C75BD04035
:109BC000C854DF4F7881C85BD0401995811160CCB3
:109BD0006BCCF10181859285892B09F473C08114C6
:109BE000910439F0A401B101CE018F549F4F0E941E
:109BF0006C3ED10119968D919C91C754DF4FE8803E
:109C0000F980C95BD040DC01ED91FC910488F589B5
:109C1000E02DCE53DF4FA880C25CD040C42CCF547F
:109C2000DF4F0881C15BD040CE54DF4F1881C25B4B
:109C3000D040CD54DF4F2881C35BD040CC54DF4FA0
:109C40003881C45BD040CB54DF4F4881C55BD040E6
:109C5000CA54DF4F5881C65BD040C954DF4F68817A
:109C6000C75BD040C854DF4F7881C85BD04019959E
:109C70005C01F10181859285DC01ED91FC91048C00
:109C8000F58DE02D1995059711F4689480F892FCF4
:109C9000CBC0C554DF4FB881CB5BD040BB2321F094
:109CA0006B2FC1010E94151ECD53DF4FE881F98152
:109CB000C35CD040B401359709F402CCC1010E94C5
:109CC000423FFECB8085853009F474C0863009F7A9
:109CD000CF54DF4FD880C15BD040DD2009F46AC08B
:109CE000C1010E94AA9D8C018114910439F0A40144
:109CF000B101CE018F549F4F0E946C3E011511059A
:109D000041F2F12CE12C17FF06C0119501951109C4
:109D1000EE24E394F12CC80101978634910508F0F4
:109D2000B8CFC02E61E0802F0E94B4A4EFEFED0DFC
:109D3000E53110F5F0E08827EF55F14B8F4F0C948B
:109D40003FD4B64EB84EBC4EBC4EB84EB64EB84ED2
:109D5000BC4EBC4EBC4EBC4EBC4EBC4EB64EB64EBF
:109D6000BC4EBC4EBC4EBC4EB64EB64EF1E0EF26DD
:109D70006E2D8C2D0E9486A462EC77E08FE39AE032
:109D80000E943587B8018FE39AE00E943D9D60EC08
:109D900077E08FE39AE00E943587B7018FE39AE07E
:109DA0000E943D9D8FE39AE00E945885689480F858
:109DB00090F83AC08114910439F0A401B101CE01A8
:109DC0008F549F4F0E946C3E02E06016710481F137
:109DD00013E06116710429F06A94672809F059CFDD
:109DE000E5CFC1010E94B31D892B49F4D101ED914A
:109DF000FC91608171818EE694E00E9426AACE01DA
:109E00008F549F4F0E948D1520E030E048EC52E4C3
:109E10000E94D0D20E943CD56B0188E00E94991A22
:109E2000A601C1010E94A020AA24A394B12C31CF85
:109E3000689480F891F8F8CFCD53DF4F08811981ED
:109E4000C35CD0400530110509F43ACB40E054E042
:109E5000B101CE018F549F4F0E946C3E60E074E0D0
:109E60002DCF0E942E36672B682B692B11F00C9496
:109E70004244912C812C0C9473446114710409F0B8
:109E800045C08081882311F40C948642CE0187540A
:109E90009F4F0E94113C3C01CE54DF4F8881C25B32
:109EA000D0408F7071F5662DCE018F549F4F0E9468
:109EB000E535CF55DF4F2883C15AD040CE55DF4F0F
:109EC0003883C25AD040CD55DF4F4883C35AD04063
:109ED000CC55DF4F5883C45AD040CB55DF4F6883F1
:109EE000C55AD040CA55DF4F7883C65AD040C955AD
:109EF000DF4F8883C75AD040C855DF4F9883C85A70
:109F0000D0406114710411F40C9486426BEE79E038
:109F10008FE39AE00E943587B6018FE39AE00E94B2
:109F20003D9D64EE79E08FE39AE00E943587D10190
:109F3000ED91FC91608171818FE39AE00E94CF8660
:109F40006EED79E08FE39AE00E943587C754DF4FCA
:109F500068817981C95BD0408FE39AE00E94CF8607
:109F60006CED79E08FE39AE00E943587CE018F5443
:109F70009F4F0E948B33C754DF4F88819981C95B03
:109F8000D040009711F40C94C742FC012081243288
:109F900011F00C94C74268EC79E08FE39AE00E94DC
:109FA00035878FE39AE00E9458858CEFA82EBB245A
:109FB000BA94BDCB2F923F924F925F926F927F9255
:109FC0008F929F92AF92BF92CF92DF92EF92FF92C9
:109FD0000F931F93CF93DF93CDB7DEB7C957D10946
:109FE0000FB6F894DEBF0FBECDBF3C01562EE296F1
:109FF000EFAEE297E396FFAEE397E4960FAFE497F8
:10A00000E5961FAFE597E6962FAFE697E7963FAF49
:10A01000E797E8964FAFE897E9965FAFE997EA963A
:10A02000CFAEEA972D2C4A2C3B2C009709F466C141
:10A03000FC0180858F70843009F44BC128F488239B
:10A0400009F450C180E02DC0853009F444C0863049
:10A05000C9F76DE774E0C3010E9496984C01009720
:10A0600009F46FC0B12CA12CD12CC12CE296EFAC1D
:10A07000E297E396FFACE397E4960FADE497E5969D
:10A080001FADE597E6962FADE697E7963FADE797CC
:10A09000E8964FADE897E9965FADE997652D0E9488
:10A0A000DA4FC758DF4F0FB6F894DEBF0FBECDBFF3
:10A0B000DF91CF911F910F91FF90EF90DF90CF90A4
:10A0C000BF90AF909F908F907F906F905F904F90D8
:10A0D0003F902F900895809119078F5F8093190703
:10A0E000868097808114910431F1A42CB32CEA96D8
:10A0F000CFACEA97D22CE296EFACE297E396FFACB6
:10A10000E397E4960FADE497E5961FADE597E696E5
:10A110002FADE697E7963FADE797E8964FADE89706
:10A12000E9965FADE997652DC4010E94DA4FF4010D
:10A1300082809380D7CF809119078150809319072F
:10A1400081CF61E874E0C3010E9496987C0166E8C3
:10A1500074E0C3010E9496986C01552039F0F1E03B
:10A160005F1609F497C010E000E00CC06BE874E0E3
:10A17000C3010E9496984C0160E974E0C3010E94FB
:10A1800096988C018114910409F44301011511057D
:10A1900009F48301E114F10421F4EA96EFACEA97A3
:10A1A000F22CC114D10411F4C42CD32C81149104C9
:10A1B00009F4A1C0F40180858F70843009F09BC040
:10A1C000818492840115110509F4A0C0F8018085ED
:10A1D0008F70843009F09AC06184728410E000E0CE
:10A1E000E114F10409F4F7C08114910409F4B4C036
:10A1F00064E779E18FE39AE00E943587F701618592
:10A2000072858FE39AE00E94CF866FE679E18FE353
:10A210009AE00E943587B4018FE39AE00E94CF86CE
:10A220008FE39AE00E945885CE018F589F4F0E947D
:10A230008B33C114D10409F06AC1F70180858F7096
:10A24000843009F062C161857285CE0101960E9459
:10A25000453CCE0101960E9442168823B1F00E942F
:10A26000FC2C6B01683C71050CF08AC06AE379E153
:10A2700088E999E00E943587B60188E999E00E9453
:10A280003D9D88E999E00E945885CE0101960E9483
:10A2900078163BC165E974E0C3010E9496984C01B1
:10A2A0006AE974E0C3010E9496988C0181149104BC
:10A2B00009F032C16BE874E0C3010E9496984C012A
:10A2C0000115110509F458CF892B09F063CF43011B
:10A2D00061CF10E000E0912C812CD12CC12CF12C0D
:10A2E000E12C50CF10E000E0912C812CD12CC12C1E
:10A2F000F12CE12C4FCF912C812C64CFCA2CDB2C7C
:10A30000EA96EFACEA97F22C912C812C00E020E049
:10A3100033E040E150E0BE016F597F4FCE018F58CE
:10A320009F4F0E946A313C01E3968FADE397082F5F
:10A330000F7010E00115110509F052CFE2969FADA4
:10A34000E297911106C0807F09F44ACF02E010E045
:10A3500047CF01E010E044CF65E679E18FE39AE072
:10A360000E943587F701618572858FE39AE00E942C
:10A37000CF8660E679E18FE39AE00E94358754CF7B
:10A380008114910431F0B401CE0101960E945F9EC8
:10A390007CCFA12CCC24C394F12CE12CE2960FAD00
:10A3A000E297E3961FADE397E4962FADE497E59629
:10A3B0003FADE597E6964FADE697E7965FADE79739
:10A3C000E8966FADE897E9967FADE997CE010196E3
:10A3D0000E94CE415ACFC114D10409F496C0611431
:10A3E000710409F492C0F60180858F70843009F001
:10A3F00088C08185928525961FAE1EAE259748EEB2
:10A4000053E060E070E029964CAF5DAF6EAF7FAF78
:10A41000299725EB32E023963FAF2EAF23972F9657
:10A420009FAF8EAF2F9761961FAE1EAE619763965A
:10A430001FAE1EAE639765961FAE1EAE65976796FC
:10A440001FAE1EAE679769961FAF0EAF699740E4C7
:10A4500050E0BE016F5F7F4FCE018F5B9F4F0E9428
:10A460003D9A21E030E02C0F3D1F820F931FFC012D
:10A47000108268E579E18FE39AE00E943587F60162
:10A48000618572858FE39AE00E94CF866FE974E060
:10A490008FE39AE00E94CF86BE016F5F7F4F8FE30C
:10A4A0009AE00E94CF8663E579E18FE39AE00E940B
:10A4B0003587B3018FE39AE00E94CF868FE39AE05D
:10A4C0000E9458850E94B4988823D9F08091D208C0
:10A4D000811117C06FE270E0CE0101960E9495D8FD
:10A4E000892B51F4F6012185328543E050E060E488
:10A4F000CE0101960E94932BB301CE0101960E94DA
:10A5000026A7E114F10409F098CE81E0CACD6114C8
:10A51000710409F068CF91CE892B09F03BCE2CCE87
:10A520004F925F926F927F928F929F92AF92BF9263
:10A53000CF92DF92EF92FF920F931F93CF93DF930F
:10A54000CDB7DEB769970FB6F894DEBF0FBECDBFAB
:10A550000E9458A69B01AC0160915306709154066D
:10A560008091550690915606A12CB12C650118E8F2
:10A57000E12E13E1F12E00E010E00E94312B882340
:10A5800049F1E091AC06F091AD068281823041F054
:10A590008430B9F1813009F040C068E878E133C017
:10A5A00063EB78E188E999E00E94358788E999E0D2
:10A5B0000E9458858091AC069091AD060E9452276A
:10A5C0000E9458A6609353067093540680935506D4
:10A5D0009093560669960FB6F894DEBF0FBECDBFB6
:10A5E000DF91CF911F910F91FF90EF90DF90CF906F
:10A5F000BF90AF909F908F907F906F905F904F90A3
:10A6000008956AE978E188E999E00E94358788E948
:10A6100099E00E9458850E947929E0905106F090B7
:10A620005206E114F10431F0E0912107F091220784
:10A63000309759F46AE778E188E999E00E94358714
:10A6400088E999E00E945885BBCF80914F06909190
:10A650005006892B61F480858F70863041F48681A5
:10A660009781009721F09093500680934F06E091D8
:10A67000AC06F091AD06309721F083E198E696871D
:10A680008587E0914F06F0915006309709F448C154
:10A69000BE016E5E7F4F808191810E9425148823C8
:10A6A00009F43EC18A89883209F03AC1AE014F5F90
:10A6B0005F4FBE016E5E7F4FC7010E94E827811188
:10A6C00007C0C12CD12C2EEFE22E22ECF22E3DC081
:10A6D0006A8170E0762F6627770F770F770F2981D1
:10A6E00048E0249F90011124262B372B8A89803142
:10A6F000D1F4688570E08F81FB01E81BF109CF017F
:10A700009695982F8827979587950E942BD4CB01F3
:10A710004097B90153E0660F771F5A95E1F76078CB
:10A720009C01260F371F2138F4EE3F0754F2B90180
:10A73000330F880B990B0E9471D220E030E040E08B
:10A740005CE30E94D0D26B017C0180904F06909018
:10A7500050068114910409F480C0809121079091E2
:10A760002207892B09F479C0C4010E9414155C01E9
:10A770008FE39AE00E94588565E778E18FE39AE0DD
:10A780000E94358722E0B701A6018FE39AE00E947C
:10A79000638562E778E18FE39AE00E943587F401F0
:10A7A000608171818FE39AE00E94CF866FE678E145
:10A7B0008FE39AE00E94358720E030E04EEF52ECC4
:10A7C000C701B6010E946AD2882309F4B4C020E010
:10A7D00030E04AEA52E4C701B6010E946AD28823F7
:10A7E00009F4A9C020E030E0A901C701B6010E9428
:10A7F0006AD2882309F49FC0A114B10429F0B501DD
:10A800008FE39AE00E94CF868FE39AE00E945885FA
:10A8100019821A821B821C828A818F7080678A83C8
:10A82000CD82DE82EF82F88663E0CE0101960E943F
:10A83000E5352A873B874C875D876E877F87888BC6
:10A84000998BB12CA12CD12CC12C79018A019B01AF
:10A85000AC016FEFC4010E94DA4FE0905106F09016
:10A8600052068A89803109F47AC0BE016E5E7F4F3C
:10A87000C7010E940228182F882309F451C0F7014C
:10A88000858196810E945227882309F449C0BE0120
:10A890006E5E7F4FF701858196810E942527F70123
:10A8A000408164E4858196810E94FF26F7018281C0
:10A8B0008823B1F119508EEE882E82E0982E133045
:10A8C00040F4E12FF0E0EE0FFF1FE555FD4F8080D3
:10A8D0009180F7018381882309F443C0808181112D
:10A8E00040C00E9458A62B013C01092C000CAA086C
:10A8F000BB08AE014F5F5F4FBE016E5E7F4FC70169
:10A900000E949327898181110BC00E9458A6681963
:10A9100079098A099B09641575058605970548F329
:10A92000E0914F06F09150068281938190935006FA
:10A9300080934F0645CEA114B10409F48ECF6EE585
:10A9400078E18FE39AE00E943587B5018FE39AE0C2
:10A950000E94CF868FE39AE00E9458857ECF1CE04C
:10A960008ECFB401990C880B990B0E9425A6D8CFE5
:10A970006F927F928F929F92AF92BF92CF92DF920F
:10A98000EF92FF920F931F93CF93DF93CDB7DEB774
:10A99000A0970FB6F894DEBF0FBECDBF8C01862EF8
:10A9A0007A01DC018D919C911197892B09F460C08B
:10A9B0001496ED91FC91309709F45AC08081807112
:10A9C000BFEF6B1357C0B1F481E0A0960FB6F894B7
:10A9D000DEBF0FBECDBFDF91CF911F910F91FF90D2
:10A9E000EF90DF90CF90BF90AF909F908F907F902F
:10A9F0006F9008954330510539F3818082942FE0A0
:10AA0000822266E577E08FE39AE00E943587D801DD
:10AA100013966C918FE39AE00E94369D64E577E08F
:10AA20008FE39AE00E943587D8011496ED91FC914E
:10AA300061816F708FE39AE00E94369D61E577E057
:10AA40008FE39AE00E943587682D8FE39AE00E9499
:10AA5000369D8FE39AE00E945885D8011496ED91B7
:10AA6000FC9181818F70881207C080818F7E8083E6
:10AA700080E0ABCF8111FCCF198E1A8E1B8E1C8EFD
:10AA80001D8E1E8E1F8E18A28A8D8F708A8FD80100
:10AA90001496ED91FC9181818F70881579F1B3E066
:10AAA000EB16F10459F16FE477E08FE39AE00E942E
:10AAB0003587F80163818FE39AE00E94369D6DE44B
:10AAC00077E08FE39AE00E943587D8011496ED91E4
:10AAD000FC9161816F708FE39AE00E94369D6AE479
:10AAE00077E08FE39AE00E943587682D8FE39AE044
:10AAF0000E94369D8FE39AE00E945885F8012081DC
:10AB00003181FCE0F81508F416C1E82DF0E0882743
:10AB1000E357FA4A8F4F0C943FD49A55D75558565D
:10AB20006F567B565856315658567E56895645565E
:10AB30008C569856D8011496CD90DC90F601818100
:10AB40008F70853009F4F7C050F48230C1F060EBAB
:10AB500074E0C9010E9496983C01912C4BC087304B
:10AB6000D1F08A30A1F769EA74E0C9010E94969891
:10AB70003C01D6019C9092FA992490F83BC063EA7C
:10AB800074E0C9010E9496983C01D6019C9090FA0D
:10AB9000992490F82FC062EA74E0C9010E94969847
:10ABA0003C01F601908091FA992490F823C065EB5E
:10ABB00074E0C9010E9496983C01D8011496ED9169
:10ABC000FC91808180FB992490F8982F9E7F80FFD4
:10ABD000916090836114710469F461E0CE0149963B
:10ABE0000E940C36298B3A8B4B8B5C8B6D8B7E8B4A
:10ABF0008F8B988FF801A080B18061E874E0C50167
:10AC00000E9496986C0166E874E0C5010E949698CF
:10AC10005C01892B81F4C114D10469F460E0CE0198
:10AC200049960E940C3629833A834B835C836D835B
:10AC30007E838F839887D8011496ED91FC916114DF
:10AC4000710409F07CC0898D811179C0B82DBF7065
:10AC50008B2E8181807F882A818280818F7E808374
:10AC6000B3CE6AEB74E0C9010E9496983C01D8010A
:10AC70001496ED91FC91808181FB992490F8982F96
:10AC80009D7F81FF92609083B5CF60EC74E0C90135
:10AC90000E9496983C01D8011496ED91FC91808118
:10ACA00082FB992490F8982F9B7F82FF9460EBCFD2
:10ACB00060EB74E0C9010E9496983C01892B09F071
:10ACC0004CCF62E0CE0149960E940C3629873A8724
:10ACD0004B875C876D877E878F87988B3ECF66EC2E
:10ACE00074E0C9010E9496983C01D8011496ED9138
:10ACF000FC9190804CCF6BEC74E0F3CF61ED74E08D
:10AD0000C9010E9496983C01D8011496ED91FC91DE
:10AD100049CF67ED74E0F4CF6EED74E0C9010E9495
:10AD200096983C01D8011496ED91FC91908023CF28
:10AD300064EE74E0F3CF912C712C612C5BCF83E037
:10AD4000E816F104B9F0982D9F70892E8181807FDB
:10AD5000882A818280818F7E8083E98CFA8C0B8D9A
:10AD60001C8D2D8D3E8D4F8D58A1692DC3010E94E4
:10AD7000DA4F2ACE81818F70881509F425CE82940E
:10AD800090EF8922882A81828081806168CF2F920A
:10AD90003F924F925F926F927F928F929F92AF926B
:10ADA000BF92CF92DF92EF92FF920F931F93CF93B8
:10ADB000DF93CDB7DEB763970FB6F894DEBF0FBE53
:10ADC000CDBF4C013B0140E058E060E070E00E94E4
:10ADD0001E3F672B682B692B09F45CC019821A820D
:10ADE0001B821C821D821E821F8218868A818F70A0
:10ADF0008A8340E053E0B401CE0101960E941F35E2
:10AE0000D40119968D919C91892B09F443C040E09F
:10AE100058E060E070E0C4010E941A3E69E47AE004
:10AE20008FE39AE00E943587F40181859285DC01E9
:10AE3000ED91FC910488F589E02DA12CCC24C394DC
:10AE4000F12CE12C09811A812B813C814D815E819D
:10AE50006F81788519958F3F9807E1F0D401ED91C6
:10AE6000FC9160817181892B09F0B8C08FE39AE071
:10AE70000E94CF8667E47AE08FE39AE00E943587EC
:10AE80006FE37AE08FE39AE00E9435878FE39AE0E0
:10AE90000E94588565E0F401808191810E940E999D
:10AEA0006C01009709F4D0C0DC011896BC91B98BF5
:10AEB000BB2EB2942FE0B222FC0121843284438461
:10AEC00054840E9458A6BB2009F4BEC0261A370A33
:10AED000480A590A19861A861B861C86B9861A855D
:10AEE0001F70106A1A872D863E864F86588AF4E0B6
:10AEF0006F16710439F5E12C90E2F92E0B2D2B859C
:10AF00003C854D855E856F857889C4010E9441A787
:10AF1000C201B10128EE33E040E050E00E94D6D3F8
:10AF2000BA01A9012AE030E08FE39AE00E94498645
:10AF300060E77AE08FE39AE00E9435878FE39AE03A
:10AF40000E94588557FE80C022E022163104410439
:10AF500020E852060CF478C00E94FC2C1B017B8B6D
:10AF60006A8BE12C80E2F82E09851A852B853C85B9
:10AF70004D855E856F857889C4010E9441A78A89C5
:10AF80009B89883C9105BCF567E57AE088E999E002
:10AF90000E943587B10188E999E00E943D9D88E9CA
:10AFA00099E00E9458858FEF9FEF63960FB6F89453
:10AFB000DEBF0FBECDBFDF91CF911F910F91FF90EC
:10AFC000EF90DF90CF90BF90AF909F908F907F9049
:10AFD0006F905F904F903F902F9008958FE39AE08D
:10AFE0000E94CF866DE37AE08FE39AE00E94358776
:10AFF00069E37AE047CFD60118968C9118978F7045
:10B0000018968C9319821A821B821C821D821E82C2
:10B010001F8218868A818F708A83B98289898F708E
:10B02000AA24A394873009F0A12CCC24C394F12C3A
:10B03000E12C09811A812B813C814D815E816F81D8
:10B040007885C4010E94CE41B1E06B167104E9F429
:10B0500040E053E060E070E0C4010E941E3F6115D3
:10B0600071058105910589F020911D0730911E071A
:10B070002630310551F4C4010E94423F40E053E0C4
:10B0800060E070E0C4010E941A3EF401818592855F
:10B09000009719F490E080E088CFDC01ED91FC91FD
:10B0A0000284F385E02D1995892BA1F3F4018185A4
:10B0B0009285DC01ED91FC910480F581E02DB301D6
:10B0C000199573CFAF92BF92CF92DF92EF92FF921A
:10B0D0000F931F93CF93DF93CDB7DEB76D970FB666
:10B0E000F894DEBF0FBECDBF0E9458A69B01AC01F5
:10B0F0006091490670914A0680914B0690914C06EA
:10B10000A12CB12C650118EEE12E13E0F12E00E028
:10B1100010E00E94312BF82E882351F00E9458A68F
:10B120006093490670934A0680934B0690934C06B1
:10B13000809119078F5F80931907E0911F07F091A5
:10B1400020070681178194E0C92ED12CF11003C08D
:10B1500082E0C82ED12CA0901F07B0902007A11428
:10B16000B10429F10115110511F1F80180858F70E5
:10B170008530A9F7C8010E949A9D823080F3B801FA
:10B18000CE0101960E94DF21CE0101960E94421657
:10B19000882329F0B601CE0101960E94C756F80116
:10B1A00002811381CE0101960E947816D4CF80913E
:10B1B000190781508093190780911D0790911E07F0
:10B1C0000597D9F1FF20C9F110E060914706709111
:10B1D00048066115710589F111112FC0FB018085A9
:10B1E0008F70853091F4CE0101960E94DF2161E0DD
:10B1F00070E0CE0101960E94C75611E0892B09F438
:10B2000010E0CE0101960E947816E0914706F09179
:10B210004806309791F082819381909348068093FD
:10B220004706892B91F6E0911F07F0912007868150
:10B23000978190934806809347066D960FB6F894D1
:10B24000DEBF0FBECDBFDF91CF911F910F91FF9059
:10B25000EF90DF90CF90BF90AF9008952F923F92E4
:10B260004F925F926F927F928F929F92AF92CF9206
:10B27000DF92EF92FF920F931F93CF93DF93CDB79F
:10B28000DEB76D970FB6F894DEBF0FBECDBF009747
:10B2900009F4A9C0FC0130853F70353009F0A3C026
:10B2A000D22E1A014B0166807780809119078F5F3B
:10B2B000809319076114710409F490C0F30180852B
:10B2C0008F70843009F086C06185728580911F0778
:10B2D000909120070E9496982C01009709F47AC05B
:10B2E000FC0180858F70853009F074C0B201CE01F9
:10B2F00001960E94DF2181149104B1F0CE010196E4
:10B300000E944216882381F0AD2CC12C7101F401FA
:10B310000081118122813381448155816681778149
:10B32000CE0101960E94CE4160E0C2010E940E99BA
:10B330000097E9F1FC0120852F702230C1F581854D
:10B340009285A385B4850797A105B10581F561E0D4
:10B35000C2010E940E992D2DA101B4010E942E5907
:10B360008114910499F5882389F1809119078150FE
:10B3700080931907CE0101960E94781681E06D96A0
:10B380000FB6F894DEBF0FBECDBFDF91CF911F91F6
:10B390000F91FF90EF90DF90CF90AF909F908F90A4
:10B3A0007F906F905F904F903F902F900895811401
:10B3B000910461F4CE0101960E944216882331F077
:10B3C000CE0101960E94F559892B79F6CE0101969E
:10B3D0000E947816F301628073806CCF8091190708
:10B3E00081508093190780E0CACFDF92EF92FF92DD
:10B3F0000F931F93CF93DF9300D000D01F921F9223
:10B40000CDB7DEB77C0119821A821B821C821D8295
:10B410001E821F8218868A818F708A83D701ED91E0
:10B42000FC91608171818FE39AE00E94CF8667E38F
:10B430007AE08FE39AE00E943587C7010E944216A6
:10B4400081111BC06EE27AE08FE39AE00E9435879B
:10B450008FE39AE00E9458850FEF1FEFC8012896EE
:10B460000FB6F894DEBF0FBECDBFDF91CF911F9115
:10B470000F91FF90EF90DF900895C7010E94441E46
:10B48000D82EF70181859285009791F0DC01ED912E
:10B49000FC910688F789E02D19958C0197FD08C06D
:10B4A00081E00115110509F480E00E947C1BD6CFD4
:10B4B000F7018085873009F42EC0EFEFED0DE43100
:10B4C00050F5F0E08827E859F54A8F4F0C943FD4A7
:10B4D0007C5A855A8B5A8B5A855A7C5A8B5A8B5A6E
:10B4E0008B5A8B5A8B5A8B5A8B5A7C5A8B5A8B5A43
:10B4F0008B5A8B5A7C5A7C5A6FE07AE08FE39AE041
:10B500000E94358701E010E0A9CF80E00E947C1BFB
:10B5100010E000E0A3CF40E052E0B701CE01019679
:10B520000E941F35D70118968C911897873071F1BA
:10B5300060F4833009F454C0843061F06FE17AE044
:10B540008FE39AE00E943587E3CF883009F448C042
:10B550008930A1F7CE0101960E941D998C0164E10A
:10B560007AE08FE39AE00E943587B8018FE39AE092
:10B570000E943D9D8FE39AE00E94588591E080E013
:10B58000012B09F490E0092F182F68CF1296ED9146
:10B59000FC9180858F7010E000E0853001F76CE24F
:10B5A0007AE08FE39AE00E94358720E050E040E0A7
:10B5B00070E060E0F701828193810E942E59F82E9D
:10B5C000082F10E069E27AE08FE39AE00E94358765
:10B5D0008F2D0E947C1B8FE39AE00E9458853ECFFE
:10B5E000CE0101960E942E368B01B9CF2F923F9249
:10B5F0004F925F926F927F928F929F92AF92BF9283
:10B60000CF92DF92EF92FF920F931F93CF93DF932E
:10B61000CDB7DEB760970FB6F894DEBF0FBECDBFD3
:10B620006130710509F494C0DC0112966D917C9132
:10B630006115710509F48CC04C0119821A821B82B4
:10B640001C821D821E821F8218868A818F708A83C7
:10B6500040E052E0CE0101960E941F35CE010196D6
:10B660000E941D991C01F401828193810E94B31DE7
:10B670002B013C01D40117962D913D914D915C9188
:10B680001A97D1010E9400D42FEF30E040E050E043
:10B690000E94B4D329873A874B875C870E9458A6BB
:10B6A0009B01AC0189859A85AB85BC850097A10576
:10B6B000B10509F468C0A12CB12C65017C018D0194
:10B6C000C301B2010E94312B8987411451046104E6
:10B6D0007104F1F1D40117968D919D910D90BC915B
:10B6E000A02D8D879E87AF87B88B0E9458A69B019F
:10B6F000AC018D859E85AF85B8890097A105B10500
:10B7000061F0A12CB12C65017C018D01C301B20156
:10B710000E94312B882309F451C0D40112966D90F8
:10B720007C9080E00E94991AAB01BC01C3010E9489
:10B73000A020232869F0F40184810E94D013D40151
:10B7400016969C91891304C061E0C4010E94511EA9
:10B7500090E080E060960FB6F894DEBF0FBECDBFDC
:10B76000DF91CF911F910F91FF90EF90DF90CF90DD
:10B77000BF90AF909F908F907F906F905F904F9011
:10B780003F902F90089591E099879FCFB985BB2373
:10B79000F1F060E0C4010E94511EF40182819381A6
:10B7A0000E94F559892BA1F640E050E0BA01D4017E
:10B7B00012968D919C910E94A020CACFF4018481A1
:10B7C0000E94D013D40116969C918913DFCF2328B1
:10B7D00009F4BECFF40184810E94D013D4011696DF
:10B7E0009C918913B5CFB985B111B2CFADCFCF93AD
:10B7F000DF93EC0162ED77E18FE39AE00E943587F9
:10B800006C817D818FE39AE00E943D9D6CEC77E135
:10B810008FE39AE00E9435878FE39AE00E94588573
:10B8200061E08C810E94B4A46E818C810E9486A408
:10B830008A819B81009729F040E050E0BA010E9484
:10B84000A020E881F9810484F585E02D62E0CE0135
:10B8500019958A819B810E94F559181619065CF486
:10B860000A80DB81C02D80E00E94991AAB01BC01E7
:10B87000CE010E94A02081E090E0DF91CF91089559
:10B880002F923F924F925F926F927F928F929F92F0
:10B89000AF92BF92CF92DF92EF92FF920F931F93DE
:10B8A000CF93DF93CDB7DEB7C955D1090FB6F89462
:10B8B000DEBF0FBECDBF0E9458A69B01AC016091B8
:10B8C0004306709144068091450690914606A12C4E
:10B8D000B12C650110E3E12E15E7F12E00E010E038
:10B8E0000E94312B882309F426C2E0911F07F091B2
:10B8F0002007309709F41FC2809119078F5F80934A
:10B9000019072680378010E02114310409F438C16A
:10B91000F10180858F708530F9F460E0C1010E94EB
:10B920000E99FC0181859285A385B4850597A105B3
:10B93000B10591F4B101CE0101960E94DF21CE0143
:10B9400001960E94421666968FAF6697811108C0D5
:10B95000CE0101960E947816F10122803380D4CF67
:10B9600025961CAE1DAE1EAE1FAE259729961CAEA9
:10B970001DAE1EAE1FAE299740E052E0BE016F5FC4
:10B980007F4FCE018F5B9F4F0E941F35CE010196E6
:10B990000E94B31D6B017C0169966FAF69976A962F
:10B9A000DFAE6A97CE0101960E94AA9D4C01CE019E
:10B9B0008F5B9F4F0E948D1565966CAF7DAF8EAFEC
:10B9C0009FAF6597CE0101960E94441E182FB601C5
:10B9D000DD0C880B990B0E9471D220E030E048EC1E
:10B9E00052E40E94CAD42B013C01CE0101960E9470
:10B9F000F55968969FAF8EAF68976FE077E18FE358
:10BA00009AE00E94358722E065964CAD5DAD6EAD43
:10BA10007FAD65978FE39AE00E94638569E077E1E7
:10BA20008FE39AE00E94358722E0B301A2018FE301
:10BA30009AE00E94638563E077E18FE39AE00E94D9
:10BA40003587612F70E08FE39AE00E943D9DE114FD
:10BA5000F10409F48EC088E00E94991A9B01AC01A0
:10BA600044275527B70190E080E0AA24AA94BA2C75
:10BA7000C12CD12C17E2E12E19E0F12E00E010E0EC
:10BA80000E94312B882371F1F1016081718188E975
:10BA900099E00E94CF8663EF76E188E999E00E9401
:10BAA0003587F101608171818BEE94E00E9426AAB6
:10BAB00090E080E0BC0169964FAD69976A965FADF2
:10BAC0006A97CE0101960E94A02062E070E0C40156
:10BAD0000E94271BCE0101960E94781666961FAD24
:10BAE00066973ACF20E030E048E152E4C301B2016A
:10BAF0000E9472D518163CF4F1016081718187EFC4
:10BB000094E00E9426AA68968EAD9FAD6897892B17
:10BB100019F461E070E0DBCF20E030E040E85FE363
:10BB200065966CAD7DAD8EAD9FAD65970E945DD481
:10BB30009B01AC01C301B2010E946AD270E060E0D7
:10BB400087FDC5CFA301920165966CAD7DAD8EAD2D
:10BB50009FAD65970E946AD21816DCF664EE76E116
:10BB60008FE39AE00E9435878FE39AE00E94588520
:10BB7000B1CF6AED76E18FE39AE00E943587AACFD4
:10BB8000809119078150809319070E9458A66093ED
:10BB900043067093440680934506909346060E94A0
:10BBA000FC2C2B013C010E9458A66B017C010E94D9
:10BBB000B498882309F489C08091D208811185C086
:10BBC00030E020E041E050E060E4CE0101960E94C8
:10BBD000932B4FE350E061EC7DE1CE0101960E9492
:10BBE0008ECC6BEF73E0CE0101960E948AD84FE3B2
:10BBF00050E061EB76E1CE0101960E948ECC2AE006
:10BC0000AE014F5B5F4FC301B2010E9419CDBE016F
:10BC10006F5B7F4FCE0101960E9426A730E020E0A7
:10BC200041E050E060E4CE0101960E94932B4FE387
:10BC300050E061EC7DE1CE0101960E948ECC6BEF6D
:10BC400073E0CE0101960E948AD84FE350E06AEA81
:10BC500076E1CE0101960E948ECCC701B60128EE96
:10BC600033E040E050E00E94B4D3CA01B9012AE0B9
:10BC7000AE014F5B5F4F0E9419CDBE016F5B7F4FDE
:10BC8000CE0101960E9426A730E020E041E050E07E
:10BC900060E4CE0101960E94932B4FE350E061EFE8
:10BCA0007DE1CE0101960E948ECC4FE050E06BEE1C
:10BCB0007DE1CE018F5B9F4F0E94ACCCBE016F5BDC
:10BCC0007F4FCE0101960E9426A7112309F44DC093
:10BCD00064ED76E18FE39AE00E9435870E94FC2CA8
:10BCE000AB01BC018FE39AE00E94339D6CEC76E1DE
:10BCF0008FE39AE00E94358760911907062E000CA9
:10BD0000770B8FE39AE00E943D9D6AEB76E18FE32B
:10BD10009AE00E94358740913F065091400660911D
:10BD20004106709142068FE39AE00E94339D8FE3B3
:10BD30009AE00E945885C75ADF4F0FB6F894DEBFCD
:10BD40000FBECDBFDF91CF911F910F91FF90EF906C
:10BD5000DF90CF90BF90AF909F908F907F906F902B
:10BD60005F904F903F902F9008956AEC76E18FE3BB
:10BD70009AE00E9435870E94FC2CAB01BC018FE346
:10BD80009AE00E94339D62EC76E1B2CF2F923F920F
:10BD90004F925F926F927F928F929F92AF92BF92DB
:10BDA000CF92DF92EF92FF920F931F93CF93DF9387
:10BDB000CDB7DEB7C556D1090FB6F894DEBF0FBEBA
:10BDC000CDBFDC0114962D913C91232B09F43DC786
:10BDD0003B014C01FC0182819B0122503109223040
:10BDE000310508F0F8C5803409F4F7C208F04AC0FC
:10BDF000843008F085C2809103068F5F809303062C
:10BE0000A3016FEFC4010E94B854D40112960C91A3
:10BE100012970695017013961C9113978AEC810F67
:10BE2000803108F043C064E075E08D919C910E94E0
:10BE300096987C010097D1F1FC0180858F70853048
:10BE4000A9F580917E0A181324C080917F0A80345E
:10BE500001F58091800A9091810A5C01990FCC08CC
:10BE6000DD0860E0C7010E940E99FC018185928582
:10BE7000A385B485A816B906CA06DB060CF065C012
:10BE8000512C3EC0823409F4A8C208F439C280584B
:10BE9000AFCF10937E0A80E480937F0A812F0E94A7
:10BEA000F0A49093810A8093800AD7CF212F30E0AD
:10BEB000F901E152F04E8491F901E756F04E1491E8
:10BEC000F901ED5AF04EF490FF2009F43BC08111C6
:10BED0000E941FA4EF2DF0E0EE0FFF1FE952F94F73
:10BEE000A591B491EC911E2331E020E009F430E0FB
:10BEF000832F922F552453940817190609F0C0CFA9
:10BF0000F3E06F16710409F488C0D4011496ED9122
:10BF1000FC91E181EF70E150EC3008F07EC0F0E080
:10BF20008827EA56F04A8F4F0C943FD4B75F3361AD
:10BF3000ED5F236033613C60336170609D60B6608B
:10BF4000F8601A6190E080E0D5CF61E0C7010E94FF
:10BF50000E9955245394FC0181859285A385B4855F
:10BF60008A159B05AC05BD050CF0CACF89CF0E9490
:10BF700058A69B01AC0144275527D4011496ED9196
:10BF8000FC916281738190E080E0AA24AA94BA2C8B
:10BF9000C12CD12C18EEE12E13E0F12E00E010E0C0
:10BFA0000E94312B8823C9F1F4010081118166ECD4
:10BFB00074E0C8010E949698892B41F46BEC74E000
:10BFC000C8010E949698892B09F40EC142E050E006
:10BFD00063E0C4010E94B85420C00E9458A69B018F
:10BFE000AC0144275527D4011496ED91FC91628150
:10BFF000738190E080E0AA24AA94BA2CC12CD12CA1
:10C000001CE2E12EFF24F39400E010E00E94312BAB
:10C0100042E050E064E0811184C0D4011496ED91B7
:10C02000FC91808183FB992790F9951509F4D2C181
:10C03000982F907E09F439C1982F907E90528F717D
:10C04000892B808358C10E9458A69B01AC014427CC
:10C050005527D4011496ED91FC916281738190E093
:10C0600080E0AA24AA94BA2CC12CD12C16E9E12E86
:10C07000F12C00E010E0CACF0E9458A69B01AC0151
:10C0800044275527D4011496ED91FC916281738168
:10C0900090E080E0AA24AA94BA2CC12CD12C18EEEE
:10C0A000E12E13E0F12E00E010E00E94312B8823F6
:10C0B00009F4B3CFF4010081118161ED74E0C8018E
:10C0C0000E949698892B41F467ED74E0C8010E94A4
:10C0D0009698892B09F488C042E050E068E079CF57
:10C0E0000E9458A69B01AC0144275527D401149601
:10C0F000ED91FC916281738190E080E0AA24AA9482
:10C10000BA2CC12CD12C1CE2E12EFF24F39400E0C8
:10C1100010E00E94312B42E050E069E0882309F4EE
:10C120007CCFC4010E94B8540E9458A6D401149632
:10C13000ED91FC917383628370CF0E9458A69B019E
:10C14000AC0144275527D4011496ED91FC916281EE
:10C15000738190E080E0AA24AA94BA2CC12CD12C3F
:10C1600016E9E12EF12C00E010E0D3CF0E9458A692
:10C170009B01AC0144275527D4011496ED91FC9105
:10C180006281738190E080E0AA24AA94BA2CC12C29
:10C19000D12C18EEE12E13E0F12E00E010E00E9409
:10C1A000312B882309F439CFF401008111816EED20
:10C1B00074E0C8010E949698892B39F464EE74E00B
:10C1C000C8010E949698892B21F042E050E06BE074
:10C1D00000CF60EC74E0C8010E94969842E050E005
:10C1E00066E0892B09F4F5CE42E050E06DE0F1CE37
:10C1F0000E9458A69B01AC0144275527D4011496F0
:10C20000ED91FC916281738190E080E0AA24AA9470
:10C21000BA2CC12CD12C1CE2E12EFF24F39400E0B7
:10C2200010E00E94312B882309F4F7CE42E050E061
:10C230006CE077CF0E9458A69B01AC01442755279C
:10C24000D4011496ED91FC916281738190E080E0BD
:10C25000AA24AA94BA2CC12CD12C16E9E12EF12CD7
:10C2600000E010E0DECF0E9458A69B01AC014427FD
:10C270005527D4011496ED91FC916281738190E071
:10C2800080E0AA24AA94BA2CC12CD12C18E5E12E66
:10C2900012E0F12E00E010E00E94312B882309F417
:10C2A000BCCE42E050E060E094CE0E9458A6D4019B
:10C2B0001496ED91FC91159773836283E181EF7081
:10C2C000552009F445C0E230F1F050F4EE23E9F1D5
:10C2D000D4011496ED91FC91808150FA83F9B1CE8E
:10C2E000E53089F0A3016AE0E73091F7C4010E94CC
:10C2F000B8548111EDCF80910306815080930306DD
:10C3000090E080E0A4C4F401008111816AEB74E044
:10C31000C8010E949698892BA9F461ED74E0C801C8
:10C320000E949698892B71F467ED74E0C8010E9411
:10C330009698892B39F462EA74E0C8010E949698B5
:10C34000892B19F0A30166E0D1CFA30161E0CECF24
:10C35000E150ED3008F0BCCFF0E08827ED54FE4905
:10C360008F4F0C943FD4C0616861C361C361686141
:10C37000C6616861E761E761E761E761E761C36141
:10C38000A30162E0B3CFA30165E0B0CF0D911C9192
:10C390006AEB74E0C8010E949698892BA9F461EDBC
:10C3A00074E0C8010E949698892B71F467ED74E0DF
:10C3B000C8010E949698892B39F462EA74E0C8019A
:10C3C0000E949698892B19F0A30167E08FCFA301F3
:10C3D00060E08CCF8F71806434CEB3E06B16710453
:10C3E00009F48ECF64E075E0F401808191810E94B0
:10C3F00096988C01D40113968C9190917E0A8913A2
:10C40000CEC090917F0A903409F0C9C08091800A13
:10C410009091810A3C010115110509F4F0C0F80161
:10C4200020852F70253009F0EAC0C8010E949A9D2E
:10C43000A4968FAFA497843008F4BDC063E0C80110
:10C440000E940E99DC0119968D919C916AE0D62E7E
:10C45000D89EF001D99EF00D1124A396FFAFEEAF48
:10C46000A39762E0C8010E940E99DC0119968D9194
:10C470009C91D89E7001D99EF00C112457010F2C6D
:10C48000000CCC08DD0861E0C8010E940E99A69658
:10C490009FAF8EAFA69760E0C8010E940E99FC0185
:10C4A00021843284438454849301072C000C440B70
:10C4B000550B2219330944095509A396AEADBFADFA
:10C4C000A397BD01BB0F880B990B6A197B098C09D7
:10C4D0009D090E94A4D3A696EEADFFADA697218537
:10C4E00032854385548522193309440955090E9430
:10C4F000D6D3A20EB31EC41ED51EA496FFADA4971C
:10C50000F53009F46BC081E090E0A396EEADFFAD8D
:10C51000A3971F01FF0F440855082A143B044C043D
:10C520005D040CF464C01501260197010F2C000C6A
:10C53000440B550B22163306440655060CF45CC01A
:10C54000A2019101A496FFADA497F23009F06BC04F
:10C550006301770CEE08FF0860E0C8010E940E99A5
:10C56000FC0181859285A385B485C816D906EA06A3
:10C57000FB060CF486C361E0C8010E940E99FC0121
:10C5800081859285A385B4858C159D05AE05BF0573
:10C590000CF0B6CE81E090E0A0E0B0E075C38093EF
:10C5A0007E0A90E490937F0A0E94F0A49093810AFF
:10C5B0008093800A2FCF8AE0869D5001879DB00C22
:10C5C00011240B2C000CCC08DD08F12CE12C20E010
:10C5D00038E2A3963FAF2EAFA39795CF64E0C80192
:10C5E0000E940E99DC0119968D919C918ECF662444
:10C5F0006A9453E0752E99CF712C612CA3CF2AE059
:10C60000289F5001299FB00C11249501BB0C440BAD
:10C61000550BF12CE12C80E098E2A3969FAF8EAFF2
:10C62000A39781E090E0D4011496ED91FC91628192
:10C630007381D301A61BB70BB7FF03C0B195A195BA
:10C64000B1098A179B070CF4C1C08081982F92957D
:10C6500096959770963008F0BCC09F5F9295990FA1
:10C66000907E8F71892BB4C0F70161857285DB01E3
:10C670008C91811196C3A114B10409F473C0D50142
:10C6800018968C9118978F70843009F06BC01996AA
:10C690006D917C91CE0101960E94453CCE010196A0
:10C6A0000E944216882309F459C06114710409F4E8
:10C6B00060C0E114F10431F0F70180858F7084309F
:10C6C00009F442C025961CAE1DAE1EAE1FAE2597C6
:10C6D00029961CAE1DAE1EAE1FAE299723961FAD28
:10C6E00023971F7023961FAF239781E022968FAF69
:10C6F0002297A12CCC24C394F12CE12C01E02496A8
:10C700002FAD249725963FAD259740E027965FAD46
:10C71000279728966FAD289729967FAD2997CE0148
:10C7200001960E94CE411AC00115110529F0F801A9
:10C7300080858F70843019F06BE075E032C36185BD
:10C740007285FB01808195CF61857285FB018081B7
:10C75000882321F0CE0101960E945F9ECE010196B2
:10C760000E947816D4011496ED91FC917382628236
:10C77000C7CD0115110531F0D80118968C918F7035
:10C780008430F1F025961CAE1DAE1EAE1FAE25976F
:10C7900029961CAE1DAE1EAE1FAE299723961FAD67
:10C7A00023971F7023961FAF239782E022968FAFA7
:10C7B0002297A12CCC24C394F12CE12C02E09FCF32
:10C7C000F80161857285DB018C91C2CF80818F7108
:10C7D00080838081803AB8F0C701FF0CAA0BBB0BA5
:10C7E00082179307A407B50771F0A396EEADFFADCE
:10C7F000A397CF01FF0FAA0BBB0B82179307A407C8
:10C80000B50709F07DCD6615770509F479CD6D96EC
:10C810001CAE1DAE1EAE1FAE6D976B968FAD6B97A7
:10C820008F7080666B968FAF6B976D968CAD9DAD5C
:10C83000AEADBFAD6D9765968CAF9DAFAEAFBFAFE0
:10C840006597AAE0B0E00E94F5D369966CAF7DAF22
:10C850008EAF9FAF699766EC76E08FE39AE00E9417
:10C860003587D40113966C918FE39AE00E94369D30
:10C8700064EC76E08FE39AE00E943587CE018F5A10
:10C880009F4F0E948B336DE774E0F40180819181AA
:10C890000E949698B12CA12CD12CC12C6296EFACA1
:10C8A00062976396FFAC639764960FAD6497659645
:10C8B0001FAD659766962FAD669767963FAD6797F4
:10C8C00068964FAD689769965FAD69976FEF0E9464
:10C8D000DA4FD4010D911C9161E874E0C8010E9407
:10C8E00096987C0166E874E0C8010E9496988C01D5
:10C8F0000097E1F1FC0180858F708430B9F5618586
:10C90000728540E450E0CE0101960E94CED86FE2DD
:10C9100070E0CE0101960E9495D8892B59F4D80178
:10C9200019962D913C9143E050E060E4CE010196D0
:10C930000E94932B00E020E032E040E150E0BE0195
:10C940006F5B7F4FCE018F5A9F4F0E946A310E94CA
:10C95000B498882359F08091D208811107C0BE0194
:10C960006F5B7F4FCE0101960E9426A7E114F10470
:10C9700009F4F8CEF70180858F70843009F0F2CE8B
:10C9800061857285CE0101960E94453CCE010196DB
:10C990000E944216882309F4E1CEA12CCC24C39432
:10C9A000F12CE12C62960FAD629763961FAD6397F1
:10C9B00064962FAD649765963FAD659766964FADCB
:10C9C000669767965FAD679768966FAD689769964B
:10C9D0007FAD6997A4CE883009F444C0803109F056
:10C9E0008FCC0E9458A62B013C01C4010E94AD16B9
:10C9F000A12CB12C650110E3E12E15E7F12E00E02A
:10CA000010E0A30192010E94312B882309F478CC15
:10CA100066E874E0D4018D919C910E9496988C01F7
:10CA2000009709F407C1FC0180858F70843009F0FC
:10CA300001C10E9458A62AE0AE014F5F5F4F0E94DD
:10CA400019CD0E94B498882309F4F4C08091D208CB
:10CA50008111F0C0BE016F5F7F4FD80119968D9193
:10CA60009C91E6C00E9458A62B013C01C4010E9483
:10CA7000AD16A12CB12C650118E9E12E1AE3F12EB7
:10CA800000E010E0A30192010E94312B882309F4F9
:10CA900037CCD4011496ED91FC91159781811396B2
:10CAA0001C91811153C01630F0F58CE0EEE1F2E0FC
:10CAB000DE01119601900D928A95E1F7E12FF0E0E9
:10CAC000EE0FFF1F21E030E02C0F3D1FE20FF31FA0
:10CAD00060E080810E94B4A46DEF76E183E01330C2
:10CAE000C9F070F465E077E181E0113099F061E020
:10CAF00077E182E0123071F069E077E180E00AC00E
:10CB000069EF76E184E0143029F065EF76E185E0A5
:10CB1000153091F70E94459DD4011496ED91FC913A
:10CB200081E08183EDCB65E477E08FE39AE00E94BA
:10CB30003587F40163818FE39AE00E94369D68E1B6
:10CB400077E08FE39AE00E943587DACB24E0129FEA
:10CB5000F0011124EC5FF94FC080D180E280F380B6
:10CB600064E177E08FE39AE00E943587D401139661
:10CB70006C918FE39AE00E94369D60E077E08FE34E
:10CB80009AE00E9435872AE030E0B701A6018FE3E2
:10CB90009AE00E94498666E874E0F4018081918100
:10CBA0000E9496988C01009709F44CC0DC011896FD
:10CBB0008C9118978F70843009F044C019966D914C
:10CBC0007C9140E450E0CE0101960E94CED86FE205
:10CBD00070E0CE0101960E9495D8892B51F4F8019E
:10CBE0002185328543E050E060E4CE0101960E9449
:10CBF000932BFF92EF92DF92CF9283E294E09F9388
:10CC00008F938E010F5B1F4F1F930F930E9425D9A7
:10CC10000E94B4980FB6F894DEBF0FBECDBF882334
:10CC200049F08091D208811105C0B801CE0101966A
:10CC30000E9426AA0E9458A6AB01BC01C4010E9412
:10CC400086165ECB61EF76E07CCF8FEF9FEFCB59FE
:10CC5000DF4F0FB6F894DEBF0FBECDBFDF91CF918F
:10CC60001F910F91FF90EF90DF90CF90BF90AF900A
:10CC70009F908F907F906F905F904F903F902F90FC
:10CC8000089580E090E0DC01F40124813581F90110
:10CC900042815381052E000C660B770B8417950794
:10CCA000A607B70709F42CCB3C01D4010D911C91C8
:10CCB00061E874E0C8010E9496985C0166E874E03F
:10CCC000C8010E9496986C01A114B10419F4892B33
:10CCD00009F448CD65EB74E0C8010E9496987C0188
:10CCE00060EB74E0C8010E9496988C016CEC76E0D1
:10CCF0008FE39AE00E943587F40163818FE39AE025
:10CD00000E94369D6AEC76E08FE39AE00E943587B8
:10CD1000B3018FE39AE00E943D9D8FE39AE00E9469
:10CD20005885C114D10409F4A6CCD60118968C916B
:10CD300018978F70843009F09ECC19966D917C9174
:10CD400040E450E0CE0101960E94CED80E94B498F3
:10CD5000882309F490CC8091D20881118CCC6FE2A9
:10CD600070E0CE0101960E9495D8892B51F4F6010E
:10CD70002185328543E050E060E4CE0101960E94B7
:10CD8000932B6114710409F4CFCCE114F10439F050
:10CD9000D70118968C918F70843009F465CC68E0C7
:10CDA00075E0CE0101960E9426A765CCEF92FF9216
:10CDB0000F931F93CF93DF93EC018B011D821C8295
:10CDC0001A821B82E880F980E114F10409F470C032
:10CDD00080914D0690914E06892B09F469C0672B0E
:10CDE00009F48701F80180858F708630A9F46FE01F
:10CDF00075E0C8010E949698009719F0FC018185A2
:10CE00008A836CEF75E0C8010E949698009709F438
:10CE100056C0FC0181858B8361E175E0C7010E94EA
:10CE20009698009709F041C06FEB76E08FE39AE0A7
:10CE30000E9435876B818FE39AE00E94369D6DEBEF
:10CE400076E08FE39AE00E9435876A818FE39AE06B
:10CE50000E94369D8FE39AE00E945885E880F98011
:10CE60000E946B8E8C01892BC1F082E0F8018087D3
:10CE7000118612861386148680819181009711F0A5
:10CE80000E94EB8B81E195E00E941A8CF80191835E
:10CE90008083B801C7010E94159D61E175E088811A
:10CEA00099810E949698009719F009969D838C832A
:10CEB000DF91CF911F910F91FF90EF900895F801AE
:10CEC000808191810E9409CCA6CF8F929F92AF92D0
:10CED000BF92CF92DF92EF92FF920F931F93CF9367
:10CEE000DF9300D000D0CDB7DEB720911B07309183
:10CEF0001C07232B09F484C020911A07211180C03C
:10CF00004C0180911A078F5F80931A07809119074F
:10CF10008F5F809319070E9458A69B01AC01609116
:10CF20003B0670913C0680913D0690913E06A12CF7
:10CF3000B12C65011BE0E12EF12C00E010E00E9415
:10CF4000312B882309F452C0E0911B07F0911C0794
:10CF50000681178101151105B9F1F80180858F70DF
:10CF6000863071F56DE774E0C8010E9496980097CD
:10CF7000D1F0FC0120852F702530A9F4E680F780E0
:10CF8000E114F104E9F0FA82E982B801CE010196D8
:10CF90000E94D666B401CE0101960E94C65EF701DA
:10CFA000E280F380EDCF1A83098370E060E0CE0168
:10CFB00001960E94D666B401CE0101960E94C65E1B
:10CFC000F80102811381C6CFF3E08F16910451F06E
:10CFD0000E9458A660933B0670933C0680933D06E2
:10CFE00090933E0610927E0A10927F0A8091190754
:10CFF00081508093190780911A07815080931A07F6
:10D0000026960FB6F894DEBF0FBECDBFDF91CF914D
:10D010001F910F91FF90EF90DF90CF90BF90AF9056
:10D020009F908F900895A89582E090E00C9465679A
:10D030008091D2088F5F8093D208A89583E090E01A
:10D040000E9465670E94A58B8091D20881508093D1
:10D05000D2080895CF92DF92EF92FF92CF93DF93A1
:10D06000EC018C85883068F40E941C940E9458A6BC
:10D070006B017C018C850E943894811109C088E085
:10D080008C87DF91CF91FF90EF90DF90CF90089544
:10D090000E94186861E070E080E090E00E9425A6A0
:10D0A0000E9458A6AB01BC014C195D096E097F09AD
:10D0B0008D859E85B0E0A0E0481759076A077B0779
:10D0C000C8F28C850E942A94DACFCF92DF92EF9239
:10D0D000FF921F93CF93DF93EC017B016A018C8554
:10D0E000883048F40E943894882319F08C850E9477
:10D0F0001C9488E08C87F70182819381A481B5819B
:10D100000097A105B10551F490E080E0DF91CF9147
:10D110001F91FF90EF90DF90CF9008958F3F9F4F2A
:10D12000AF4FBF4F89F370E060E081E20E947394DB
:10D13000182F8C87883040F780E591E00E948AA103
:10D14000A7014E5F5F4F24E030E06CE070E0812F7C
:10D150000E94C222B601812F0E94479464E070E0D1
:10D16000812F0E94548F0E9458A66B017C018C85F0
:10D170000E943894873121F18C3111F1882321F2FA
:10D180000E9458A6AB01BC014C195D096E097F09CC
:10D190008D859E85B0E0A0E084179507A607B707A8
:10D1A00048F00E94186861E070E080E090E00E9422
:10D1B00025A6DDCF8C850E942A9488E08C87A4CF99
:10D1C00081E090E0A3CF4F925F926F927F92AF92F7
:10D1D000BF92CF92DF92EF92FF920F931F93CF9364
:10D1E000DF93CDB7DEB76D970FB6F894DEBF0FBEF5
:10D1F000CDBF20914D0630914E06FF24F394232B92
:10D2000009F412C1811149C0FF24F3946BE47CE05E
:10D210008FE39AE00E9435878FE39AE00E94588559
:10D2200080913A068F5F80933A06E0911F07F09154
:10D230002007309709F48BC006811781011511056D
:10D2400009F48FC0D80118968C918F70853009F53C
:10D25000C8010E949A9D8823E1F0F80160817181E4
:10D26000CE0101960E94453CCE0101960E944216D5
:10D27000882359F08A859B85009739F0DC01ED9170
:10D28000FC910084F185E02D1995CE0101960E9454
:10D290007816F80102811381D1CF64E87CE08FE336
:10D2A0009AE00E9435878FE39AE00E9458850E9499
:10D2B00058A62B013C0180911907882371F10E9427
:10D2C00058A69B01AC01A12CB12C650110E1E12E07
:10D2D00017E2F12E00E010E0C301B2010E94312BF1
:10D2E00081111BC00E94A58B80912307811126C04C
:10D2F00080911D0790911E07059741F080911F07AF
:10D3000090912007892B11F00E9462580E94405C86
:10D3100082E090E00E946567CECF80911907882354
:10D3200009F472CF61E67CE088E999E00E943587D4
:10D3300088E999E00E945885F12C68CF80912107F7
:10D3400090912207892BA1F20E949052D1CF6BE3DA
:10D350007CE08FE39AE00E9435878FE39AE00E9499
:10D360005885109248061092470663E37CE08FE3ED
:10D370009AE00E9435878FE39AE00E94588564E620
:10D3800070E080E090E00E9425A61092A90610921D
:10D3900018076BE17CE08FE39AE00E9435870E94DA
:10D3A000FC2CAB01BC018FE39AE00E94339D80917D
:10D3B0004D0690914E06009711F00E9429A11092FF
:10D3C0004E0610924D0610921C0710921B071092E9
:10D3D000200710921F071092AB061092AA06109217
:10D3E0001607109215071092140710921307109247
:10D3F00022071092210766E17CE08FE39AE00E9409
:10D4000035870E94FC2CAB01BC018FE39AE00E949F
:10D41000339D8FE39AE00E94588510921707809100
:10D420003A06815080933A068F2D6D960FB6F89488
:10D43000DEBF0FBECDBFDF91CF911F910F91FF9047
:10D44000EF90DF90CF90BF90AF907F906F905F9004
:10D450004F9008958F929F92BF92CF92DF92EF925A
:10D46000FF920F931F93CF93DF93CDB7DEB7A597AE
:10D470000FB6F894DEBF0FBECDBF80914D069091E0
:10D480004E06892B09F47FC48091190781117BC452
:10D49000809119078F5F809319076AEC71E18EE81C
:10D4A00099E00E9435878EE899E00E9458850091A6
:10D4B0004D0610914E0664E175E0C8010E949698F1
:10D4C0009093200780931F076AE175E0C8010E94CE
:10D4D00096989093AB068093AA066FE375E0C80117
:10D4E0000E94969890931C0780931B0761E275E059
:10D4F000C8010E94969890931607809315070E9482
:10D50000C32F66E275E080914D0690914E060E9411
:10D5100096989093220780932107892BA1F0809100
:10D520002307811110C08091AC069091AD06892B24
:10D5300009F47CC081E0809323076AEB71E18EE8F7
:10D5400099E00E9435871092480610924706E091B4
:10D550001F07F0912007309709F4F6C2E680F780A4
:10D5600000911F07109120070115110509F4E5C26C
:10D57000E114F10409F4E1C2F70180858F70853070
:10D5800099F7C7010E949A9D823070F3B701CE01CE
:10D5900001960E94DF21CE0101960E944216882347
:10D5A000E1F18A859B85009709F440C2DC01ED9189
:10D5B000FC910284F385E02D1995892B49F08A8529
:10D5C0009B85DC01ED91FC910084F185E02D19959E
:10D5D0008A859B85DC01ED91FC910680F781E02D29
:10D5E0001995892BD1F0CE0101960E94441E882303
:10D5F00041F040E051E060E070E0CE0101960E9411
:10D60000433E8D819E81892B41F040E052E060E0F5
:10D6100070E0CE0101960E94433ED7011296ED9034
:10D62000FC90CE0101960E9478169ACF6CE771E1CA
:10D630008FE39AE00E9435878FE39AE00E94588535
:10D640008FE090E00E943CCA8C0188E1D8011196DD
:10D650008C93119712961C9212971C921E961C92F4
:10D660001E921D970E9455A11093AD060093AC0623
:10D67000012B69F46DE671E188E999E00E94358734
:10D6800088E999E00E945885109223075CCF0E9498
:10D6900055A18091AC069091AD060E94E61A8823B0
:10D6A00009F490C06EE471E18EE899E00E94598718
:10D6B0008091AC069091AD060E9444278091AC0603
:10D6C0009091AD0621E0FC0120830E9452276AE37D
:10D6D00071E1811102C065E271E18FE39AE00E947D
:10D6E00059878091210790912207892B69F28091B7
:10D6F000510690915206892B09F0EAC083E190E02F
:10D700000E943CCA8C018091AC069091AD0623E248
:10D710003AE7D80152963C932E93519716969C93D4
:10D720008E93159714961C9214971C9289E011966B
:10D730008C93119781E012968C93129713968C9389
:10D7400010935206009351060E9458A66B017C016B
:10D75000B0E1CB0EB7E2DB1EE11CF11CD80115963F
:10D76000ED91FC9116978FEF8387148613821482B4
:10D7700015821682178210861186128614961C92C4
:10D78000BB24B394BE01625E7F4FF8018581968110
:10D790000E942C2818160CF096C00E9458A66C15F2
:10D7A0007D058E059F0508F08EC0DE015E9698E02F
:10D7B00080E0915019F1ED91E827F0E0E753F64E43
:10D7C0008491F7CF0E9479298091AC069091AD06A3
:10D7D0000E94E61A882359F068E071E18EE899E02A
:10D7E0000E9435878EE899E00E9458857ACF6CEECA
:10D7F00070E188E999E00E94598746CF9DA198136E
:10D80000C1CFD8018C91811138C015968D919C9112
:10D810000E945227BE01625E7F4FF801858196818A
:10D820000E94252740E064EBD80115968D919C91CC
:10D830000E94FF26F80185809680C4010E948826F8
:10D84000C4010E94161367E88FEF98E00E94A113AD
:10D8500060E88FEF98E00E94A1130E9422A6C40105
:10D860000E948826982ED80115968D919C910E9431
:10D87000522795FC02C0F801B082AE014F5F5F4FA6
:10D88000BE01625E7F4FC8010E949327D8011196A6
:10D890009C908E8D803109F488C2BE01625E7F4FFC
:10D8A000C8010E940228891508F0B4C0F8018181DE
:10D8B000D80111968C93119714968C9114978F5FC1
:10D8C00014968C935FCFE0915106F091520612822C
:10D8D000E0912107F0912207E680F7809FE7D92E9B
:10D8E0008091210790912207892B09F423CEE1141E
:10D8F000F10409F41FCEBE01625E7F4FF701808103
:10D9000091810E942514882309F414CE65ED70E1FD
:10D910008FE39AE00E943587D7016D917C918FE368
:10D920009AE00E94CF868FE39AE00E94588500918A
:10D93000510610915206AE014F5F5F4FBE01625E0D
:10D940007F4FC8010E94E827882309F45EC08E8DAE
:10D95000803109F45AC0DD82F801858196810E94E8
:10D960005227BE01625E7F4FD80115968D919C9122
:10D970000E94252740E06EE4F801858196810E948F
:10D98000FF2640E06B81D80115968D919C910E94F5
:10D99000FF2640E06C81F801858196810E94FF2678
:10D9A0008E8D803141F040E06D81D80115968D91CA
:10D9B0009C910E94FF26F801858196810E94522742
:10D9C000BE01625E7F4FD80115968D919C910E9499
:10D9D0002527F801408168E4858196810E94FF2611
:10D9E00064E170E080E090E00E9425A6D8018C916F
:10D9F000882331F06AE070E080E090E00E9425A684
:10DA0000F801858196810E945227D7011296ED90E8
:10DA1000FC9066CF8E8D803111F48CE049CFBE0131
:10DA2000625E7F4FC8010E94022842CFCE0101965C
:10DA30000E94AA9D8C01912C812C97FF06C0119504
:10DA40000195110988248394912CCE0101960E949E
:10DA5000441EC82ED12C8985853091F0863009F07E
:10DA6000DCCDB02E61E0802F0E94B4A461E0892853
:10DA700009F441C0CA94CD2809F041C060E03FC01C
:10DA8000CD2829F462E0CE0101960E94151E40E0E7
:10DA900051E060E070E0CE0101960E94433E8D812E
:10DAA0009E81892B41F040E052E060E070E0CE01C1
:10DAB00001960E94433E61E0802F0E94B4A460E082
:10DAC000802F0E9486A462EB71E18FE39AE00E94AE
:10DAD0003587B8018FE39AE00E943D9D6DEA71E1C0
:10DAE0008FE39AE00E9435876BEA71E18FE39AE059
:10DAF0000E94358792CDCA94CD2809F0BFCFC62E9B
:10DB0000D12C8B2D0E9486A466EA71E18FE39AE006
:10DB10000E943587B8018FE39AE00E943D9D64EA38
:10DB200071E18FE39AE00E943587B6018FE39AE0B6
:10DB30000E943D9D62EA71E1D9CFF801868197810B
:10DB400090934806809347068FE39AE00E94588599
:10DB5000E0911B07F0911C07309709F48AC080916F
:10DB600019078F5F80931907068117810115110529
:10DB700009F47AC0D80118968C918F70863009F01C
:10DB800069C01F8F0E8F70E060E0CE014E960E943C
:10DB9000D6668AA19BA1892B09F45CC080914D06B1
:10DBA00090914E06892B09F455C0EE8CFF8CF7013D
:10DBB00080858F70863099F56DE774E0C7010E940B
:10DBC00096980097F1F0DC0118962C9118972F7019
:10DBD0002530B9F41696CD90DC90C114D104F9F03B
:10DBE000DA82C982B701CE0101960E94D666ED8124
:10DBF000FE811082118212821382F601C280D380CC
:10DC0000ECCFFA82E98270E060E0CE0101960E94DA
:10DC1000D66662E070E0CE0101960E94C65EEAA17F
:10DC2000FBA1108211821282138288A1843068F4D1
:10DC300062E0823008F060E089A10E94B4A4EAA109
:10DC4000FBA18181807F818305C0803441F060E049
:10DC5000823431F0D80112960D911C9187CF62E089
:10DC600089A10E94B4A4F6CF8091190781508093B6
:10DC7000190768EC70E18EE899E00E94358760EC46
:10DC800070E18EE899E00E94358781E020911F07BE
:10DC900030912007232B09F480E00E94661B67EB7C
:10DCA00070E18EE899E00E94358781E020911B07A2
:10DCB00030911C07232B09F480E00E94661B60EB67
:10DCC00070E18EE899E00E94358781E02091150788
:10DCD00030911607232B09F480E00E94661B67EA47
:10DCE00070E18EE899E00E94358781E0209121075C
:10DCF00030912207232B09F480E00E94661B6EE915
:10DD000070E18EE899E00E9435878091A9060E9413
:10DD1000661B8EE899E00E94588569E970E18EE8FB
:10DD200099E00E9435870E94FC2CAB01BC018EE873
:10DD300099E00E94339D8EE899E00E94588581E029
:10DD4000809318078BE599E00E94EC19882351F025
:10DD50008BE599E00E942A6884E090E090931E078A
:10DD600080931D0780911D0790911E07079731F43E
:10DD700084E090E090931E0780931D07809119071F
:10DD8000815080931907A5960FB6F894DEBF0FBE99
:10DD9000CDBFDF91CF911F910F91FF90EF90DF905A
:10DDA000CF90BF909F908F900895BCE0B91508F474
:10DDB0007DCD33CEAF92BF92DF92EF92FF920F9361
:10DDC0001F93CF93DF9300D000D0CDB7DEB78C0187
:10DDD0007B01D42EFB0184819581892BF9F0A080F1
:10DDE000B1806FE370E0C5010E9495D80097B1F053
:10DDF0009C012A193B0937FD11C050E040E0B701F2
:10DE0000CE0101960E941883BE016F5F7F4FC7014C
:10DE10000E94CE81CE0101960E94C88269E275E01F
:10DE2000C7010E944981882321F1F801128A118AD1
:10DE300080E090E19587848784E890E0948B838BE1
:10DE400081E0868780E090E2908B8787D58A81E0A9
:10DE500090E026960FB6F894DEBF0FBECDBFDF91DF
:10DE6000CF911F910F91FF90EF90DF90BF90AF90F7
:10DE7000089566E375E0C7010E944981882369F02F
:10DE8000F801128A118A148A138A84E890E095872F
:10DE90008487168680E090E3D7CF90E080E0D9CFEA
:10DEA000EF92FF920F931F93CF93DF9300D01F92B7
:10DEB000CDB7DEB78C017B01FB0184858830A8F0EB
:10DEC00087EE93E0F801918380831282138214829B
:10DED0001582C8010F900F900F900F90DF91CF9196
:10DEE0001F910F91FF90EF90089580E591E00E94BF
:10DEF0008AA124E030E0AE014F5F5F4F6CE070E03C
:10DF0000F70184850E94F123BE016F5F7F4FC80136
:10DF10000E947587DECFCF93DF93CDB7DEB72E9704
:10DF20000FB6F894DEBF0FBECDBF809119078F5F8B
:10DF3000809319076AE877E18EE899E00E943587B7
:10DF40008EE899E00E94588510928A0910928909FA
:10DF500080E090E1909385098093840984E890E0C3
:10DF600090938C0980938B0981E08093860980E0EF
:10DF700090E2909388098093870982E780938D09C6
:10DF800088E799E00E94AF228B37910509F0BEC067
:10DF90006CE777E18FE39AE00E9435878FE39AE0A0
:10DFA0000E9458851C821B8289E992E09A838983AA
:10DFB00088E799E09E838D838FEF9FEF98878F830B
:10DFC00080E00E94E368CE0101960E946CA19093CC
:10DFD0004E0680934D0688E799E00E94861B80914B
:10DFE0004D0690914E06892B01F560E777E188E9AF
:10DFF00099E00E94358788E999E00E9458856FE88A
:10E0000075E0CE0109960E940783CE0109960E9411
:10E01000DFAECE0109960E94C88280911907815017
:10E020008093190790E080E019C06DE577E18EE8F4
:10E0300099E00E9435878EE899E00E94588580918A
:10E0400019078150809319070E942A6A80916A09F2
:10E0500090916B09892B59F481E090E02E960FB6D0
:10E06000F894DEBF0FBECDBFDF91CF9108950E941F
:10E07000F899882389F382E70E94E39980916A09DD
:10E0800090916B09DC01ED91FC910088F189E02D04
:10E0900060E670E0199560916A0970916B0940E043
:10E0A000CE0109960E94E484BE01675F7F4F8CE633
:10E0B00099E00E94CE81CE0109960E94C88280918B
:10E0C0006A0990916B09DC01ED91FC910488F58956
:10E0D000E02D19956FE377E18FE39AE00E94358791
:10E0E0006CE679E0CE0109960E94FE82BE01675F70
:10E0F0007F4F8FE39AE00E9427878FE39AE00E9488
:10E100005885CE0109960E94C882A6CF88E799E07B
:10E110000E941F17892BA1F088E799E00E944917F8
:10E120006FE875E0CE0101960E940783CE0101964B
:10E130000E94DFAECE0101960E94C8820E944EAFBF
:10E1400088E799E00E94861B6CE477E18EE899E00D
:10E150000E9435878EE899E00E9458855ECFEF9245
:10E16000FF920F931F93CF93DF9300D000D0CDB7D2
:10E17000DEB780916A0990916B09892B09F46CC014
:10E1800087E70E94E39980916A0990916B09DC010D
:10E19000ED91FC910088F189E02D70E060E0199527
:10E1A00010E000E080916A0990916B09DC01ED912B
:10E1B000FC9111971C962D913C910217130740F486
:10E1C0000190F081E02D60E019950F5F1F4FEACFBD
:10E1D0000088F189E02D70E060E0199504EF12E00D
:10E1E00088EFE82E82E0F82E80916A0990916B0901
:10E1F000F80161918F01DC01ED91FC910190F081BA
:10E20000E02D1995E016F10679F780916A09909151
:10E210006B09DC01ED91FC910488F589E02D1995DD
:10E220006FE875E0CE0101960E940783CE0101964A
:10E230000E94DFAECE0101960E94C88287E090E086
:10E240000E94FF9C87E090E00E94099D6BE272E1D2
:10E250008EE899E00E94358710928A091092890908
:10E2600080E090E1909385098093840984E890E0B0
:10E2700090938C0980938B0981E08093860980E0DC
:10E2800090E2909388098093870982E780938D09B3
:10E2900088E799E00E94491788E799E00E94861B69
:10E2A00088EC90E026960FB6F894DEBF0FBECDBF87
:10E2B000DF91CF911F910F91FF90EF900895FF9202
:10E2C0000F931F93CF93DF9300D000D0CDB7DEB76D
:10E2D0008C01BC01CE0101960E94FE82BE016F5FDF
:10E2E0007F4F8FE39AE00E9427878FE39AE00E9496
:10E2F0005885CE0101960E94C88267EB73E1CE017A
:10E3000001960E94D082BE016F5F7F4FC8010E94BC
:10E310002E81F82ECE0101960E94C882FF2069F05E
:10E32000B801CE0101960E94FE82CE0101960E94A4
:10E33000DFAECE0101960E94C88226960FB6F894F1
:10E34000DEBF0FBECDBFDF91CF911F910F91FF9028
:10E3500008954F925F926F927F928F929F92AF92A9
:10E36000BF92CF92DF92EF92FF920F931F93CF93C2
:10E37000DF93CDB7DEB7C859D1090FB6F894DEBF29
:10E380000FBECDBF8E010F5B1F4FD8011D921C9297
:10E39000FE01ED5BFF4F8EE1DF011D928A95E9F7EB
:10E3A00080916A0990916B09892B09F4CEC10E9472
:10E3B000F899882309F4C9C182E70E94E399809102
:10E3C0006A0990916B09DC01ED91FC910088F1895B
:10E3D000E02D60E270E019954FE150E0B8018091C6
:10E3E0006A0990916B090E943D9A7C0180916A09AB
:10E3F00090916B09DC01ED91FC910488F589E02D89
:10E400001995E114F10409F4A0C1F801EE0DFF1D06
:10E410001082809177091F928F93809176091F92C5
:10E420008F93809175091F928F93809174091F9229
:10E430008F93809173091F928F93809172091F921D
:10E440008F9382E495E09F938F931F9280E48F9344
:10E45000FE0131966F01FF93EF930E94E8D86AE9BD
:10E4600074E18EE899E00E943587B8018EE899E062
:10E470000E94CF86B6018EE899E00E94CF868EE892
:10E4800099E00E9458857E01F1E6EF0EF11CD7015C
:10E4900013961C921E92129788EE93E0A0E0B0E0D3
:10E4A000F70184839583A683B78388E0848788EE09
:10E4B00093E09687858785E693E091838083108A31
:10E4C0001786128B018B148A138A80E590E0968B55
:10E4D000858B118E6EEB73E18FE39AE00E94358796
:10E4E0006CE679E0CE0185589F4F0E94FE82BE0106
:10E4F00065587F4F8FE39AE00E9427878FE39AE069
:10E500000E945885CE0185589F4F0E94C88261E7BE
:10E5100075E0CE0183579F4F0E94078361E775E046
:10E52000CE0185589F4F0E940783BE0165587F4FDB
:10E53000CE018B579F4F0E94FE826CE679E0CE01A0
:10E540008B579F4F0E946482BE0163577F4F0E948A
:10E550006482BC01CE018D569F4F0E94FE82CE0187
:10E560008B579F4F0E94C882CE0185589F4F0E94B3
:10E57000C882CE0183579F4F0E94C88283E795E0EF
:10E58000CB57DF4F99838883C558D040C757DF4F9B
:10E5900019821882C958D040C557DF4F1982188296
:10E5A000CB58D040CD56DF4F88819981C359D04098
:10E5B000C957DF4F99838883C758D04064E974E115
:10E5C0008FE39AE00E9435870E94FC2CAB01BC01CE
:10E5D0008FE39AE00E94339D8FE39AE00E94588572
:10E5E00064E670E080E090E00E9425A68FE591E768
:10E5F000D70150969C938E931F9760E37EE78EE938
:10E600009EE80E947FCD8C010FB6F894DEBF0FBE4E
:10E61000CDBF892B09F4F4C083E090E00E943CCA8E
:10E62000D8011D969C938E931C97FC01F182E08289
:10E630001282C7010E94EC19882319F0C7010E94B9
:10E640002A68D70153966D917C9154975596AD9059
:10E65000BC906115710509F48FC0CE0185589F4F9C
:10E660000E947587A501BE0165587F4FC7010E94B2
:10E670006568181619060CF0C0C0D7015196BC90F9
:10E6800051975296AC90DF92CF9289E194E19F939B
:10E690008F931F930F930E9406CEDF92CF9284E157
:10E6A00094E19F938F931F930F930E9406CED801FE
:10E6B0001C96ED91FC9181E08283DF92CF9281E103
:10E6C00094E19F938F931F930F930E9406CED801DE
:10E6D0001C96ED91FC911282AF92BF928BED93E16B
:10E6E0009F938F931F930F930E9406CE0FB6F894BB
:10E6F000DEBF0FBECDBFB12C82EDC82E83E1D82E78
:10E700008B2D94E08902F0011124A5E8B0E0AC0F54
:10E71000BD1FEA0FFB1F808191810097A9F1228123
:10E72000338121153105C9F33F932F939F938F9325
:10E73000DF92CF921F930F930E9406CEB3940FB631
:10E74000F894DEBF0FBECDBFDBCF40E250E06CECF3
:10E7500074E1C8010E94ACCC6EEA74E18EE899E0E5
:10E760000E943587B8018EE899E00E94CF868EE836
:10E7700099E00E9458854DCEF70161897289A50103
:10E78000C7010E940E1A75CF86E194E19F938F9383
:10E790001F930F930E9406CED70158961C921E928B
:10E7A0005797D8011C96ED91FC91C080D1800F90B5
:10E7B0000F900F900F9033E3A32EB12CD601ED9163
:10E7C000FC910084F185E02DC601199541975CF418
:10E7D000B1E0AB1AB10839F064E170E080E090E09C
:10E7E0000E9425A6EBCFD601ED91FC910084F18526
:10E7F000E02DC6011995419734F4C8010E94778E27
:10E8000010E000E05AC06FE875E0CE0183579F4FDB
:10E810000E940783912CA12CD601ED91FC910688D2
:10E82000F789E02DC60119958823E1F1BDE0AB120F
:10E8300001C0A92CD601ED91FC910688F789E02D45
:10E84000C60119958111D4C0D601ED91FC910084C7
:10E85000F185E02DC6011995892B09F4DBC0D6019D
:10E86000ED91FC910284F385E02DC6011995B82E37
:10E87000BAE08B1709F4D0C0EDE08E1709F4CCC0D4
:10E88000FFEF8F1709F4C6C0682FCE0183579F4F43
:10E890000E94BA819A2CAB2CBFCFBAE0BB12FACF40
:10E8A000AB12F8CFCC24C394D12CCE0183579F4F09
:10E8B0000E94C882CD2809F4A3CFD7015796ED90C6
:10E8C000FC9066E874E18FE39AE00E943587B70117
:10E8D0008FE39AE00E943D9D8FE39AE00E94588565
:10E8E00064E670E080E090E00E9425A60115110525
:10E8F00009F451C1B8ECEB16F10409F02AC16AE73A
:10E9000074E18EE899E00E94358764EF71E080E061
:10E9100090E00E9425A6EF961FAE1EAEEF97C1585D
:10E92000DF4F19821882CF57D0408FEF9FEFCF571C
:10E93000DF4F99838883C158D04083E892E0ED96F9
:10E940009FAF8EAFED97CD57DF4F19830883C35824
:10E95000D040F89481E00E94E368CE0185589F4F33
:10E960000E946CA190934E0680934D067894C80146
:10E970000E94778E80914D0690914E06892B09F06A
:10E98000D6C06FE875E0CE0183579F4F0E94078382
:10E99000CE0183579F4F0E94DFAECE0183579F4F1A
:10E9A0000E94C88263E674E188E999E00E94358795
:10E9B000F12CE12CCE018D569F4F0E94C882C701D9
:10E9C000C856DF4F0FB6F894DEBF0FBECDBFDF9144
:10E9D000CF911F910F91FF90EF90DF90CF90BF905C
:10E9E000AF909F908F907F906F905F904F90089521
:10E9F000D601ED91FC910084F185E02DC6011995B9
:10EA0000892B09F021CF64E670E080E090E00E945D
:10EA100025A610CFBB24BA9461E875E082EA99E09C
:10EA20000E94CF86BE0163577F4F82EA99E00E9421
:10EA3000278782EA99E00E94588569EC73E1CE014C
:10EA400085589F4F0E94D082BE0165587F4FCE01EE
:10EA500083579F4F0E942E81982ECE0185589F4F3D
:10EA60000E94C882992099F1CF56DF4F28813981C1
:10EA7000C159D04049E050E0BE0163577F4FCE01FD
:10EA800085589F4F0E941883ED968EAD9FADED97F0
:10EA9000412C512C3201009719F00E9427CC2B01F8
:10EAA0004201CE0185589F4F0E94C88241145104F3
:10EAB00029F0D70158965C924E925797B40182EA9A
:10EAC00099E00E943D9D82EA99E00E945885F701F5
:10EAD0008784908881149104D1F0CF56DF4F8881CC
:10EAE0009981C159D040892B91F0BE0163577F4F66
:10EAF000CE0185589F4F0E94FE82CE0185589F4FC0
:10EB0000F4011995CE0185589F4F0E94C8826FE885
:10EB100075E0CE0183579F4F0E949882FFEFBF128E
:10EB2000BCCEC8010E94778ED12CC12CBECE0E94D3
:10EB30002A6A80911807882329F00E94579C67FF52
:10EB40000E94501D6CE574E18EE899E00E943587C3
:10EB500031CFE0E3EE16E1E0FE0651F468E474E143
:10EB60008EE899E00E943587C8010E94778E22CFF7
:10EB700060E374E188E999E00E943587C8010E944A
:10EB8000778EB70188E999E00E943D9D88E999E078
:10EB90000E9458850FCF6DE174E18FE39AE00E94E7
:10EBA0003587EE24EA94FE2C05CF0F931F93CF9365
:10EBB000DF93EB0102970CF485C00A811B816BED9A
:10EBC00072E1C8010E9457CC892B51F481E00E9468
:10EBD000F59C88EC90E0DF91CF911F910F91089503
:10EBE00064EE72E1C8010E9457CC892B11F480E0D9
:10EBF000EECF62EB72E18EE899E00E9435870E94C9
:10EC0000579C63FB662760F981E0682770E08EE817
:10EC100099E00E943D9D8EE899E00E945885809180
:10EC20006A0990916B09892BE9F10A811B810E9485
:10EC3000F8998823B9F1F80101900020E9F731979C
:10EC4000E01BF10BB09770F582E70E94E399809189
:10EC50006A0990916B09DC01ED91FC910088F189C2
:10EC6000E02D60E270E01995B80180916A099091F9
:10EC70006B090E94CF8680916A0990916B09DC0133
:10EC8000ED91FC910190F081E02D60E0199580916B
:10EC90006A0990916B09DC01ED91FC910488F5897A
:10ECA000E02D19956A817B818EE899E00E94CF86DC
:10ECB0006BEA72E18EE899E00E9435878EE899E070
:10ECC0000E94588580911D0790911E0702977CF144
:10ECD0000E94A971883C910539F424E030E030931A
:10ECE0001E0720931D0777CF8F3F9807C9F460E96F
:10ECF00072E18FE39AE00E9435878FE39AE00E94E9
:10ED000058851092170783E090E090931E07809338
:10ED10001D078BE599E00E942A6889EC90E05BCFA3
:10ED2000209118072111D9CF2FE030E0D8CF63E828
:10ED300072E188E999E00E94358788E999E00E94AC
:10ED4000588584EF91E047CF5F926F927F928F92C8
:10ED50009F92AF92BF92CF92DF92EF92FF920F936A
:10ED60001F93CF93DF93CDB7DEB7CF56D1090FB640
:10ED7000F894DEBF0FBECDBF4C018B01F42E642F83
:10ED80008FE39AE00E94369D66E37DE08FE39AE090
:10ED90000E943587B801CE0101965C010E94FE8277
:10EDA000B5018FE39AE00E9427878FE39AE00E94E3
:10EDB0005885C5010E94C88292E0F9126BC264E3D3
:10EDC0007DE0C5010E94D082B501C8010E945E812C
:10EDD000F82EC5010E94C882FF2009F4D0C220E0AD
:10EDE0004DE251E0B40189E399E00E94068BE09086
:10EDF0001307F09014076DE27DE0CE0186599F4F16
:10EE00000E94D08266E27DE0CE018C599F4F0E9425
:10EE1000D082CE01885A9F4F0E9440256E961FAD2A
:10EE20006E976D960FAD6D976C96DFAC6C976B9689
:10EE3000CFAC6B976FE875E0CE0181960E94078397
:10EE4000BE016F5D7F4FC5010E94FE826C2DC50122
:10EE50000E94198264E875E00E944A826D2D0E942A
:10EE6000198264E875E00E944A82602F0E9419822C
:10EE700064E875E00E944A82612F0E941982BC01F9
:10EE8000CE01825A9F4F0E94FE82C5010E94C88215
:10EE9000CE0181960E94C88261E27DE0CE018E5A49
:10EEA0009F4F0E94D0826FE875E0CE01845B9F4F38
:10EEB0000E9407830AE619E0D80118966C9170E069
:10EEC00084E0759567958A95E1F7C5010E94B79929
:10EED0004D815E8169817A81CE01845B9F4F0E9462
:10EEE0008E81C5010E94C882F80160856F7070E054
:10EEF000C5010E94B7994D815E8169817A81CE01F9
:10EF0000845B9F4F0E948E81C5010E94C8820F5F63
:10EF10001F4FF9E000371F0779F66BE17DE0CE0166
:10EF20008A5B9F4F0E94D0826AEF7CE0CE0181967F
:10EF30000E94D082BE016F5D7F4FCE01CE960E94AF
:10EF4000FE82BE016A5B7F4FCE01CE960E94648234
:10EF5000BE01645B7F4F0E946482BE016E5A7F4F88
:10EF60000E946482BE01625A7F4F0E946482BE0189
:10EF70006C597F4F0E9464828C014AE0B50180E5A4
:10EF800090E00E94F1CCF50101900020E9F7319763
:10EF9000AF014A195B09B501C8010E948E81811138
:10EFA00003C0C8010E940782BE0166597F4FC80195
:10EFB0000E946482B7010E944A82BC01C4010E947F
:10EFC0002787C4010E945885CE01CE960E94C88230
:10EFD000CE0181960E94C882CE018A5B9F4F0E941B
:10EFE000C882CE01845B9F4F0E94C882CE018E5A98
:10EFF0009F4F0E94C882CE01825A9F4F0E94C882B2
:10F00000CE018C599F4F0E94C882CE0186599F4FD6
:10F010000E94C882C4010E94588564E670E080E0C6
:10F0200090E00E9425A6D401ED91FC910488F58919
:10F03000E02DC401199501E010E088C028966EAD5E
:10F040007FAD2897CE0181960E945F9E892B09F49F
:10F0500050C122961CAE1DAE1EAE1FAE2297269644
:10F060001CAE1DAE1EAE1FAE26978FAD8F708FAF3C
:10F0700040E053E0BE016F5D7F4FCE01CE960E940F
:10F080001F3500E020E033E040E250E0B501CE0162
:10F09000CE960E946A31BC01C6010E94A28208EC91
:10F0A00010E129C1EE2009F4F3C046E050E070E021
:10F0B00060E0C8010E94CB80D8016D917C91CE01A7
:10F0C00081960E94453CCE0181960E94421600E93D
:10F0D00011E08823B9F189A5873061F4CE018196CA
:10F0E0000E94F55961E0892B09F462E0CE01819616
:10F0F0000E94151E22961CAE1DAE1EAE1FAE22979C
:10F1000026961CAE1DAE1EAE1FAE26978FAD8F701D
:10F110008FAF40E053E0BE016F5D7F4FCE01CE96D2
:10F120000E941F3500E020E033E040E250E0B501EE
:10F13000CE01CE960E946A31BC01C6010E94A28215
:10F1400008EC10E1CE0181960E947816C801C159E1
:10F15000DF4F0FB6F894DEBF0FBECDBFDF91CF916A
:10F160001F910F91FF90EF90DF90CF90BF90AF90E5
:10F170009F908F907F906F905F900895F8016081CD
:10F1800071810E9496987C01892B09F040C104E9A5
:10F1900011E0DCCFEE2009F47BC049E050E070E0E4
:10F1A00060E0C8010E94CB804AE0B401C5010E9422
:10F1B000E48441E050E067E574E0C8010E948E817C
:10F1C0004D815E8169817A81C8010E948E8166EDE0
:10F1D0007CE08FE39AE00E943587B801CE018196EA
:10F1E0000E94FE82BE016F5D7F4F8FE39AE00E9416
:10F1F00027878FE39AE00E945885CE0181960E946E
:10F20000C8826EEC7CE0CE0181960E94D082F8012B
:10F21000848195812DA13EA182179307E1F4892B6A
:10F22000A1F1E080F18069A07AA0D7018D917D01E4
:10F23000882359F1082E000C990B0E9425D86C01E7
:10F24000F30181913F01082E000C990B0E9425D8F3
:10F25000C816D90651F3CE0181960E94C882552066
:10F2600041F021E048EC50E0B40189E399E00E94CC
:10F27000068BD8018D919C910E94348B009711F4DC
:10F2800084E991E08C01C5013DC055245394E3CF3E
:10F2900001E97ECFB1E0FB1270C063EF7CE0C501F5
:10F2A0000E94D082B501C8010E942E81582EC5014E
:10F2B0000E94C882552049F1EE2051F346E050E00B
:10F2C00070E060E0C8010E94CB804AE0B401CE014A
:10F2D0008A5B9F4F0E94E484F80160817181CE01B6
:10F2E00081960E94453CCE0181960E944216811172
:10F2F000A5CE00E911E0CE0181960E947816CE01DC
:10F300008A5B9F4F0E94C88221CF6CED7CE0C501D3
:10F310000E94D082B501C8010E942E81F82EC5013D
:10F320000E94C882F11036CF61EC7CE0C5010E94DA
:10F33000D082B501C8010E942E81182FC5010E94FC
:10F34000C88200E0112309F401CF80E00E94F59CFF
:10F3500069E97CE08EE899E00E9435878EE899E0C3
:10F360000E9458856FE875E0C5010E940783C501BA
:10F370000E94DFAEC5010E94C88200E05DCE6CEE47
:10F380007CE0C5010E94D082B501C8010E942E8197
:10F39000F82EC5010E94C882F11084CE66EE7CE092
:10F3A000C5010E94D082B501C8010E942E81F82EAD
:10F3B000C5010E94C882FF2001F3EE2009F468CF46
:10F3C00045E050E070E060E0C8010E94CB8064E856
:10F3D00075E0C8010E944981882339F0E0901F0739
:10F3E000F0902007E114F10491F46FE875E0C80192
:10F3F0000E944981811107C080911F0790912007C9
:10F40000009709F0BBCEE0904D06F0904E0620E04C
:10F4100048EC50E2B40189E399E00E94068BC401F4
:10F420000E9458851C821B8289E992E09A83898315
:10F430009E828D828FEF9FEF98878F83B701C501E2
:10F440000E945D8CEACD0895FC012481358162170C
:10F45000730748F480819181009729F0860F971FE8
:10F46000FC018081089580E0089508950895AF9289
:10F47000BF92CF92DF92EF92FF920F931F93CF93A1
:10F48000DF936C017B018B01040F151FEB015E0103
:10F49000AE18BF08C017D10759F06991D601ED9198
:10F4A000FC910190F081E02DC6011995892B79F727
:10F4B000C501DF91CF911F910F91FF90EF90DF90E9
:10F4C000CF90BF90AF900895FC01538D448D252FB0
:10F4D00030E0842F90E0821B930B541710F0CF96EE
:10F4E000089501970895FC01918D828D981761F020
:10F4F000A28DAE0FBF2FB11D5D968C91928D9F5F37
:10F500009F73928F90E008958FEF9FEF0895FC0115
:10F51000918D828D981731F0828DE80FF11D858DC8
:10F5200090E008958FEF9FEF0895FC01918D228D5B
:10F53000892F90E0805C9F4F821B91098F739927E0
:10F54000089582EA99E00E94957A21E0892B09F4D6
:10F5500020E0822F0895FC01A48DA80FB92FB11DC2
:10F56000A35ABF4F2C91848D90E001968F739927F9
:10F57000848FA689B7892C93A089B1898C918370D7
:10F5800080648C93938D848D981306C00288F389D0
:10F59000E02D80818F7D80830895EF92FF920F93FD
:10F5A0001F93CF93DF93EC0181E0888F9B8D8C8D2F
:10F5B00098131AC0E889F989808185FF15C09FB723
:10F5C000F894EE89FF896083E889F98980818370E6
:10F5D000806480839FBF81E090E0DF91CF911F9195
:10F5E0000F91FF90EF900895F62E0B8D10E00F5FB6
:10F5F0001F4F0F731127E02E8C8D8E110CC00FB68C
:10F6000007FCFACFE889F989808185FFF5CFCE0123
:10F610000E94AB7AF1CFEB8DEC0FFD2FF11DE35A79
:10F62000FF4FF0829FB7F8940B8FEA89FB898081A6
:10F630008062CFCFCF93DF93EC01888D8823B9F020
:10F64000AA89BB89E889F9898C9185FD03C08081ED
:10F6500086FD0DC00FB607FCF7CF8C9185FFF2CF6A
:10F66000808185FFEDCFCE010E94AB7AE9CFDF919B
:10F67000CF91089580E090E0892B29F00E94A17A33
:10F6800081110E94000080E090E0892B49F080E029
:10F6900090E0892B29F00E94000081110E94000057
:10F6A00080E090E0892B49F080E090E0892B29F000
:10F6B0000E94000081110E94000080E090E0892BF0
:10F6C00049F080E090E0892B29F00E940000811130
:10F6D0000C94000008950F931F93FC0162857385BD
:10F6E000848595850281138124813581601B710B8E
:10F6F000820B930B0685178520893189601B710B5E
:10F70000820B930B1F910F910895DC01ED91FC91F9
:10F710000190F081E02D19948FEF9FEF0895FC0187
:10F7200062897389848995890895EF920F931F9355
:10F73000CF93DF93FC01248D222341F0213051F13E
:10F74000DF91CF911F910F91EF9008952289338916
:10F750004489558986899789A08DB18D821B930B29
:10F76000A40BB50B892F9A2FAB2FBB278C010F5FF2
:10F770001F4F6281738184819581CFB7F894DCB784
:10F78000E1E0ECBFEE24E394E2E0FEEF1995DCBF8C
:10F79000CFBFD6CFF0E0E0E0DF91CF911F910F9186
:10F7A000EF901994FC01138E128E41110CC08289C6
:10F7B0009389A489B589868B978BA08FB18F148E7E
:10F7C00081E090E0089590E080E00895CF92DF928C
:10F7D000EF92FF92CF93DF93DC01CB01642FCFB781
:10F7E000F8946D01EE24FF24CBBEDCB741E04CBFA2
:10F7F000A901E1E0FEEF1995DCBFCFBFDF91CF910A
:10F80000FF90EF90DF90CF900895CF93DF93FC01AE
:10F81000248D211110C0EC01828D938D892B49F02C
:10F8200066897789808D918D30E020E045E00E94E7
:10F83000E67B1B8E1A8EDF91CF9108951F93CF9395
:10F84000DF93FC01248D211145C0162FEC01828D20
:10F85000938D892B49F466897789808D918D30E06D
:10F8600020E043E00E94E67B4A8D5B8DCA018170F7
:10F870009927FE01E80FF91F158F892B69F02D8D4F
:10F880003E8D6E897F89888D998D640F751F811DCE
:10F89000911D41E00E94E67B8A8D9B8D01969B8F96
:10F8A0008A8F81159140B1F46E897F89888D998DF9
:10F8B00030E020E045E00E94E67B1B8E1A8E8E89A8
:10F8C0009F89A88DB98D9F5FAF4FBF4F8E8B9F8B48
:10F8D000A88FB98F81E090E0DF91CF911F910895BB
:10F8E000DC01ED91FC910280F381E02D40E0199460
:10F8F000FB01448155812281338121503109421716
:10F90000530750F4A081B181A40FB51F8C9384815B
:10F91000958101969583848380E00895CF93DF934A
:10F92000EC01E881F9810284F385E02DCE0119957F
:10F930000196B9F7DF91CF910895CF92DF92EF92C0
:10F94000FF920F931F93CF93DF937C016A018B018A
:10F95000D0E0C0E0CC15DD0581F0D701ED91FC9140
:10F960000284F385E02DC70119958F3F980729F090
:10F97000F80181938F012196EDCFCE01DF91CF91D8
:10F980001F910F91FF90EF90DF90CF900895CF934C
:10F99000C62FDC01ED91FC910088F189E02D1995CD
:10F9A000DC01ED91FC910190F081E02D6C2FCF9165
:10F9B0001994062E000C770BFC017783668308955B
:10F9C000CF93DF93EC018E819F81019611F5E88141
:10F9D000F9810088F189E02DCE011995DC01ED91C6
:10F9E000FC910084F185E02D1995892BB1F0E88117
:10F9F000F9810284F385E02DCE01199581329105BC
:10FA000034F3E881F9810684F785E02D682FCE0173
:10FA1000199581E0DF91CF91089580E0FBCFFC0143
:10FA200020812EBD9B012150310941F051810DB43F
:10FA300007FEFDCF4EB55EBD4193F5CF6150710914
:10FA4000860F971F0DB407FEFDCF2EB5FC01208356
:10FA50000895E0912507F091260780819091240771
:10FA6000892B80830895E0912507F09126079081E6
:10FA70008091240780958923808308958EBD00009E
:10FA80000DB407FEFDCF8EB5089590E020916A0871
:10FA9000233339F40C96982F990F990F990F80E022
:10FAA00008954896F8CFEF92FF920F931F93CF934C
:10FAB000DF93EC018B017A010E9458A6688B798B49
:10FAC0008A8B9B8B8C819D81DC01ED91FC91028066
:10FAD000F381E02DA701B801DF91CF911F910F9124
:10FAE000FF90EF9019941F93CF93DF93EC01162FA3
:10FAF0000E9458A6688B798B8A8B9B8B8C819D8109
:10FB0000DC01ED91FC910190F081E02D612FDF91FE
:10FB1000CF911F911994CF92DF92EF92FF92CF93E2
:10FB2000DF93EC018E819F818F3F980759F02FEF73
:10FB30003FEF3F832E83DF91CF91FF90EF90DF90D7
:10FB4000CF9008950E9458A66B017C01A4EFCA0EC5
:10FB5000A1E0DA1EE11CF11CE881F9810088F1893D
:10FB6000E02DCE011995DC01ED91FC910084F18529
:10FB7000E02D1995892B39F40E9458A66C157D0546
:10FB80008E059F0548F3E881F9810088F189E02D11
:10FB9000CE011995DC01ED91FC910284F385E02DF5
:10FBA000DF91CF91FF90EF90DF90CF901994FB0100
:10FBB00001900020E9F73197AF01461B570BDC019C
:10FBC000ED91FC910280F381E02D19940E9420D8E0
:10FBD0000F931F93CF93DF93D0E0C0E0009791F095
:10FBE0008C01C9E6D7E0688179816115710529F03A
:10FBF000C8010E94A0D8892B29F00B80DC81C02D80
:10FC0000209789F7CE01DF91CF911F910F91089531
:10FC10000F931F93CF93DF93EC0188819981009715
:10FC200059F02A813B812617370730F081E0DF91B8
:10FC3000CF911F910F9108958B016F5F7F4F0E94AD
:10FC40003FD7009759F0998388831B830A832C81BF
:10FC50003D81232B59F7FC011082E8CF80E0E7CFEC
:10FC6000EF92FF920F931F93CF93DF93009751F47E
:10FC7000CFEFDFEFCE01DF91CF911F910F91FF907A
:10FC8000EF900895DC011C96ED90FC90F701008147
:10FC90001181D801ED91FC910688F789E02DC8010A
:10FCA0001995882329F3D801ED91FC910084F18501
:10FCB000E02DC8011995D801ED91FC91892B61F3D4
:10FCC0000284F385E02DC8011995EC01019681F2BB
:10FCD000F801818D882329F06C2F82EA99E00E9437
:10FCE000369DD70112968C91882321F2C532D10519
:10FCF00009F6D801ED91FC910084F185E02DC80151
:10FD0000199502975CF0D801ED91FC910688F7896E
:10FD1000E02DC80119958111ECCFAACFD1E0C0E048
:10FD2000D801ED91FC910284F385E02DC80119956D
:10FD30008F3F980709F49CCF9C01215431092A3147
:10FD4000310570F48D2F8295807F829FC00D112424
:10FD5000D11104C00C2E000CDD0B8CCFD0E0E0CF15
:10FD60009C01215631092A31310560F3C0978A3050
:10FD7000910570F79D2F9295907F989FC00D11244B
:10FD8000E7CFCF92DF92EF92FF920F931F93CF9323
:10FD9000DF936C018B0186E090E00E943CCAEC018D
:10FDA0009093AB078093AA07F60101900020E9F732
:10FDB000CF018C199D090E943CCA7C01B6010E94AA
:10FDC000A9D8F60101900020E9F73197EC19FD0957
:10FDD000EE0DFF1D1082F982E8821B830A83809159
:10FDE000AC079091AD079D838C83D093AD07C093F2
:10FDF000AC07DF91CF911F910F91FF90EF90DF90B3
:10FE0000CF900895FC01868197818F3F980729F054
:10FE10002FEF3FEF378326830895808591850C94DB
:10FE2000CACD7F928F929F92AF92BF92CF92DF9274
:10FE3000EF92FF920F931F93CF93DF93CDB7DEB76F
:10FE4000A6970FB6F894DEBF0FBECDBF8C01762EFD
:10FE5000942E852E20E2A22ECE0101967C01DC019B
:10FE6000EA2D1D92EA95E9F76801F3E4CF0ED11C63
:10FE700087EE93E09AA389A38FEF8BA38CA38DA326
:10FE80008EA343E450E0BE016F5D7F4FC6010E9428
:10FE90008324019609F4BFC081E089838A8386E0C8
:10FEA000B82EBB821C82D80114966D917D918D91E4
:10FEB0009C9117970E9447D46D837E838F83988788
:10FEC00089869A8680E890E09C878B874CE150E099
:10FED000B701C6010E941824FE0137968AE1DF01AE
:10FEE0001D928A95E9F74801B8E08B0E911CF40148
:10FEF000D70101900D92BA94E1F740E150E0B701CB
:10FF0000C6010E941824F7011192AA94E9F796E01D
:10FF1000A92EB12C40E250E0B701C6010E9418247E
:10FF2000F1E0AF1AB108B1F783E6898392E89A83CA
:10FF300093E59B838C8385E38D8381E08E837F8231
:10FF40009DE3988797E099878A8786E0F401DE0130
:10FF50001B9601900D928A95E1F78CE0898B8A8B34
:10FF600066E875E0CE0143960E94A9D8D8011B9699
:10FF70006C91CE0149960E94CBA1F8016485CE0117
:10FF80004B960E94CBA1D8011D966C91CE014D9647
:10FF90000E94CBA14EE150E0B701C6010E94182497
:10FFA000B3E07B121EC082E3898384E08A83F80178
:10FFB00096859B8397859C8390899D8391899E8359
:10FFC00096E39F838887828D8987838D8A87848D36
:10FFD0008B87858D8C874CE050E0B701C6010E946D
:10FFE000182487E3898386E08A8391E09B8393E0EA
:10FFF0009C838D838FE08E838AE38F838BE3888756
:020000021000EC
:100000008FEF898749E050E0B701C6010E941824AC
:10001000C6010E945224A6960FB6F894DEBF0FBE0A
:10002000CDBFDF91CF911F910F91FF90EF90DF90A7
:10003000CF90BF90AF909F908F907F90089590E069
:1000400080E00C94F022CF93DF93C4E1D0E00E94D3
:100050001F80882361F061E070E080E090E00E9402
:1000600025A62197A1F780E0DF91CF91089581E047
:10007000FBCFFF920F931F93CF93DF931F921F929B
:10008000CDB7DEB7F82E22E030E0AE014F5F5F4F14
:1000900066E270E00E94F12309811A81102701278E
:1000A000102722E030E0AE014F5F5F4F66E270E064
:1000B0008F2D0E94F12389819A819827892798277B
:1000C0000817190749F4C8010F900F90DF91CF91DD
:1000D0001F910F91FF9008958C01E3CFAF92BF92D3
:1000E000CF92DF92EF92FF920F931F93CF93DF9304
:1000F000DC01CD90DC901197C114D10439F0149635
:10010000CD91DC918C017601209761F4DF91CF9144
:100110001F910F91FF90EF90DF90CF90BF90AF9025
:10012000089575015701BFEFAB1ABB0AF701808133
:10013000082E000C990B0E944ECC892B91F7219729
:10014000CC0DDD1D8881082E000C990B0E944ECC31
:10015000892B29F0CE15DF0510F02197F3CFAE01E2
:100160004F5F5F4F4E195F09D80115965C934E9310
:100170001497CE14DF0420F4B701C6010E945CD8A6
:10018000D801ED91FC91119714968D919C91E80FF7
:10019000F91F1082BBCFCF93DF93DC011496ED9152
:1001A000FC916E177F0728F54115510511F19F014C
:1001B000261B370B4217530708F49A01DB01EC01A9
:1001C00088819981E21BF30BFD83EC83AF01461B11
:1001D000570B260F371FBC01620F731F8A0F9B1F1F
:1001E0000E94CED8E881F9818C819D81E80FF91FAA
:1001F0001082DF91CF910895DF92EF92FF920F93DB
:100200001F93CF93DF93FC01E480F580E114F104A8
:1002100051F48FEF9FEFDF91CF911F910F91FF90DE
:10022000EF90DF900895EC010190F081E02DEE0D4C
:10023000FF1DD080108208811981062E000C770BDB
:10024000C8010E94DDD80E0D1F1DF801D082009755
:1002500001F328813981821B930BDDCFFB0144819F
:100260005581FC01248135812417350778F0808180
:100270009181009759F0FB016081718161157105D1
:1002800029F00E94C0D821E0892B09F020E0822FBC
:100290000895FC0124813581232B39F421E0FB01F1
:1002A0008081882349F020E007C0808191810E94ED
:1002B000A0D821E0892BB9F7822F0895FC01248171
:1002C0003581FB014481558124173507E1F4FC0198
:1002D00080819181FB01608171810097D1F061156E
:1002E0007105A1F4232BC1F0FC01808190E008C0CE
:1002F000232B91F0FB01808190E0919581959109EC
:1003000021E0892B09F020E0822F08950E94A0D8D7
:10031000F7CF6115710561F721E0F6CFEF92FF92FB
:100320000F931F93CF93DF936115710541F480E024
:10033000DF91CF911F910F91FF90EF90089541159C
:100340005105B1F07B01EC010C811D81040F151FDB
:10035000B8010E94087E882351F3288139818C815D
:100360009D81B701820F931F0E94A9D81D830C8322
:1003700081E0DECFCF93DF931F921F92CDB7DEB720
:1003800069831A8241E050E0BE016F5F7F4F0E9497
:100390008E810F900F90DF91CF9108950F931F934F
:1003A000CF93DF938C01EB01FC0180819181009759
:1003B000E1F06881798161157105A9F0428153816D
:1003C0002C813D814217530770F00E94A9D88C817F
:1003D0009D81F801958384831D821C82DF91CF91DA
:1003E0001F910F9108950E94D8CA88819981F801C0
:1003F000918380838A819B81938382838C819D8179
:1004000095838483198218821B821A82E5CFCF9349
:10041000DF93EC0188819981009711F00E94D8CA7E
:10042000198218821D821C821B821A82DF91CF9151
:100430000895EF92FF920F931F93CF93DF9300D015
:100440001F92CDB7DEB77C01862F4AE08E010F5F89
:100450001F4FB80190E00E94F1CCF80101900020FC
:10046000E9F73197AF01401B510BB801C7010E945A
:100470008E81811103C0C7010E940782C7010F90BE
:100480000F900F900F90DF91CF911F910F91FF90E0
:10049000EF900895CF93DF93EC016115710539F466
:1004A000CE010E940782CE01DF91CF910895FB011A
:1004B00001900020E9F73197AF01461B570B0E94CE
:1004C0008E81882369F3EFCFCF93DF93EC01FB019B
:1004D00044815581608171810E948E81811103C0A8
:1004E000CE010E940782CE01DF91CF910895EF9255
:1004F000FF920F931F93CF93DF93EC017B018A014F
:10050000BA010E94087E81110BC0CE010E940782B1
:10051000CE01DF91CF911F910F91FF90EF90089541
:100520001D830C83B701888199810E94A9D8F0CFDF
:10053000FB0101900020E9F73197AF01461B570BF3
:100540000C947782CF93DF93EC016115710531F044
:100550000E949882CE01DF91CF9108950E94078278
:10056000F9CFCF93DF93EC01FB018617970749F092
:10057000608171816115710541F0448155810E944E
:100580007782CE01DF91CF9108950E940782F9CF43
:10059000FC0180819181009711F00C94D8CA0895D4
:1005A000EF92FF920F931F93CF93DF93EC018B0198
:1005B000198218821B821A821D821C82CB010E9422
:1005C00085CC7C01BC01CE010E94087E811109C04E
:1005D000CE01DF91CF911F910F91FF90EF900C947E
:1005E0000782FD82EC82B80188819981DF91CF91E9
:1005F0001F910F91FF90EF900C947ECCFC01118223
:10060000108213821282158214820C94B182FC0132
:10061000118210821382128215821482FB010190D2
:100620000020E9F73197AF01461B570B0C947782F6
:10063000AF92BF92CF92DF92EF92FF920F931F93F0
:10064000CF93DF935C016B017A0189012417350791
:1006500020F48F2D7901042F182F6FE875E0C50164
:100660000E940783D6011496CD91DC91EC16FD060D
:10067000C8F40C171D0708F4E801D601ED91FC91B0
:100680001197EC0FFD1F108110826D917C916E0D02
:100690007F1DC5010E94A282F60180819181C80F51
:1006A000D91F1883C501DF91CF911F910F91FF9042
:1006B000EF90DF90CF90BF90AF9008951F920F9270
:1006C0000FB60F9211240BB60F922F933F934F93B7
:1006D0005F936F937F938F939F93AF93BF93EF93AA
:1006E000FF93E0911202F09113021995FF91EF919F
:1006F000BF91AF919F918F917F916F915F914F913A
:100700003F912F910F900BBE0F900FBE0F901F9037
:1007100018951F920F920FB60F9211240BB60F92DD
:100720002F933F934F935F936F937F938F939F93F9
:10073000AF93BF93EF93FF93E0911002F0911102FA
:100740001995FF91EF91BF91AF919F918F917F91FB
:100750006F915F914F913F912F910F900BBE0F9032
:100760000FBE0F901F9018951F920F920FB60F9209
:1007700011240BB60F922F933F934F935F936F9378
:100780007F938F939F93AF93BF93EF93FF93E091EA
:100790000602F09107021995FF91EF91BF91AF9179
:1007A0009F918F917F916F915F914F913F912F9189
:1007B0000F900BBE0F900FBE0F901F9018951F92B9
:1007C0000F920FB60F9211240BB60F922F933F93F7
:1007D0004F935F936F937F938F939F93AF93BF9349
:1007E000EF93FF93E0910402F09105021995FF91B8
:1007F000EF91BF91AF919F918F917F916F915F9199
:100800004F913F912F910F900BBE0F900FBE0F9005
:100810001F9018951F920F920FB60F9211240BB6CE
:100820000F922F933F934F935F936F937F938F9389
:100830009F93AF93BF93EF93FF93E0910E02F091DC
:100840000F021995FF91EF91BF91AF919F918F91F9
:100850007F916F915F914F913F912F910F900BBEC0
:100860000F900FBE0F901F9018951F920F920FB60A
:100870000F9211240BB60F922F933F934F935F93D8
:100880006F937F938F939F93AF93BF93EF93FF9358
:10089000E0910C02F0910D021995FF91EF91BF913B
:1008A000AF919F918F917F916F915F914F913F9108
:1008B0002F910F900BBE0F900FBE0F901F901895A9
:1008C0001F920F920FB60F9211240BB60F922F9317
:1008D0003F934F935F936F937F938F939F93AF93C8
:1008E000BF93EF93FF93E0910A02F0910B021995E9
:1008F000FF91EF91BF91AF919F918F917F916F91F8
:100900005F914F913F912F910F900BBE0F900FBEB3
:100910000F901F9018951F920F920FB60F921124EF
:100920000BB60F922F933F934F935F936F937F93E9
:100930008F939F93AF93BF93EF93FF93E091080240
:10094000F09109021995FF91EF91BF91AF919F919D
:100950008F917F916F915F914F913F912F910F9068
:100960000BBE0F900FBE0F901F9018950F931F9303
:10097000CF93DF93EC010E9458A6688779878A8716
:100980009B87E881F9810284F385E02DCE011995DA
:1009900097FF15C00E9458A6088519852A853B85B2
:1009A000601B710B820B930B0C811D812E813F818B
:1009B000601771078207930720F38FEF9FEFDF9196
:1009C000CF911F910F910895EF92FF920F931F9374
:1009D000CF93DF93EC017B01042F6FE875E00E9459
:1009E0000783C7010E94B684002E000C110B97FDEF
:1009F0000BC00817190741F0682FCE010E94BA8179
:100A0000C7010E94B684F3CFCE01DF91CF911F9131
:100A10000F91FF90EF9008958F929F92AF92BF92A7
:100A2000EF92FF920F931F93CF93DF93CDB7DEB773
:100A3000A1970FB6F894DEBF0FBECDBF7C01FA01BF
:100A4000CB0119A2223008F42AE08E010F5D1F4F5E
:100A5000822E912CB12CA12CBF01A50194010E94E2
:100A6000B4D3F901CA016A300CF5605DD8016E9308
:100A70008D01232B242B252B79F790E080E0109714
:100A800021F0BD01C7010E94D77DA1960FB6F89451
:100A9000DEBF0FBECDBFDF91CF911F910F91FF90B1
:100AA000EF90BF90AF909F908F900895695CDECFDC
:100AB0006DE875E00C94D77DDC01ED91FC9101901F
:100AC000F081E02D19942F923F924F925F926F9296
:100AD0007F928F929F92AF92BF92CF92DF92EF92CE
:100AE000FF921F93CF93DF93EC016A017B01722E7B
:100AF000AB019601CB01B6010E94D2D560E975E049
:100B0000811126C046015701E894B7F82FEF3FEF57
:100B10004FE75FE7C501B4010E94D2D581110CC037
:100B20002FEF3FEF4FE75FE7C501B4010E946AD2A4
:100B300064E975E0181664F02FEF3FEF4FE75FE4CC
:100B4000C701B6010E9472D51816B4F468E975E0C1
:100B5000CE01DF91CF911F91FF90EF90DF90CF906A
:100B6000BF90AF909F908F907F906F905F904F90CD
:100B70003F902F900C94D77D2FEF3FEF4FE75FEC26
:100B8000C701B6010E946AD287FDE0CF20E030E0C5
:100B9000A901C701B6010E946AD2312C212C87FF1E
:100BA00009C06DE2CE010E945C851C01F7FAF09449
:100BB000F7F8F09410E060E070E080E09FE37116D9
:100BC00041F020E030E040E251E40E94CAD41F5FCF
:100BD000F6CFA70196010E945ED42B013C010E9432
:100BE00043D54B015C012AE0BC01A401CE010E9467
:100BF0000C857C01E20CF31C1123C1F1C501B40189
:100C00000E946FD29B01AC01C301B2010E945DD46E
:100C10004B015C016EE2CE010E945C85E80EF91E7C
:100C2000115020F120E030E040E251E4C501B40170
:100C30000E94D0D22B013C010E9443D54B01B12C24
:100C4000A12C2AE0B501A401CE010E940C85E80E7A
:100C5000F91EC501B4010E946FD29B01AC01C30112
:100C6000B2010E945DD44B015C01DACFC701DF9174
:100C7000CF911F91FF90EF90DF90CF90BF90AF90FA
:100C80009F908F907F906F905F904F903F902F90AC
:100C90000895CF92DF92EF92FF920F931F93CF931D
:100CA000DF932115310581F4DC01ED91FC91019078
:100CB000F081E02D642FDF91CF911F910F91FF9074
:100CC000EF90DF90CF9019942A30310501F52AE09A
:100CD00077FF1DC06A017B01EC016DE20E945C851B
:100CE0008C0144275527BA014C195D096E097F090B
:100CF0002AE0CE010E940C85800F911FDF91CF91D9
:100D00001F910F91FF90EF90DF90CF900895DF91AA
:100D1000CF911F910F91FF90EF90DF90CF900C94A7
:100D20000C858F929F92AF92BF92CF92DF92EF92FB
:100D3000FF920F931F93CF93DF937C018B014C01A4
:100D400082E0880E911C5701E5E0AE0EB11CD0E0A8
:100D5000C0E0F40161914F01C8010E94369D6C0111
:100D60006EE2C8010E945C858C0D9D1DC80FD91FC5
:100D70008A149B0471F7F7016581C8010E94369DB2
:100D80008C0F9D1FDF91CF911F910F91FF90EF90DE
:100D9000DF90CF90BF90AF909F908F900895611596
:100DA000710511F00C94D77D90E080E008950F93C9
:100DB0001F93CF93DF93EC018B0161E775E00E94F5
:100DC000CF8601151105C1F1F80161918F016623EC
:100DD00099F1603240F0623231F06C3521F0CE0191
:100DE0000E945C85F1CF6CE5CE010E945C85F80124
:100DF000319780818C30D1F044F48930D9F08A3039
:100E0000B9F0883009F762E6EACF823259F024F46B
:100E100062E78D3021F3D8CF8F3231F06CE58C351D
:100E2000F1F2D2CF62E2DBCF6FE2D9CF66E6D7CF65
:100E30006EE6D5CF64E7D3CF62E2CE010E945C8537
:100E400090E080E0DF91CF911F910F910895DB0139
:100E500014964D915C9115976D917C91DC01ED910B
:100E6000FC910280F381E02D1994EF92FF920F9391
:100E70001F93CF93DF938C017B01D0E0C0E0F7019B
:100E8000EC0FFD1F6491662361F0D801ED91FC9198
:100E90000190F081E02DC8011995892B11F0219660
:100EA000EECFCE01DF91CF911F910F91FF90EF9088
:100EB00008950F931F93CF93DF93EC010E94358722
:100EC0008C01CE010E945885800F911FDF91CF9138
:100ED0001F910F91089582EA99E00E94588569EC6C
:100EE0007AE182EA99E00C943587DC0187EE93E0A1
:100EF0008D939D9384E0FB0101900D928A95E1F71B
:100F000008953F924F925F926F927F928F929F923D
:100F1000AF92BF92CF92DF92EF92FF920F931F9307
:100F2000CF93DF93CDB7DEB7EA970FB6F894DEBF65
:100F30000FBECDBF7C012A013B0169010E9458A66A
:100F40004B015C0187010D5B1F4FC8010E94B8185F
:100F500018161906ACF00E9458A6681979098A0972
:100F60009B09461657066806790608F468C10E9470
:100F7000186861E070E080E090E00E9425A6E5CF6F
:100F800042E250E0BE016F5F7F4FC8010E944318EC
:100F900089818230D1F0312C832DEA960FB6F894F6
:100FA000DEBF0FBECDBFDF91CF911F910F91FF909C
:100FB000EF90DF90CF90BF90AF909F908F907F90F9
:100FC0006F905F904F903F900895F80184899589C4
:100FD0008334910501F76D817E818F8198850E9410
:100FE00047D44B015C01F60180829182A282B382D8
:100FF00046E050E0B701685F7F4FCE014D960E94FA
:101000004FD8892B41F6F70180819181A281B3816C
:1010100088169906AA06BB0608F4BDCF848195817F
:10102000A681B78188159905AA05BB0508F4B3CF39
:1010300089899A89AB89BC8986879787A08BB18B70
:101040004EEC50E070E060E0C8010E944318312C83
:10105000C701829698AB8FA7F701B696FAABE9ABBA
:1010600008969CAB8BAB67019AE1C90ED11CBD966B
:10107000FEABEDABC701429698AF8FABFD97FAAFD1
:10108000E9AF4701FEE18F0E911CF801818D928D31
:10109000181619060CF080CFC8010E94621883331D
:1010A000910509F4B2C014F58130910509F464C0CA
:1010B00044F4892B51F3C8010E946218AC015527F2
:1010C00075C08330910509F462C00697A1F7C80185
:1010D0000E946218B82E44E050E0B401C8010E949A
:1010E0004318EB2DE450FF0BAF0160C08A3391052C
:1010F00009F45FC084F585339105B1F1C697D9F63F
:10110000C8010E9462185C01B601CE0189960E9456
:1011100075878BA59CA5ADA5BEA5892B8A2B8B2B8E
:10112000B1F0EDA9FEA94080518062807380B601C4
:10113000CE0183960E9475878DA19EA1AFA1B8A50F
:10114000A501481659066A067B0609F0B8CF44E0A7
:1011500050E0B60118C08B33910509F440C08F3FB1
:10116000910509F492CFA7CFC8010E946218C80167
:101170000E946218382E89CFC8010E94621844E08C
:1011800050E06FA978ADC8010E9443187ECFC80116
:101190000E946218B82E44E050E069AD7AADC801F3
:1011A0000E9443188B2D8450990BAC0170E060E0D5
:1011B000EACFC8010E94621844E050E069A97AA908
:1011C000C8010E944318F70166A177A180A591A5E7
:1011D0000E9447D466A377A380A791A756CFC801E2
:1011E0000E94621844E050E06BA97CA9C8010E94EB
:1011F0004318F70162A573A584A595A50E9447D45D
:1012000062A773A784A795A740CFC8010E94621860
:1012100044E050E06FA578A9C8010E944318F70187
:1012200062A173A184A195A10E9447D462A373A374
:1012300084A395A366A777A780AB91AB26CF332471
:101240003A94AACE2F923F924F925F926F927F92E2
:101250008F929F92AF92BF92CF92DF92EF92FF92C6
:101260000F931F93CF93DF9300D000D0CDB7DEB79D
:101270008C010E94ADCB2FEC37E040E050E00E94A3
:10128000D6D3DC01CB010196A11DB11DF8018483E9
:101290009583A683B78380839183A283B383580108
:1012A000F3E4AF0EB11CC5010E940D1864E470E0B8
:1012B000C5010E948719882309F445C10E9458A6D8
:1012C0002B013C01480182E4880E911C48EEC42E9B
:1012D00043E0D42EE12CF12C52E0252E1E821D82FB
:1012E000D4018C918330B1F1811166C0F801848101
:1012F0009581A681B7810196A11DB11D8483958337
:10130000A683B7830E9458A66419750986099709B0
:10131000A70196010E94B4D3A90161E0C8010E940F
:10132000117F81E0D4018C938D819E810197C1F260
:101330000E9458A66419750986099709D801D6969E
:101340002D913D914D915C91D9972617370748070C
:10135000590720F6C5010E940D18F8018481958176
:10136000A681B7810196A11DB11D84839583A683B3
:10137000B7830E9458A6F801FE966083718382832A
:1013800093838D819E8126960FB6F894DEBF0FBEA3
:10139000CDBFDF91CF911F910F91FF90EF90DF9024
:1013A000CF90BF90AF909F908F907F906F905F9005
:1013B0004F903F902F9008958430F1F4F80184818C
:1013C0009581A681B7810196A11DB11D8483958366
:1013D000A683B7830E9458A66419750986099709E0
:1013E000A70196010E94B4D3A90163E0C8010E943D
:1013F000117FD4012C9298CF813051F5F80142AD84
:1014000053AD64AD75AD9E012F5F3F4FC8010E9483
:101410008187382EF2E08F1390C089819A81AB8149
:10142000BC81F80184839583A683B7830E9458A664
:101430006419750986099709A70196010E94B4D31A
:10144000A90163E0C8010E94117FD4013C926CCFD6
:10145000823009F069CFF80142AD53AD64AD75AD8E
:101460009E012F5F3F4FC8010E948187382EF5E013
:101470008F135DC0E3E0D401EC93F80182A193A146
:10148000A4A1B5A1892B8A2B8B2B41F484E893E08E
:10149000A0E0B0E082A393A3A4A3B5A3F80186A122
:1014A00097A1A0A5B1A5892B8A2B8B2B61F482A1D2
:1014B00093A1A4A1B5A1B695A7959795879586A365
:1014C00097A3A0A7B1A7F80182A593A5A4A5B5A548
:1014D000892B8A2B8B2BA9F482A193A1A4A1B5A15E
:1014E000AC01BD0123E076956795579547952A9500
:1014F000D1F7841B950BA60BB70B82A793A7A4A7C4
:10150000B5A7F80186A197A1A0A5B1A586A797A721
:10151000A0ABB1AB82A593A5A4A5B5A582AB93ABB7
:10152000A4ABB5AB81E090E09E838D83FDCE96E0C9
:10153000891303C0D4011C92F7CEBFEF3B12F4CE47
:10154000F4011082F1CE1E821D821BCF1F920F92DA
:101550000FB60F9211240BB60F922F933F934F9318
:101560005F936F937F938F939F93AF93BF93EF930B
:10157000FF9382EA99E00E94AB7AFF91EF91BF91CD
:10158000AF919F918F917F916F915F914F913F911B
:101590002F910F900BBE0F900FBE0F901F901895BC
:1015A0001F920F920FB60F9211240BB60F922F932A
:1015B0008F939F93EF93FF93E091B209F091B3095A
:1015C0008081E091B809F091B90982FD1DC0908138
:1015D0008091BB098F5F8F732091BC09821741F006
:1015E000E091BB09F0E0EE55F64F958F8093BB0973
:1015F000FF91EF919F918F912F910F900BBE0F90C4
:101600000FBE0F901F9018958081F2CFDF92EF925E
:10161000FF920F931F93CF93DF9300D000D0CDB7ED
:10162000DEB78B017A01D22E6FE875E0CE0101960C
:101630000E9407839E012F5F3F4F4D2DB701C801C8
:101640000E94C5AFCE0101960E94C88226960FB6B1
:10165000F894DEBF0FBECDBFDF91CF911F910F91E8
:10166000FF90EF90DF900895CF92DF92EF92FF927C
:101670000F931F93CF93DF93CDB7DEB7EC970FB6E1
:10168000F894DEBF0FBECDBFDC012C91222309F4FC
:1016900059C067E574E00E94BBCC9A8389837E01C0
:1016A000B3E0EB0EF11C01E010E0D02EC12E67E597
:1016B00074E090E080E00E94BBCCF70181939193AD
:1016C0007F010E31110521F00F5F1F4F892B69F744
:1016D0000091AA071091AB07E980FA800115110566
:1016E00049F1D8016D917C91C7010E94A0D8892B46
:1016F000E9F4D8011296ED91FC91BE016F5F7F4F26
:101700008D2D9C2D19958C010E946B87C801EC963C
:101710000FB6F894DEBF0FBECDBFDF91CF911F9102
:101720000F91FF90EF90DF90CF900895F801048122
:101730001581D4CF6DEC7AE182EA99E00E94598755
:101740000E946B8710E000E0E1CFCF9382EA99E03E
:101750000E94957A892BE9F182EA99E00E94737AD6
:10176000C82F8A3089F08D3079F0883001F568E033
:1017700082EA99E00E945C858091AE07882331F36C
:1017800081508093AE07E2CFE091AE07F0E0E259DE
:10179000F84F10826DE875E082EA99E00E94CF86EA
:1017A0008EE697E00E94348B1092AE07CFCF682F61
:1017B00082EA99E00E945C85E091AE07EB3330F657
:1017C00081E08E0F8093AE07F0E0E259F84FC083BE
:1017D000BDCFCF910895CF93DF930E94E87DEC01B8
:1017E000892B99F08A8181508A8381110EC088816A
:1017F00099810E94D8CA19821882E0916C07F091F1
:101800006D07C9E6D7E0309719F4DF91CF910895BD
:101810009381848120813181232B41F49B838C83AC
:10182000CF010E94D8CA9B818C81FE01EF01E92F74
:10183000F82FE9CFEF92FF920F931F93CF93DF938F
:101840007C010E94E87DFC01892B61F082818F5F21
:10185000828380819181DF91CF911F910F91FF90C1
:10186000EF900895C9E6D7E088819981892B51F4DA
:10187000C7010E9435D89983888321E02A83EBCF62
:10188000EC01F2CF8B819C810097D1F785E090E04D
:101890000E943CCA8C0190E080E001151105D9F24C
:1018A0001C830B83C7010E9435D8F8019183808384
:1018B00021E0228314821382CECF8F929F92AF9227
:1018C000BF92CF92DF92EF92FF920F931F93CF932D
:1018D000DF936115710509F48FC0DB011896EC9157
:1018E0001897EF70E73008F087C0EC01F0E0882728
:1018F000E358F3478F4F0C943FD4848C958C9E8C87
:10190000B58CFF8C118D4A8D6CE975E0CE01DF91AD
:10191000CF911F910F91FF90EF90DF90CF90BF90EC
:10192000AF909F908F900C94D77D19968C9166EA1A
:1019300075E0882359F361EA75E0E8CF19964D9177
:101940005D916D917C911C972AE030E0CE01DF9192
:10195000CF911F910F91FF90EF90DF90CF90BF90AC
:10196000AF909F908F900C9449861996CD90DD9002
:10197000ED90FC901C9720E030E0A901C701B60172
:101980000E946AD287FF09C06DEF73E0CE010E940A
:10199000CF86F7FAF094F7F8F094C701B6010E94E9
:1019A00043D54B015C01BC01A401CE010E94339DD3
:1019B00064E875E0CE010E94CF86C501B4010E94A3
:1019C0006FD29B01AC01C701B6010E945DD42DEC22
:1019D0003CEC4CE45DE30E945ED420E030E040E269
:1019E00051E40E94D0D20E9443D5AB0170E060E088
:1019F0002AE0CE010E940C8590E080E01DC019967F
:101A00006D917C91CE01DF91CF911F910F91FF904D
:101A1000EF90DF90CF90BF90AF909F908F900C94FD
:101A2000D78616960D911C916BE5CE010E945C85C0
:101A3000019679F48FEF9FEFDF91CF911F910F9176
:101A4000FF90EF90DF90CF90BF90AF909F908F90DE
:101A500008950115110579F0B801CE010E945D8C41
:101A6000019641F3D80112960D911C9101151105B3
:101A700011F06CE2DACF6DE5CE010E945C8521E0C9
:101A800030E0019611F030E020E088279927821B92
:101A9000930BD2CF16960D911C916BE7CE010E944D
:101AA0005C85019639F20115110529F1D8016D9176
:101AB0007C91CE010E94D786019609F4BBCF6AE3E0
:101AC000CE010E945C85019609F4B4CFB801CE0125
:101AD0000E945D8C019609F4ADCFD80112960D914C
:101AE0001C910115110539F06CE2CE010E945C8554
:101AF0000196C9F69FCF6DE7BFCF0F931F93CF938A
:101B0000DF93EC01E881F9810284F385E02D1995DA
:101B100000E011E08F3F9807D1F081329105E4F4A5
:101B200001501109E881F9810F3F100731F002845B
:101B3000F385E02DCE011995EDCFE881F98106847A
:101B4000F785E02D682FCE01199590E080E0DF91B8
:101B5000CF911F910F910895012B79F78FEF9FEF90
:101B6000F6CFCF92DF92EF92FF920F931F93CF9316
:101B7000DF937C016B01DC01ED91FC910284F38524
:101B8000E02D1995829761F0CFEFDFEFCE01DF9165
:101B9000CF911F910F91FF90EF90DF90CF9008951C
:101BA00084E0F601808786E090E00E943CCA8C01C8
:101BB000009751F3E9E2F7E0DC01ED93FC9380E458
:101BC000DF011D928A95E9F780E490E0F8019383A4
:101BD000828315821482D701ED91FC910284F385F2
:101BE000E02DC7011995EC010196C9F0C232D1056B
:101BF00009F44DC0C032D1050CF449C0B8018C2F96
:101C0000CC35D10549F5D701ED91FC910284F385DE
